:020000040800F2
:1000000000060020E1010008E3010008E301000808
:10001000E3010008E3010008E3010008E301000830
:10002000E3010008E3010008E30100086D2F000868
:10003000E3010008E3010008E3010008E301000810
:10004000E3010008E3010008E3010008E301000800
:10005000E3010008E3010008153200083D32000802
:10006000653200088D320008B5320008E30100084F
:10007000E3010008E3010008E3010008E3010008D0
:10008000E3010008E3010008E3010008E3010008C0
:10009000E3010008E3010008E3010008DD32000885
:1000A000E3010008E3010008E3010008E3010008A0
:1000B000B1330008E3010008E3010008E301000890
:1000C000E3010008E3010008E3010008E301000880
:1000D000E3010008E3010008E3010008E301000870
:1000E00041330008E3010008E3010008E3010008D0
:1000F000E3010008E3010008E3010008E301000850
:10010000E3010008E3010008E3010008E30100083F
:10011000E3010008E3010008E3010008E30100082F
:10012000E3010008E3010008E3010008E30100081F
:10013000E3010008E3010008E3010008E30100080F
:10014000E3010008E3010008E3010008212700089B
:10015000E3010008E3010008E3010008E3010008EF
:10016000E3010008E3010008E3010008E3010008DF
:10017000E3010008E3010008E3010008E3010008CF
:10018000E3010008E3010008E3010008E3010008BF
:10019000E3010008E3010008E3010008E3010008AF
:1001A000E3010008E3010008E3010008E30100089F
:1001B000E3010008E3010008E3010008E30100088F
:1001C000E3010008E3010008E3010008E30100087F
:1001D000E3010008E3010008E3010008E30100086F
:1001E00002E000F000F8FEE772B6374880F30888B6
:1001F000364880F3098836483649086040F20000E6
:10020000CCF200004EF63471CEF200010860BFF36C
:100210004F8FBFF36F8F40F20000C0F2F0004EF638
:100220008851CEF200010860BFF34F8FBFF36F8F8C
:100230004FF00000E1EE100A4EF63C71CEF20001E4
:100240000860062080F31488BFF36F8F01F030FF41
:1002500002F02AFE4FF055301F491B4A91423CBF25
:1002600041F8040BFAE71D49184A91423CBF41F896
:10027000040BFAE71A491B4A1B4B9A423EBF51F83E
:10028000040B42F8040BF8E700201849184A914281
:100290003CBF41F8040BFAE701F00EFF02F058FEF4
:1002A000144C154DAC4203DA54F8041B8847F9E7A7
:1002B00000F042F8114C124DAC4203DA54F8041B22
:1002C0008847F9E701F0F6BE000600200022002072
:1002D0000000000808ED00E00000002000060020FB
:1002E0007837000800220020402200204022002011
:1002F000602E0020E0010008E0010008E001000895
:10030000E00100082DE9F04F2DED108AC1F80CD066
:10031000C3689D46BDEC108ABDE8F08F002383F3CF
:1003200011882846A047002001F072FAFEE701F08C
:1003300001FA00DFFEE7000038B500F0BBFB01F07A
:1003400087FE054601F0AAFE0446C8B90E4B9D4241
:1003500018D001339D4218BF044641F2883504BFCE
:1003600001240025002001F07DFE0CB100F074F89E
:1003700000F000FD284600F0BFF800F06DF8F9E746
:100380000025EFE70546EDE7010007B008B500F0EE
:1003900063FBA0F120035842584108BD07B541F264
:1003A0001203022101A8ADF8043000F073FB03B082
:1003B0005DF804FB38B5302383F3118817480368D0
:1003C0000BB101F0F1FA164A144800234FF47A7188
:1003D00001F0E0FA002383F31188124C236813B173
:1003E0002368013B2360636813B16368013B63606A
:1003F0000D4D2B7833B963687BB9022000F024FCE3
:10040000322363602B78032B07D163682BB902205A
:1004100000F01AFC4FF47A73636038BD402200206C
:10042000B50300086023002058220020084B1870F4
:1004300003280CD8DFE800F008050208022000F0CD
:10044000F9BB022000F0ECBB024B00225A6070475F
:100450005822002060230020234B244A10B51C465C
:10046000196801313FD004339342F9D16268A24246
:1004700039D31F4B9B6803F1006303F540439A4255
:1004800031D2002000F030FB0220FFF7CFFF194BE4
:100490001A6C00221A64196E1A66196E596C5A6425
:1004A000596E5A665A6E5A6942F080025A615A6908
:1004B00022F080025A615A691A6942F000521A61A8
:1004C0001A6922F000521A611B6972B64FF0E023DC
:1004D0003021C3F8084DD4E9003281F311889D46DC
:1004E00083F30888104710BD00C0000820C0000832
:1004F00000220020003802402DE9F04F93B0AA4BB3
:1005000000902022FF210AA89D6800F0DDFBA74A89
:100510001378A3B9A648012103601170302383F337
:10052000118803680BB101F03FFAA24AA0480023EA
:100530004FF47A7101F02EFA002383F31188009BA7
:1005400013B19D4B009A1A609C4A009C1378032BB0
:100550001EBF00231370984A4FF0000A18BF536063
:10056000D3465646D146012000F064FB24B1924B9D
:100570001B68002B00F01182002000F06DFA039040
:10058000039B002BF2DB012000F04AFB039B213B85
:10059000162BE8D801A252F823F000BFF905000895
:1005A00021060008B5060008670500086705000871
:1005B000670500083F0700080F0900082908000820
:1005C0008B080008B3080008D90800086705000870
:1005D000EB080008670500085D0900089906000897
:1005E00067050008A109000805060008990600082B
:1005F000670500088B0800080220FFF7C7FE0028E7
:1006000040F0F581009B0221BAF1000F08BF1C46A3
:1006100005A841F21233ADF8143000F03BFAA2E71E
:100620004FF47A7000F018FA071EEBDB0220FFF798
:10063000ADFE0028E6D0013F052F00F2DA81DFE8A9
:1006400007F0030A0D10133605230593042105A8AE
:1006500000F020FA17E054480421F9E75848042133
:10066000F6E758480421F3E74FF01C08404600F035
:100670003DFA08F104080590042105A800F00AFAE3
:10068000B8F12C0FF2D1012000FA07F747EA0B0B63
:100690005FFA8BFB4FF0000900F062FB26B10BF014
:1006A0000B030B2B08BF0024FFF778FE5BE74648DF
:1006B0000421CDE7002EA5D00BF00B030B2BA1D10D
:1006C0000220FFF763FE074600289BD0012000F0C0
:1006D0000BFA0220FFF7AAFE00261FFA86F8404612
:1006E00000F012FA044690B10021404600F01CFAD6
:1006F00001360028F1D1BA46044641F21213022114
:1007000005A8ADF814303E4600F0C4F92BE70120EF
:10071000FFF78CFE2546244B9B68AB4207D9284641
:1007200000F0E4F9013040F067810435F3E7234B32
:1007300000251D70204BBA465D603E46ACE7002E9A
:100740003FF460AF0BF00B030B2B7FF45BAF022089
:10075000FFF76CFE322000F07FF9B0F10008FFF6E1
:1007600051AF18F003077FF44DAF0F4A926808EBC2
:10077000050393423FF646AFB8F5807F3FF742AF9F
:10078000124B0193B84523DD4FF47A7000F064F901
:100790000390039A002AFFF635AF019B039A03F8F2
:1007A000012B0137EDE700BF002200205C23002071
:1007B00040220020B50300086023002058220020BA
:1007C00004220020082200200C2200205C220020AD
:1007D000C820FFF7DBFD074600283FF413AF1F2DAD
:1007E00011D8C5F1200242450AAB25F0030028BF0D
:1007F000424683490192184400F040FA019A804829
:10080000FF2100F061FA4FEAA8037D490193C8F384
:100810008702284600F060FA064600283FF46DAFD4
:10082000019B05EB830537E70220FFF7AFFD0028AA
:100830003FF4E8AE00F0A4F900283FF4E3AE00274F
:10084000B846704B9B68BB4218D91F2F11D80A9B22
:1008500001330ED027F0030312AA134453F8203CAF
:1008600005934046042205A900F0AEFA04378046FD
:10087000E7E7384600F03AF90590F2E7CDF8148042
:10088000042105A800F006F906E70023642104A866
:10089000049300F0F5F800287FF4B4AE0220FFF7CF
:1008A00075FD00283FF4AEAE049800F051F90590B4
:1008B000E6E70023642104A8049300F0E1F800288F
:1008C0007FF4A0AE0220FFF761FD00283FF49AAE4E
:1008D000049800F04DF9EAE70220FFF757FD0028E1
:1008E0003FF490AE00F05CF9E1E70220FFF74EFD27
:1008F00000283FF487AE05A9142000F057F9042121
:100900000746049004A800F0C5F83946B9E732203C
:1009100000F0A2F8071EFFF675AEBB077FF472AEBB
:10092000384A926807EB090393423FF66BAE022008
:10093000FFF72CFD00283FF465AE27F003074F4476
:10094000B9453FF4A9AE484600F0D0F8042105901F
:1009500005A800F09FF809F10409F1E74FF47A7057
:10096000FFF714FD00283FF44DAE00F009F9002810
:1009700044D00A9B01330BD008220AA9002000F0C2
:10098000ABF900283AD02022FF210AA800F09CF9F8
:10099000FFF704FD1C4800F041FF13B0BDE8F08FE5
:1009A000002E3FF42FAE0BF00B030B2B7FF42AAE7F
:1009B0000023642105A8059300F062F8074600288B
:1009C0007FF420AE0220FFF7E1FC804600283FF4D0
:1009D00019AEFFF7E3FC41F2883000F01FFF0598E5
:1009E00000F0F0F9464600F0BBF93C46BBE5064690
:1009F00052E64FF0000905E6BA467EE637467CE649
:100A00005C22002000220020A086010070B50F4B60
:100A10001B780133DBB2012B0C4611D80C4D296831
:100A20004FF47A730E6AA2FB03320146224628462F
:100A3000B047844204D1074B00221A70012070BDD8
:100A40004FF4FA7000F0EAFE0020F8E710220020D0
:100A5000082600209423002007B500230246012128
:100A60000DF107008DF80730FFF7D0FF20B19DF89A
:100A7000070003B05DF804FB4FF0FF30F9E700001A
:100A80000A4608B50421FFF7C1FF80F00100C0B29B
:100A9000404208BD30B4054C2368DD69044B0A466A
:100AA000AC460146204630BC604700BF0826002007
:100AB000A086010070B501F0D1F9094E094D3080D2
:100AC000002428683388834208D901F0C1F92B68D3
:100AD00004440133B4F5404F2B60F2D370BD00BF26
:100AE000962300206823002001F066BA00F1006020
:100AF00000F540400068704700F10060920000F58A
:100B0000404001F0F1B90000054B1A68054B1B8805
:100B10009B1A834202D9104401F09AB90020704711
:100B2000682300209623002038B5084D044629B1DB
:100B300028682044BDE8384001F0AAB9286820445C
:100B400001F08EF90028F3D038BD00BF68230020E3
:100B500010F003030AD1B0F5047F05D200F1005074
:100B6000A0F51040D0F80038184670470023FBE786
:100B700000F10050A0F51040D0F8100A70470000B6
:100B8000064991F8243033B10023086A81F82430F3
:100B90000822FFF7B1BF0120704700BF6C2300207F
:100BA000014B1868704700BF002004E070B5194B76
:100BB0001D68194B0138C5F30B0408442D0C0422A1
:100BC0001E88A6420BD15C680A46013C824213464D
:100BD0000FD214F9016F4EB102F8016BF6E7013A3A
:100BE00003F10803ECD181420B4602D22C2203F818
:100BF000012B0A4A05241688AE4204D1984284BFCC
:100C0000967803F8016B013C02F10402F3D1581A03
:100C100070BD00BF002004E0943400088034000858
:100C2000022802BF024B4FF000529A61704700BF8A
:100C300000000240022802BF024B4FF400529A61AA
:100C4000704700BF00000240022801BF024A5369FA
:100C500083F40053536170470000024070B50446AE
:100C60004FF47A764CB1412C254628BF412506FB2E
:100C700005F000F0D3FD641BF4E770BD10B5002350
:100C8000934203D0CC5CC4540133F9E710BD00009B
:100C900010B5013810F9013F3BB191F900409C4279
:100CA00003D11AB10131013AF4E71AB191F90020E8
:100CB000981A10BD1046FCE703460246D01A12F9F6
:100CC000011B0029FAD1704702440346934202D027
:100CD00003F8011BFAE770472DE9F8431F4D14464E
:100CE00095F824200746884652BBDFF870909CB3E5
:100CF00095F824302BB92022FF2148462F62FFF7B8
:100D0000E3FF95F82400C0F10802A24228BF224662
:100D1000D6B24146920005EB8000FFF7AFFF95F891
:100D20002430A41B1E44F6B2082E17449044E4B2AB
:100D300085F82460DBD1FFF723FF0028D7D108E036
:100D40002B6A03EB82038342CFD0FFF719FF002801
:100D5000CBD10020BDE8F8830120FBE76C23002005
:100D6000024B1A78024B1A70704700BF9423002080
:100D70001022002010B5104C104800F0B5F82146A4
:100D80000E4800F0DDF82468626DD2F8043843F0B4
:100D90000203C2F804384FF47A70FFF75FFF084986
:100DA000204600F0D3F9626DD2F8043823F0020334
:100DB000C2F8043810BD00BF6035000808260020C6
:100DC000683500087047000030B5094D0A4491426B
:100DD0000DD011F8013B5840082340F30004013BBB
:100DE0002C4013F0FF0384EA5000F6D1EFE730BD4A
:100DF0002083B8ED026843681143016003B11847CE
:100E00007047000013B5446BD4F894341A68117815
:100E1000042915D1217C022912D1197912890123C3
:100E20008B4013420CD101A904F14C0001F0F8FEF3
:100E3000D4F89444019B21790246206800F0D0F94F
:100E400002B010BD143001F07BBE00004FF0FF3344
:100E5000143001F075BE00004C3001F04DBF0000B1
:100E60004FF0FF334C3001F047BF0000143001F069
:100E700049BE00004FF0FF31143001F043BE0000C6
:100E80004C3001F019BF00004FF0FF324C3001F040
:100E900013BF00000020704710B5D0F894341A68D2
:100EA00011780429044617D1017C022914D15979FB
:100EB000528901238B4013420ED1143001F0DCFD26
:100EC000024648B1D4F894444FF4807361792068A5
:100ED000BDE8104000F072B910BD0000406BFFF794
:100EE000DBBF0000704700007FB5124B036000239A
:100EF0004360C0E90233012502260F4B0574044606
:100F00000290019300F18402294600964FF4807309
:100F1000143001F08DFD094B0294CDE9006304F516
:100F200023724FF48073294604F14C0001F054FE03
:100F300004B070BDB4340008DD0E0008050E0008D2
:100F40000B68302282F311880A7903EB82029061E8
:100F50004A79093243F822008A7912B103EB8203FD
:100F600098610223C0F894140374002080F3118860
:100F70007047000038B5037F044613B190F8543031
:100F8000ABB9201D01250221FFF734FF04F1140045
:100F900025776FF0010100F069FC84F8545004F1EA
:100FA0004C006FF00101BDE8384000F05FBC38BD77
:100FB00010B5012104460430FFF71CFF00232377FE
:100FC00084F8543010BD000038B5044600251430B4
:100FD00001F046FD04F14C00257701F015FE201DBF
:100FE00084F854500121FFF705FF2046BDE8384042
:100FF000FFF752BF90F8443003F06003202B07D175
:1010000090F84520212A4FF0000303D81F2A06D864
:1010100000207047222AFBD1C0E90E3303E0034AC7
:1010200082630722C26303640120704711220020FB
:1010300037B5D0F894341A681178042904461AD1C7
:10104000017C022917D11979128901238B4013429F
:1010500011D100F14C05284601F096FE58B101A9C6
:10106000284601F0DDFDD4F89444019B2179024625
:10107000206800F0B5F803B030BD0000F0B500EB1B
:10108000810385B09E6904460D46FEB1302383F38B
:10109000118804EB8507301D0821FFF7ABFEFB68C4
:1010A0005B691B6806F14C001BB1019001F0C6FDA5
:1010B000019803A901F0B4FD024648B1039B2946FB
:1010C000204600F08DF8002383F3118805B0F0BDB1
:1010D000FB685A691268002AF5D01B8A013B13404D
:1010E000F1D104F14402EAE7093138B550F8214062
:1010F000DCB1302383F31188D4F894241368527937
:1011000003EB8203DB689B695D6845B104216018CD
:10111000FFF770FE294604F1140001F0B7FC2046E9
:10112000FFF7BAFE002383F3118838BD7047000033
:1011300001F016B8012303700023C0E90133C36135
:1011400083620362C36243620363704738B5044637
:10115000302383F311880025C0E90355C0E9055504
:10116000416001F00DF80223237085F311882846B1
:1011700038BD000070B500EB810305465069DA60A8
:101180000E46144618B110220021FFF79DFDA069FC
:1011900018B110220021FFF797FD31462846BDE81F
:1011A000704001F0B7B80000826802F0011282605E
:1011B0000022C0E90422826101F038B9F0B400EBEA
:1011C00081044789E4680125A4698D403D43458138
:1011D00023600023A2606360F0BC01F053B90000FB
:1011E000F0B400EB81040789E468012564698D404F
:1011F0003D43058123600023A2606360F0BC01F0E1
:10120000CDB9000070B50223002504460370C0E983
:101210000255C0E90455C564856180F8345001F079
:1012200015F863681B6823B129462046BDE8704065
:10123000184770BD0378052B10B504460AD080F816
:1012400050300523037043681B680BB10421984795
:101250000023A36010BD00000178052906D190F895
:101260005020436802701B6803B1184770470000A4
:1012700070B590F83430044613B1002380F8343050
:1012800004F14402204601F0F3F863689B68B3B9A7
:1012900094F8443013F0600535D00021204601F069
:1012A00093FB0021204601F085FB63681B6813B1A6
:1012B000062120469847062384F8343070BD204626
:1012C00098470028E4D0B4F84A30E26B9A4288BFCD
:1012D000E36394F94430E56B002B4FF0300380F268
:1012E0000381002D00F0F280092284F8342083F37A
:1012F00011880021D4E90E232046FFF771FF002357
:1013000083F31188DAE794F8452003F07F0343EA7A
:10131000022340F20232934200F0C58021D8B3F597
:10132000807F48D00DD8012B3FD0022B00F0938056
:10133000002BB2D104F14C02A2630222E2632364C7
:10134000C1E7B3F5817F00F09B80B3F5407FA4D166
:1013500094F84630012BA0D1B4F84C3043F002038E
:1013600032E0B3F5006F4DD017D8B3F5A06F31D090
:10137000A3F5C063012B90D8636894F846205E689B
:1013800094F84710B4F848302046B047002884D07D
:101390004368A3630368E3631AE0B3F5106F36D0C4
:1013A00040F6024293427FF478AF5C4BA363022382
:1013B000E3630023C3E794F84630012B7FF46DAF5D
:1013C000B4F84C3023F00203C4E90E55A4F84C30B5
:1013D000256478E7B4F84430B3F5A06F0ED194F8E3
:1013E000463084F84E30204600F088FF63681B6862
:1013F00013B1012120469847032323700023C4E939
:101400000E339CE704F14F03A3630123C3E7237862
:10141000042B10D1302383F311882046FFF7C4FE3C
:1014200085F311880321636884F84F5021701B688D
:101430000BB12046984794F84630002BDED084F854
:101440004F300423237063681B68002BD6D0022121
:1014500020469847D2E794F848301D0603F00F0164
:1014600020460AD500F0F6FF012804D002287FF4B8
:1014700014AF2B4B9AE72B4B98E700F0DDFFF3E717
:1014800094F84630002B7FF408AF94F8483013F0FE
:101490000F01B3D01A06204602D501F0A9FAADE734
:1014A00001F09CFAAAE794F84630002B7FF4F5AEE1
:1014B00094F8483013F00F01A0D01B06204602D547
:1014C00001F082FA9AE701F075FA97E7142284F89E
:1014D000342083F311882B462A4629462046FFF7FD
:1014E0006DFE85F31188E9E65DB1152284F834209C
:1014F00083F311880021D4E90E232046FFF75EFE16
:10150000FDE60B2284F8342083F311882B462A460B
:1015100029462046FFF764FEE3E700BFE4340008F5
:10152000DC340008E034000838B590F83430044664
:10153000002B3ED0063BDAB20F2A34D80F2B32D81C
:10154000DFE803F0373131082232313131313131C6
:1015500031313737C56BB0F84A309D4214D2C36879
:101560001B8AB5FBF3F203FB12556DB9302383F3ED
:1015700011882B462A462946FFF732FE85F311884B
:101580000A2384F834300EE0142384F834303023F6
:1015900083F3118800231A4619462046FFF70EFEF2
:1015A000002383F3118838BD036C03B198470023EF
:1015B000E7E70021204601F007FA0021204601F06C
:1015C000F9F963681B6813B1062120469847062382
:1015D000D7E7000010B590F83430142B044629D01A
:1015E00017D8062B05D001D81BB110BD093B022B23
:1015F000FBD80021204601F0E7F90021204601F048
:10160000D9F963681B6813B1062120469847062361
:1016100019E0152BE9D10B2380F83430302383F304
:10162000118800231A461946FFF7DAFD002383F3D9
:101630001188DAE7C3689B695B68002BD5D1036C1E
:1016400003B19847002384F83430CEE700230375B4
:10165000826803691B6899689142FBD25A680360EB
:101660004260106058607047002303758268036908
:101670001B6899689142FBD85A6803604260106009
:101680005860704708B50846302383F311880B7DF6
:10169000032B05D0042B0DD02BB983F3118808BD83
:1016A0008B6900221A604FF0FF338361FFF7CEFF92
:1016B0000023F2E7D1E9003213605A60F3E700003B
:1016C000FFF7C4BF054BD9680875186802681A602F
:1016D000536001220275D860FEF714BE98230020E3
:1016E00030B50C4BDD684B1C87B004460FD02B4641
:1016F000094A684600F04EF92046FFF7E3FF009BD9
:1017000013B1684600F050F9A86907B030BDFFF783
:10171000D9FFF9E79823002085160008044B1A68C2
:10172000DB6890689B68984294BF00200120704756
:1017300098230020084B10B51C68D86822681A60EE
:10174000536001222275DC60FFF78EFF01462046C0
:10175000BDE81040FEF7D6BD9823002038B5074CF1
:1017600007490848012300252370656001F044FB08
:101770000223237085F3118838BD00BF00260020A6
:10178000EC3400089823002000F044B9034A516863
:1017900053685B1A9842FBD8704700BF001000E006
:1017A0008B60022308618B82084670478368A3F12F
:1017B000840243F8142C026943F8442C426943F82C
:1017C000402C094A43F8242CC26843F8182C022202
:1017D00003F80C2C002203F80B2C044A43F8102CBD
:1017E000A3F12000704700BF1D03000898230020CC
:1017F00008B5FFF7DBFFBDE80840FFF761BF000059
:10180000024BDB6898610F20FFF75CBF9823002034
:10181000302383F31188FFF7F3BF000008B50146BA
:10182000302383F311880820FFF75AFF002383F346
:10183000118808BD064BDB6839B1426818605A60F0
:10184000136043600420FFF74BBF4FF0FF30704739
:10185000982300200368984206D01A6802605060FE
:1018600099611846FFF72CBF7047000038B5044651
:101870000D462068844200D138BD036823605C6057
:101880008561FFF71DFFF4E710B503689C68A2426D
:101890000CD85C688A600B604C6021605960996864
:1018A0008A1A9A604FF0FF33836010BD1B68121BC9
:1018B000ECE700000A2938BF0A2170B504460D463E
:1018C0000A26601901F092FA01F07EFA041BA54283
:1018D00003D8751C2E460446F3E70A2E04D9BDE84A
:1018E0007040012001F0C8BA70BD0000F8B5144B7B
:1018F0000D46D96103F1100141600A2A196982601D
:1019000038BF0A22016048601861A818144601F027
:101910005FFA0A2701F058FA431BA342064606D392
:101920007C1C281901F062FA27463546F2E70A2F97
:1019300004D9BDE8F840012001F09EBAF8BD00BF0F
:1019400098230020F8B506460D4601F03DFA0F4AEF
:10195000134653F8107F9F4206D12A46014630466F
:10196000BDE8F840FFF7C2BFD169BB68441A2C1923
:1019700028BF2C46A34202D92946FFF79BFF2246E7
:1019800031460348BDE8F840FFF77EBF98230020AA
:10199000A823002010B4C0E9032300235DF8044B02
:1019A0004361FFF7CFBF000010B5194C236998427F
:1019B0000DD0D0E90032816813605A609A680A44F9
:1019C0009A60002303604FF0FF33A36110BD2346EC
:1019D000026843F8102F53600022026022699A4285
:1019E00003D1BDE8104001F0FBB9936881680B4456
:1019F000936001F0E9F92269E1699268441AA24210
:101A0000E4D91144BDE81040091AFFF753BF00BFE5
:101A1000982300202DE9F047DFF8BC8008F110077B
:101A20002C4ED8F8105001F0CFF9D8F81C40AA6815
:101A3000031B9A423ED81444D5E900324FF0000906
:101A4000C8F81C4013605A60C5F80090D8F81030F0
:101A5000B34201D101F0C4F989F31188D5E903310A
:101A600028469847302383F311886B69002BD8D020
:101A700001F0AAF96A69A0EB04094A4582460DD231
:101A8000022001F0F9F90022D8F81030B34208D151
:101A900051462846BDE8F047FFF728BF121A2244F6
:101AA000F2E712EB090938BF4A4629463846FFF7E4
:101AB000EBFEB5E7D8F81030B34208D01444211A31
:101AC000C8F81C00A960BDE8F047FFF7F3BEBDE809
:101AD000F08700BFA8230020982300200020704733
:101AE000FEE70000704700004FF0FF307047000035
:101AF00002290CD0032904D00129074818BF00206F
:101B00007047032A05D8054800EBC2007047044817
:101B100070470020704700BFC43500082022002015
:101B20007835000870B59AB00546084601A91446F4
:101B300000F0C2F801A8FFF7BFF8431C5B00C5E93D
:101B400000340022237003236370C6B201AB023459
:101B50001046D1B28E4204F1020401D81AB070BD11
:101B600013F8011B04F8021C04F8010C0132F0E721
:101B700008B5302383F311880348FFF759FA00238F
:101B800083F3118808BD00BF0826002090F8443078
:101B900003F01F02012A07D190F845200B2A03D138
:101BA0000023C0E90E3315E003F06003202B08D1B9
:101BB000B0F848302BB990F84520212A03D81F2AC5
:101BC00004D8FFF717BA222AEBD0FAE7034A826358
:101BD0000722C26303640120704700BF182200205F
:101BE00007B5052917D8DFE801F0191603191920E0
:101BF000302383F31188104A01900121FFF7BAFACC
:101C000001980E4A0221FFF7B5FA0D48FFF7DCF9FB
:101C1000002383F3118803B05DF804FB302383F3C2
:101C200011880748FFF7A6F9F2E7302383F31188FC
:101C30000348FFF7BDF9EBE7183500083C3500080D
:101C40000826002038B50C4D0C4C0D492A4604F1ED
:101C50000800FFF767FF05F1CA0204F11000094907
:101C6000FFF760FF05F5CA7204F118000649BDE8E8
:101C70003840FFF757BF00BFD02A002020220020A5
:101C8000F8340008023500080D35000870B5044628
:101C900008460D46FFF710F8C6B220460134037817
:101CA0000BB9184670BD32462946FEF7F1FF0028F1
:101CB000F3D10120F6E700002DE9F84F05460C4668
:101CC000FEF7FAFF2B49C6B22846FFF7DFFF08B13F
:101CD0000536F6B228492846FFF7D8FF08B1103676
:101CE000F6B2632E0DD8DFF88C80DFF88C90234F8E
:101CF000DFF890A0DFF890B02E7846B92670BDE8E6
:101D0000F88F29462046BDE8F84F01F09BBB252EF1
:101D10002BD1072241462846FEF7BAFF58B9DBF817
:101D200000302360DBF804306360DBF80830A36028
:101D300007350C34E0E7082249462846FEF7A8FF9D
:101D400098B90F4BA21C197809090232C95D02F833
:101D5000041C13F8011B01F00F015345C95D02F883
:101D6000031CF0D118340835C6E704F8016B0135BF
:101D7000C2E700BFE43500080D350008F93500085A
:101D8000107AFF1F1C7AFF1FEC350008BFF34F8F3E
:101D9000024AD368DB03FCD4704700BF003C02401A
:101DA00008B5094B1B7873B9FFF7F0FF074B1A69A9
:101DB000002ABFBF064A5A6002F188325A601A6888
:101DC00022F480621A6008BD2E2D0020003C0240E3
:101DD0002301674508B50B4B1B7893B9FFF7D6FF76
:101DE000094B1A6942F000421A611A6842F48052A3
:101DF0001A601A6822F480521A601A6842F48062EB
:101E00001A6008BD2E2D0020003C02400B28F0B5C2
:101E100016D80C4C0C4923787BB90C4D0E460C237C
:101E20004FF0006255F8047B46F8042B013B13F099
:101E3000FF033A44F6D10123237051F82000F0BD8E
:101E40000020FCE7602D0020302D00200C3600081B
:101E5000014B53F8200070470C3600080C207047E7
:101E60000B2810B5044601D9002010BDFFF7CEFFA6
:101E7000064B53F824301844C21A0BB90120F4E77A
:101E800012680132F0D1043BF6E700BF0C360008BF
:101E90000B2810B5044621D8FFF778FFFFF780FF25
:101EA0000F4AF323D360C300DBB243F4007343F063
:101EB00002031361136943F480331361FFF766FF74
:101EC000FFF7A4FF074B53F8241000F0D9F8FFF7F1
:101ED00081FF2046BDE81040FFF7C2BF002010BDC3
:101EE000003C02400C360008F8B512F0010314461D
:101EF00042D18218B2F1016F57D82D4B1B6813F0F5
:101F0000010352D02B4DFFF74BFFF323EB60FFF79C
:101F10003DFF40F20127032C15D824F00104661878
:101F2000244C401A40F20117B142236900EB01052D
:101F300024D123F001032361FFF74CFF0120F8BDFA
:101F4000043C0430E7E78307E7D12B6923F44073AF
:101F50002B612B693B432B6151F8046B0660BFF387
:101F60004F8FFFF713FF03689E42E9D02B6923F0E0
:101F700001032B61FFF72EFF0020E0E723F44073FD
:101F8000236123693B4323610B882B80BFF34F8F71
:101F9000FFF7FCFE2D8831F8023BADB2AB42C3D057
:101FA000236923F001032361E4E71846C7E700BF74
:101FB00000380240003C0240084908B50B7828B1BF
:101FC0001BB9FFF7EDFE01230B7008BD002BFCD001
:101FD000BDE808400870FFF7FDBE00BF2E2D0020B1
:101FE00010B50244064BD2B2904200D110BD441C41
:101FF00000B253F8200041F8040BE0B2F4E700BF50
:10200000502800400F4B30B51C6F240407D41C6FC0
:1020100044F400741C671C6F44F400441C670A4CB1
:10202000236843F4807323600244084BD2B2904289
:1020300000D130BD441C00B251F8045B43F820507D
:10204000E0B2F4E700380240007000405028004041
:1020500007B5012201A90020FFF7C2FF019803B0D4
:102060005DF804FB13B50446FFF7F2FFA04205D06C
:10207000012201A900200194FFF7C4FF02B010BDA6
:1020800070470000034B1A681AB9034AD2F8742843
:102090001A607047642D00200030024008B5FFF739
:1020A000F1FF024B1868C0F3407008BD642D00209A
:1020B00070470000FEE700000A4B0B480B4A9042B5
:1020C0000BD30B4BDA1C121AC11E22F003028B42F7
:1020D00038BF00220021FEF7F7BD53F8041B40F87B
:1020E000041BECE7B8370008602E0020602E0020AB
:1020F000602E002070B5D0E915439E6800224FF095
:10210000FF3504EB42135101D3F800090028BEBF8C
:10211000D3F8000940F08040C3F80009D3F8000B61
:102120000028BEBFD3F8000B40F08040C3F8000B7E
:10213000013263189642C3F80859C3F8085BE0D22D
:102140004FF00113C4F81C3870BD0000890141F044
:102150002001016103699B06FCD41220FFF716BB26
:1021600010B5054C2046FEF7E5FF4FF0A043636530
:10217000024BA36510BD00BF682D0020603600082B
:1021800070B50378012B054650D12A4B446D984217
:102190001BD1294B5A6B42F080025A635A6D42F0B0
:1021A00080025A655A6D5A6942F080025A615A6932
:1021B00022F080025A610E2143205B6900F022FC6C
:1021C0001E4BE3601E4BC4F800380023C4F8003EE9
:1021D000C02323606E6D4FF40413A3633369002B97
:1021E000FCDA012333610C20FFF7D0FA3369DB07F7
:1021F000FCD41220FFF7CAFA3369002BFCDA002660
:10220000A6602846FFF776FF6B68C4F81068DB68A5
:10221000C4F81468C4F81C684BB90A4BA3614FF0AA
:10222000FF336361A36843F00103A36070BD064BF5
:10223000F4E700BF682D0020003802404014004041
:1022400003002002003C30C0083C30C0F8B5446DAB
:10225000054600212046FFF779FFA96D00234FF0C6
:1022600001128F68C4F834384FF00066C4F81C2897
:102270004FF0FF3004EB431201339F42C2F8006974
:10228000C2F8006BC2F80809C2F8080BF2D20B685A
:102290006A6DEB65636210231361166916F0100610
:1022A000FBD11220FFF772FAD4F8003823F4FE6352
:1022B000C4F80038A36943F4402343F01003A3613A
:1022C0000923C4F81038C4F814380A4BEB604FF0F7
:1022D000C043C4F8103B084BC4F8003BC4F8106975
:1022E000C4F80039EB6D03F1100243F48013EA6582
:1022F000A362F8BD3C36000840800010426D90F8A3
:102300004E10D2F8003823F4FE6343EA0113C2F8FA
:10231000003870472DE9F84300EB8103456DDA681A
:10232000166806F00306731E022B05EB41130C46DC
:1023300080460FFA81F94FEA41104FF00001C3F8CF
:10234000101B4FF0010104F1100398BFB60401FA0D
:1023500003F391698EBF334E06F1805606F50046B1
:1023600000293AD0578A04F15801490137436F5088
:10237000D5F81C180B43C5F81C382B180021C3F8DE
:10238000101953690127611EA7409BB3138A928BD2
:102390009B08012A88BF5343D8F85C20981842EA6A
:1023A000034301F1400205EB8202C8F85C002146BC
:1023B00053602846FFF7CAFE08EB8900C3681B8AF2
:1023C00043EA8453483464011E432E51D5F81C3827
:1023D0001F43C5F81C78BDE8F88305EB4917D7F80B
:1023E000001B21F40041C7F8001BD5F81C1821EA96
:1023F0000303C0E704F13F0305EB83030A4A5A6075
:1024000028462146FFF7A2FE05EB4910D0F8003917
:1024100023F40043C0F80039D5F81C3823EA070735
:10242000D7E700BF0080001000040002826D126830
:10243000C265FFF75FBE00005831436D49015B582C
:1024400013F4004004D013F4001F0CBF022001203D
:10245000704700004831436D49015B5813F4004058
:1024600004D013F4001F0CBF0220012070470000AD
:1024700000EB8101CB68196A0B6813604B685360ED
:102480007047000000EB810330B5DD68AA6913686E
:10249000D36019B9402B84BF402313606B8A146842
:1024A000426D1C44013CB4FBF3F46343033323F05B
:1024B000030302EB411043EAC44343F0C043C0F8B6
:1024C000103B2B6803F00303012B09B20ED1D2F8A5
:1024D000083802EB411013F4807FD0F8003B14BFA2
:1024E00043F0805343F00053C0F8003B02EB41122D
:1024F000D2F8003B43F00443C2F8003B30BD00007B
:102500002DE9F041244D6E6D06EB40130446D3F8DF
:10251000087BC3F8087B38070AD5D6F814381907A2
:1025200006D505EB84032146DB6828465B6898479F
:10253000FA071FD5D6F81438DB071BD505EB840343
:10254000D968CCB98B69488A5A68B2FBF0F600FBAF
:1025500016228AB91868DA6890420DD2121AC3E9B5
:102560000024302383F311880B482146FFF78AFFAC
:1025700084F31188BDE8F081012303FA04F26B892A
:1025800023EA02036B81CB68002BF3D0214602487B
:10259000BDE8F041184700BF682D002000EB810323
:1025A00070B5DD68436D6C692668E6604A0156BB0C
:1025B0001A444FF40020C2F810092A6802F00302FE
:1025C000012A0AB20ED1D3F8080803EB421410F422
:1025D000807FD4F8000914BF40F0805040F00050D4
:1025E000C4F8000903EB4212D2F8000940F004409D
:1025F000C2F80009D3F83408012202FA01F10143BC
:10260000C3F8341870BD19B9402E84BF4020206033
:1026100020682E8A8419013CB4FBF6F440EAC440D9
:1026200040F000501A44C6E72DE9F8433B4D6E6D6B
:1026300006EB40130446D3F80889C3F8088918F05C
:10264000010F4FEA40171AD0D6F81038DB0716D51D
:1026500005EB8003D9684B691868DA68904230D27C
:10266000121A4FF000091A60C3F80490302383F364
:10267000118821462846FFF791FF89F3118818F049
:10268000800F1CD0D6F834380126A640334216D02D
:1026900005EB84036D6DD3F80CC0DCF81420013415
:1026A000E4B2D2F800E005EB04342F4451687145E0
:1026B00015D3D5F8343823EA0606C5F83468BDE8E2
:1026C000F883012303FA04F22B8923EA02032B8106
:1026D0008B68002BD3D0214628469847CFE7BCF81B
:1026E0001000AEEB0103834228BF0346D7F8180958
:1026F00080B2B3EB800FE2D89068A0F1040959F8DA
:10270000048FC4F80080A0EB09089844B8F1040FC6
:10271000F5D818440B4490605360C7E7682D00203B
:102720002DE9F74FA24C656D6E69AB691E4016F43A
:1027300080586E6107D02046FEF764FD03B0BDE807
:10274000F04F00F047BC002E12DAD5F8003E984852
:102750009B071EBFD5F8003E23F00303C5F8003EDB
:10276000D5F8043823F00103C5F80438FEF774FDEA
:10277000370505D58E48FFF7BDFC8D48FEF75AFD9D
:10278000B0040CD5D5F8083813F0060FEB6823F425
:1027900070530CBF43F4105343F4A053EB60310764
:1027A0001BD56368DB681BB9AB6923F00803AB6119
:1027B0002378052B0CD1D5F8003E7D489A071EBF23
:1027C000D5F8003E23F00303C5F8003EFEF744FDB4
:1027D0006368DB680BB176489847F30274D4B7029C
:1027E00027D5D4F85490DFF8C8B100274FF0010A7C
:1027F00009EB4712D2F8003B03F44023B3F5802FD6
:1028000011D1D2F8003B002B0DDA62890AFA07F3E6
:1028100022EA0303638104EB8703DB68DB6813B1FF
:10282000394658469847A36D01379B68FFB29F42CF
:10283000DED9F00617D5676D3A6AC2F30A1002F0C6
:102840000F0302F4F012B2F5802F00F08580B2F58C
:10285000402F08D104EB83030022DB681B6A07F5D5
:10286000805790426AD13003D5F8184813D5E10358
:1028700002D50020FFF744FEA20302D50120FFF796
:102880003FFE630302D50220FFF73AFE270302D57D
:102890000320FFF735FE75037FF550AFE00702D543
:1028A0000020FFF7C1FEA10702D50120FFF7BCFE03
:1028B000620702D50220FFF7B7FE23077FF53EAF80
:1028C0000320FFF7B1FE39E7636DDFF8E4A0019361
:1028D00000274FF00109A36D9B685FFA87FB9B45BA
:1028E0003FF67DAF019B03EB4B13D3F8001901F4C6
:1028F0004021B1F5802F1FD1D3F8001900291BDA30
:10290000D3F8001941F09041C3F80019D3F8001929
:102910000029FBDB5946606DFFF718FC218909FA95
:102920000BF321EA0303238104EB8B03DB689B6831
:1029300013B15946504698470137CCE7910708BF75
:10294000D7F80080072A98BF03F8018B02F1010233
:1029500098BF4FEA182884E7023304EB830207F597
:1029600080575268D2F818C0DCF80820DCE9001C57
:10297000A1EB0C0C002188420AD104EB83046368AC
:102980009B699A6802449A605A6802445A606AE7EE
:1029900011F0030F08BFD7F800808C4588BF02F8FC
:1029A000018B01F1010188BF4FEA1828E3E700BF5E
:1029B000682D0020436D03EB4111D1F8003B43F437
:1029C0000013C1F8003B7047436D03EB4111D1F890
:1029D000003943F40013C1F800397047436D03EB2D
:1029E0004111D1F8003B23F40013C1F8003B7047BC
:1029F000436D03EB4111D1F8003923F40013C1F802
:102A00000039704700F1604303F561430901C9B221
:102A100083F80013012200F01F039A4043099B0032
:102A200003F1604303F56143C3F880211A607047E6
:102A300030B5039C0172043304FB0325C0E906533F
:102A4000049B03630021059BC160C0E90000C0E94D
:102A50000422C0E90842C0E90A11436330BD000006
:102A6000416A0022C0E90411C0E90A22C2606FF085
:102A70000101FEF7FBBE0000D0E90432934201D110
:102A8000C2680AB9181D70470020704703691960B1
:102A9000C2680132C260C269134482690361934211
:102AA00024BF436A03610021FEF7D4BE38B5044653
:102AB0000D46E3683BB16269131D1268A3621344BB
:102AC000E362002007E0237A33B929462046FEF767
:102AD000B1FE0028EDDA38BD6FF00100FBE7000021
:102AE000C368C269013BC36043691344826943619F
:102AF000934224BF436A436100238362036B03B1A3
:102B00001847704770B53023044683F31188866AEE
:102B10003EB9FFF7CBFF054618B186F3118828466A
:102B200070BDA36AE26A13F8015BA362934202D309
:102B30002046FFF7D5FF002383F31188EFE700005D
:102B40002DE9F84F04460E46174698464FF03009D7
:102B500089F311880025AA46D4F828B0BBF1000FEC
:102B600009D141462046FFF7A1FF20B18BF3118820
:102B70002846BDE8F88FD4E90A12A7EB050B521AD4
:102B8000934528BF9346BBF1400F1BD9334601F153
:102B9000400251F8040B43F8040B9142F9D1A36AA7
:102BA00040334036A3624035D4E90A239A4202D327
:102BB0002046FFF795FF8AF31188BD42D8D289F3EA
:102BC0001188C9E730465A46FEF758F8A36A5B44B5
:102BD0005E44A3625D44E7E710B5029C01720433D2
:102BE00003FB0421C0E906130023C0E90A33039B59
:102BF0000363049BC460C0E90000C0E90422C0E98B
:102C00000842436310BD0000026AC260426AC0E924
:102C100004220022C0E90A226FF00101FEF726BE5D
:102C2000D0E904239A4201D1C26822B9184650F86B
:102C3000043B0B60704700231846FAE7C368C2697B
:102C40000133C3604369134482694361934224BFE3
:102C5000436A43610021FEF7FDBD000038B504461C
:102C60000D46E3683BB123691A1DA262E269134471
:102C7000E362002007E0237A33B929462046FEF7B5
:102C8000D9FD0028EDDA38BD6FF00100FBE7000048
:102C900003691960C268013AC260C269134482695B
:102CA0000361934224BF436A036100238362036B81
:102CB00003B118477047000070B530230D46044635
:102CC000114683F31188866A2EB9FFF7C7FF10B14A
:102CD00086F3118870BDA36A1D70A36AE26A01338E
:102CE0009342A36204D3E16920460439FFF7D0FF81
:102CF000002080F31188EDE72DE9F84F04460D46DA
:102D0000904699464FF0300A8AF311880026B34660
:102D1000A76A4FB949462046FFF7A0FF20B187F3C5
:102D200011883046BDE8F88FD4E90A073A1AA8EBB3
:102D30000607974228BF1746402F1BD905F14003CD
:102D400055F8042B40F8042B9D42F9D1A36A403377
:102D5000A3624036D4E90A239A4204D3E1692046AB
:102D60000439FFF795FF8BF311884645D9D28AF3D2
:102D70001188CDE729463A46FDF780FFA36A3B4418
:102D80003D44A3623E44E5E7D0E904239A4217D1CB
:102D9000C3689BB1836A8BB1043B9B1A0ED013604E
:102DA000C368013BC360C3691A44836902619A42E4
:102DB00024BF436A036100238362012318467047DE
:102DC0000023FBE700F030B94FF08043586A7047AA
:102DD0004FF08043002258631A610222DA60704784
:102DE0004FF080430022DA60704700004FF08043CC
:102DF00058637047FEE7000070B51B4B0163002568
:102E0000044686B0586085620E4600F0BFF804F1B3
:102E10001003C4E904334FF0FF33C4E90635C4E9B5
:102E20000044A560E562FFF7CFFF2B460246C4E9E8
:102E3000082304F134010D4A256580232046FEF75E
:102E4000AFFC0123E0600A4A0375009272680192A8
:102E5000B268CDE90223074B6846CDE90435FEF799
:102E6000C7FC06B070BD00BF002600206C3600080D
:102E700071360008F52D0008024AD36A1843D06263
:102E8000704700BF982300204B6843608B688360C5
:102E9000CB68C3600B6943614B6903628B69436212
:102EA0000B6803607047000008B5264B26481A6976
:102EB00040F2FF110A431A611A6922F4FF7222F0EC
:102EC00001021A611A691A6B0A431A631A6D0A43DE
:102ED0001A651E4A1B6D1146FFF7D6FF02F11C0151
:102EE00000F58060FFF7D0FF02F1380100F5806047
:102EF000FFF7CAFF02F1540100F58060FFF7C4FF3D
:102F000002F1700100F58060FFF7BEFF02F18C0155
:102F100000F58060FFF7B8FF02F1A80100F58060BE
:102F2000FFF7B2FF02F1C40100F58060FFF7ACFFCC
:102F300002F1E00100F58060FFF7A6FFBDE8084060
:102F400000F0EEB800380240000002407836000879
:102F500008B500F059FAFEF701FCFFF793F8BDE859
:102F60000840FEF76FBE000070470000EFF30983D2
:102F700005494A6B22F001024A63683383F30988EA
:102F8000002383F31188704700EF00E0302080F3C6
:102F9000118862B60C4B0D4AD96821F4E06109042E
:102FA000090C0A43DA60D3F8FC20094942F0807228
:102FB000C3F8FC200A6842F001020A602022DA7796
:102FC00083F82200704700BF00ED00E00003FA051F
:102FD000001000E010B5302383F311880E4B5B68BE
:102FE00013F4006314D0F1EE103AEFF30984683C57
:102FF0004FF08073E361094BDB6B236684F3098830
:10300000FEF78CFB10B1064BA36110BD054BFBE72F
:1030100083F31188F9E700BF00ED00E000EF00E066
:103020002F030008320300080F4B1A6C42F0010214
:103030001A641A6E42F001021A660C4A1B6E9368FB
:1030400043F0010393604FF0804353229A624FF0A4
:10305000FF32DA6200229A615A63DA605A60012212
:103060005A611A60704700BF00380240002004E037
:103070004FF0804208B51169D3680B40D9B2C943FB
:103080009B07116107D5302383F31188FEF77CFB82
:10309000002383F3118808BD1F4B1A696FEAC252DF
:1030A0006FEAD2521A611A69C2F308021A614FF02C
:1030B000FF301A695A69586100215A6959615A6981
:1030C0001A6A62F080521A621A6A02F080521A6218
:1030D0001A6A5A6A58625A6A59625A6A1A6C42F0F3
:1030E00080521A641A6E42F080521A661A6E0B4AA7
:1030F000106840F480701060186F00F44070B0F5F4
:10310000007F1EBF4FF4803018671967536823F49F
:103110000073536000F054B9003802400070004062
:10312000334B4FF080521A64324A4FF440411160E1
:103130001A6842F001021A601A689107FCD59A6871
:1031400022F003029A602A4B9A6812F00C02FBD11B
:10315000196801F0F90119609A601A6842F4803226
:103160001A601A689203FCD55A6F42F001025A673E
:103170001F4B5A6F9007FCD51F4A5A601A6842F0DD
:1031800080721A601B4A53685904FCD5184B1A68A0
:103190009201FCD5194A9A60194B1A68194B9A4248
:1031A000194B21D1194A1168194A91421CD140F298
:1031B00005121A60144A136803F00F03052BFAD1A5
:1031C0000B4B9A6842F002029A609A6802F00C0275
:1031D000082AFAD15A6C42F480425A645A6E42F478
:1031E00080425A665B6E704740F20572E1E700BFAD
:1031F00000380240007000400854400700948838AE
:10320000002004E011640020003C024000ED00E0DA
:1032100041C20F41074A08B5536903F001035361E6
:1032200023B1054A13680BB150689847BDE80840C0
:10323000FFF7D0BE003C0140E02D0020074A08B552
:10324000536903F00203536123B1054A93680BB13C
:10325000D0689847BDE80840FFF7BCBE003C01407D
:10326000E02D0020074A08B5536903F004035361B9
:1032700023B1054A13690BB150699847BDE808406E
:10328000FFF7A8BE003C0140E02D0020074A08B52A
:10329000536903F00803536123B1054A93690BB1E5
:1032A000D0699847BDE80840FFF794BE003C014054
:1032B000E02D0020074A08B5536903F0100353615D
:1032C00023B1054A136A0BB1506A9847BDE808401C
:1032D000FFF780BE003C0140E02D0020164B10B5EA
:1032E0005C6904F478725A61A30604D5134A936AA0
:1032F0000BB1D06A9847600604D5104A136B0BB126
:10330000506B9847210604D50C4A936B0BB1D06BD8
:103310009847E20504D5094A136C0BB1506C9847E5
:10332000A30504D5054A936C0BB1D06C9847BDE852
:103330001040FFF74FBE00BF003C0140E02D0020D1
:10334000194B10B55C6904F47C425A61620504D5DE
:10335000164A136D0BB1506D9847230504D5134AD7
:10336000936D0BB1D06D9847E00404D50F4A136EEE
:103370000BB1506E9847A10404D50C4A936E0BB163
:10338000D06E9847620404D5084A136F0BB1506F92
:103390009847230404D5054A936F0BB1D06F984723
:1033A000BDE81040FFF716BE003C0140E02D0020B4
:1033B00008B5FFF75DFEBDE80840FFF70BBE000053
:1033C000062108B50846FFF71DFB06210720FFF779
:1033D00019FB06210820FFF715FB06210920FFF73E
:1033E00011FB06210A20FFF70DFB06211720FFF72E
:1033F00009FB06212820FFF705FBBDE8084007214F
:103400001C20FFF7FFBA000008B5FFF745FE00F0EB
:103410000BF8FDF78DFEFDF765FDFFF7A5FDBDE897
:103420000840FFF7CFBC00000023054A19460133CE
:10343000102BC2E9001102F10802F8D1704700BF59
:10344000E02D0020034611F8012B03F8012B002A80
:10345000F9D1704753544D3332463F3F3F005354E8
:103460004D3332463430780053544D333246343283
:10347000780053544D3332463434365858000000E7
:10348000012033000010410001105A0003105900C0
:10349000071031000000000054340008130400003D
:1034A0005E3400081904000068340008210400009C
:1034B0007234000800000000610E00084D0E000884
:1034C000890E0008750E0008810E00086D0E0008B8
:1034D000590E0008450E0008950E00080000000077
:1034E000010000000000000063300000E834000824
:1034F000F0230020002600204172647550696C6F33
:10350000740025424F415244252D424C002553451D
:103510005249414C2500000002000000000000005C
:103520007D100008E910000840004000A02A00209B
:10353000B02A00200200000000000000030000008C
:10354000000000002D110008000000001000000025
:10355000C02A002000000000010000000000000060
:10356000682D002001010200E11B0008F11A00088B
:103570008D1B0008711B0008430000008035000807
:1035800009024300020100C03209040000010202E6
:103590000100052400100105240100010424020299
:1035A0000524060001070582030800FF0904010045
:1035B000020A000000070501024000000705810221
:1035C0004000000012000000CC350008120110017C
:1035D00002000040091241570002010203010000ED
:1035E0000403090425424F4152442500466F786583
:1035F0006572463430357632003031323334353608
:10360000373839414243444546000000004000003D
:1036100000400000004000000040000000000100E9
:103620000000020000000200000002000000020092
:103630000000020000000200000002000000000084
:103640007112000829150008D51500084000400037
:10365000C82D0020C82D002001000000D82D00201A
:103660008000000040010000030000006D61696EF1
:103670000069646C65000000000180060000000025
:10368000AAAAAAAA00010000FFDF000000000000B3
:1036900000A00A000000000100000000AAAAAAAAD7
:1036A00000000001FFFF000000000000000000001B
:1036B0000000001000000000AAAAAAAA0000001042
:1036C000FFFF0000000000000000000000000000FC
:1036D00000000000AAAAAAAA00000000FFFF000044
:1036E00000000000000000000000000000000000DA
:1036F000AAAAAAAA00000000FFFF00000000000024
:10370000000000000000000000000000AAAAAAAA11
:1037100000000000FFFF00000000000000000000AB
:103720000000000000000000AAAAAAAA00000000F1
:10373000FFFF00000000000000000000000000008B
:10374000000000000A00000000000000030000006C
:103750000000000000000000000000000000000069
:103760000000000000000000000000000000000059
:1037700000000000000000008504000000000000C0
:1037800000400F0000000000FF009600000000084D
:10379000009600000000080004000000E03500086A
:1037A0000000000000000000000000000000000019
:1037B0000000000000000000FFFFFFFFFFFFFFFF11
:1037C000FFFFFFFFFFFFFFFFFFFFFFFFFFFFFFFF09
:1037D000FFFFFFFFFFFFFFFFFFFFFFFFFFFFFFFFF9
:1037E000FFFFFFFFFFFFFFFFFFFFFFFFFFFFFFFFE9
:1037F000FFFFFFFFFFFFFFFFFFFFFFFFFFFFFFFFD9
:10C000000006002089D20008E1E109083DE10908A5
:10C01000A9E109083DE1090875E109088BD200088A
:10C020008BD200088BD200088BD20008150F0C08A9
:10C030008BD200088BD200088BD200088BD200086C
:10C040008BD200088BD200088BD200088BD200085C
:10C050008BD200088BD2000831210C0859210C0822
:10C0600081210C08A9210C08D1210C0861CD0B08F5
:10C0700089CD0B08B5CD0B08E1CD0B080DCE0B0813
:10C0800035CE0B0861CE0B08E5CC0B088BD200082F
:10C090008BD200088BD200088BD20008F9210C0843
:10C0A00045230C0849230C085D230C0861230C0868
:10C0B00065230C0879230C088D230C08EDD30B089D
:10C0C00095D50B088BD200088BD200088BD20008C4
:10C0D0008BD20008CD220C08E1220C08F5220C08B6
:10C0E0005D220C088BD200088BD20008B1230C080B
:10C0F000B5230C08C9230C08CD230C088DCE0B08E2
:10C100008BD200088BD20008A1230C088BD2000828
:10C1100009230C081D230C088BD200088BD20008C1
:10C12000B9CE0B08E1CE0B080DCF0B0839CF0B08A9
:10C1300065CF0B088BD200088BD200088BD2000889
:10C140008BD200088BD200088BD2000841160C0855
:10C150008DCF0B08B9CF0B08E5CF0B0831230C08A6
:10C160008BD200088BD200088BD200088BD200083B
:10C170008BD200088BD200088BD200088BD200082B
:10C180008BD200088BD200088BD200088BD200081B
:10C190008BD200088BD200088BD200088BD200080B
:10C1A0008BD200088BD200088BD200088BD20008FB
:10C1B0008BD200088BD200088BD200088BD20008EB
:10C1C0008BD200088BD200088BD200088BD20008DB
:10C1D0008BD200088BD200088BD200088BD20008CB
:10C1E000052501085DF80208A96B040809F2050895
:10C1F0002DF8050841630608C9B206088DBA06087D
:10C20000C5BD0608251E07086D43070835DA07086F
:10C21000ED2B0808A9DA09083DDD0A089D490B083D
:10C22000B56F0B08017B0B08A5A80B086DAE0B08BA
:10C2300081F0004102E000BF83F0004330B54FEAD7
:10C2400041044FEA430594EA050F08BF90EA020F44
:10C250001FBF54EA000C55EA020C7FEA645C7FEAD7
:10C26000655C00F0E2804FEA5454D4EB5555B8BFFA
:10C270006D420CDD2C4480EA020281EA030382EA6B
:10C28000000083EA010180EA020281EA0303362DFD
:10C2900088BF30BD11F0004F4FEA01314FF4801CD0
:10C2A0004CEA113102D0404261EB410113F0004FE2
:10C2B0004FEA03334CEA133302D0524263EB430399
:10C2C00094EA050F00F0A780A4F10104D5F1200E37
:10C2D0000DDB02FA0EFC22FA05F2801841F1000192
:10C2E00003FA0EF2801843FA05F359410EE0A5F166
:10C2F00020050EF1200E012A03FA0EFC28BF4CF097
:10C30000020C43FA05F3C01851EBE37101F000454C
:10C3100007D54FF0000EDCF1000C7EEB00006EEB59
:10C320000101B1F5801F1BD3B1F5001F0CD34908E3
:10C330005FEA30004FEA3C0C04F101044FEA44523A
:10C3400012F5800F80F09A80BCF1004F08BF5FEAC1
:10C35000500C50F1000041EB045141EA050130BDA1
:10C360005FEA4C0C404141EB0101013C28BFB1F5B3
:10C37000801FE9D291F0000F04BF01460020B1FAFE
:10C3800081F308BF2033A3F10B03B3F120020CDAD1
:10C390000C3208DD02F1140CC2F10C0201FA0CF0AF
:10C3A00021FA02F10CE002F11402D8BFC2F1200C14
:10C3B00001FA02F120FA0CFCDCBF41EA0C019040CA
:10C3C000E41AA2BF01EB0451294330BD6FEA040413
:10C3D0001F3C1CDA0C340EDC04F11404C4F12002FE
:10C3E00020FA04F001FA02F340EA030021FA04F310
:10C3F00045EA030130BDC4F10C04C4F1200220FA67
:10C4000002F001FA04F340EA0300294630BD21FAA4
:10C4100004F0294630BD94F0000F83F4801306BF6A
:10C4200081F480110134013D4EE77FEA645C18BF5E
:10C430007FEA655C29D094EA050F08BF90EA020FF5
:10C4400005D054EA000C04BF1946104630BD91EAED
:10C45000030F1EBF0021002030BD5FEA545C05D1F0
:10C460004000494128BF41F0004130BD14F580042F
:10C470003CBF01F5801130BD01F0004545F0FE41A3
:10C4800041F470014FF0000030BD7FEA645C1ABFD8
:10C49000194610467FEA655C1CBF0B46024650EA0F
:10C4A000013406BF52EA033591EA030F41F400213B
:10C4B00030BD00BF90F0000F04BF0021704730B5C1
:10C4C0004FF4806404F132044FF000054FF0000196
:10C4D00050E700BF90F0000F04BF0021704730B557
:10C4E0004FF4806404F1320410F0004548BF40422C
:10C4F0004FF000013EE700BF42004FEAE2014FEA81
:10C5000031014FEA02701FBF12F07F4393F07F4F5B
:10C5100081F06051704732F07F4208BF704793F05E
:10C520007F4F04BF41F40021704730B54FF4607471
:10C5300001F0004521F000411CE700BF50EA010274
:10C5400008BF704730B54FF000050AE050EA01021D
:10C5500008BF704730B511F0004502D5404261EB8D
:10C5600041014FF4806404F132045FEA915C3FF4CE
:10C57000D8AE4FF003025FEADC0C18BF03325FEA6B
:10C58000DC0C18BF033202EBDC02C2F1200300FA1C
:10C5900003FC20FA02F001FA03FE40EA0E0021FA41
:10C5A00002F11444BDE600BF70B54FF0FF0C4CF42F
:10C5B000E06C1CEA11541DBF1CEA135594EA0C0FE1
:10C5C00095EA0C0F00F0DEF82C4481EA030621EA1C
:10C5D0004C5123EA4C5350EA013518BF52EA033557
:10C5E00041F4801143F4801338D0A0FB02CE4FF009
:10C5F0000005E1FB02E506F00042E0FB03E54FF039
:10C600000006E1FB03569CF0000F18BF4EF0010E30
:10C61000A4F1FF04B6F5007F64F5407404D25FEA2C
:10C620004E0E6D4146EB060642EAC62141EA5551DF
:10C630004FEAC52040EA5E504FEACE2EB4F1FD0C21
:10C6400088BFBCF5E06F1ED8BEF1004F08BF5FEA9F
:10C65000500E50F1000041EB045170BD06F0004651
:10C6600046EA010140EA020081EA0301B4EB5C04FE
:10C67000C2BFD4EB0C0541EA045170BD41F48011F6
:10C680004FF0000E013C00F3AB8014F1360FDEBF1B
:10C69000002001F0004170BDC4F10004203C35DAF7
:10C6A0000C341BDC04F11404C4F1200500FA05F37A
:10C6B00020FA04F001FA05F240EA020001F000421B
:10C6C00021F0004110EBD37021FA04F642EB060191
:10C6D0005EEA430E08BF20EAD37070BDC4F10C04BB
:10C6E000C4F1200500FA04F320FA05F001FA04F27F
:10C6F00040EA020001F0004110EBD37041F100016B
:10C700005EEA430E08BF20EAD37070BDC4F1200575
:10C7100000FA05F24EEA020E20FA04F301FA05F2DD
:10C7200043EA020321FA04F001F0004121FA04F285
:10C7300020EA020000EBD3705EEA430E08BF20EA55
:10C74000D37070BD94F0000F0FD101F0004640008F
:10C7500041EB010111F4801F08BF013CF7D041EA11
:10C76000060195F0000F18BF704703F00046520015
:10C7700043EB030313F4801F08BF013DF7D043EAE6
:10C780000603704794EA0C0F0CEA135518BF95EA9C
:10C790000C0F0CD050EA410618BF52EA4306D1D123
:10C7A00081EA030101F000414FF0000070BD50EA42
:10C7B000410606BF1046194652EA430619D094EACC
:10C7C0000C0F02D150EA013613D195EA0C0F05D1B6
:10C7D00052EA03361CBF104619460AD181EA03010A
:10C7E00001F0004141F0FE4141F470014FF00000C2
:10C7F00070BD41F0FE4141F4780170BD70B54FF05D
:10C80000FF0C4CF4E06C1CEA11541DBF1CEA1355DC
:10C8100094EA0C0F95EA0C0F00F0A7F8A4EB0504BE
:10C8200081EA030E52EA03354FEA013100F08880B5
:10C830004FEA03334FF0805545EA131343EA12637E
:10C840004FEA022245EA111545EA10654FEA002633
:10C850000EF000419D4208BF964244F1FD0404F5EC
:10C86000407402D25B084FEA3202B61A65EB030548
:10C870005B084FEA32024FF480104FF4002CB6EB05
:10C88000020E75EB030E22BFB61A754640EA0C0085
:10C890005B084FEA3202B6EB020E75EB030E22BFC5
:10C8A000B61A754640EA5C005B084FEA3202B6EB06
:10C8B000020E75EB030E22BFB61A754640EA9C00C5
:10C8C0005B084FEA3202B6EB020E75EB030E22BF95
:10C8D000B61A754640EADC0055EA060E18D04FEA53
:10C8E000051545EA16754FEA06164FEAC30343EAF3
:10C8F00052734FEAC2025FEA1C1CC0D111F4801FC0
:10C900000BD141EA00014FF000004FF0004CB6E7B8
:10C9100011F4801F04BF01430020B4F1FD0C88BF57
:10C92000BCF5E06F3FF6AFAEB5EB030C04BFB6EB62
:10C93000020C5FEA500C50F1000041EB045170BD55
:10C940000EF0004E4EEA113114EB5C04C2BFD4EB82
:10C950000C0541EA045170BD41F480114FF0000E06
:10C96000013C90E645EA060E8DE60CEA135594EA82
:10C970000C0F08BF95EA0C0F3FF43BAF94EA0C0F85
:10C980000AD150EA01347FF434AF95EA0C0F7FF4FA
:10C9900025AF104619462CE795EA0C0F06D152EA4E
:10C9A00003353FF4FDAE1046194622E750EA410632
:10C9B00018BF52EA43067FF4C5AE50EA41047FF443
:10C9C0000DAF52EA43057FF4EBAE12E74FF0FF3CA8
:10C9D00006E000BF4FF0010C02E000BF4FF0010C79
:10C9E0004DF804CD4FEA410C7FEA6C5C4FEA430CF2
:10C9F00018BF7FEA6C5C1BD001B050EA410C0CBF41
:10CA000052EA430C91EA030F02BF90EA020F0020A2
:10CA1000704710F1000F91EA030F58BF994208BF09
:10CA200090422CBFD8176FEAE37040F001007047C6
:10CA30004FEA410C7FEA6C5C02D150EA013C07D11D
:10CA40004FEA430C7FEA6C5CD6D152EA033CD3D068
:10CA50005DF8040B704700BF8446104662468C4662
:10CA60001946634600E000BF01B5FFF7B7FF002895
:10CA700048BF10F1000F01BD4DF808EDFFF7F4FFBE
:10CA80000CBF012000205DF808FB00BF4DF808ED49
:10CA9000FFF7EAFF34BF012000205DF808FB00BF6C
:10CAA0004DF808EDFFF7E0FF94BF012000205DF88E
:10CAB00008FB00BF4DF808EDFFF7CEFF94BF012043
:10CAC00000205DF808FB00BF4DF808EDFFF7C4FF3C
:10CAD00034BF012000205DF808FB00BF4FEA410C85
:10CAE0007FEA6C5C02D150EA013C0AD14FEA430C68
:10CAF0007FEA6C5C02D152EA033C02D14FF00000A5
:10CB000070474FF0010070474FEA410212F50012E2
:10CB100015D211D56FF47873B3EB625212D94FEA84
:10CB2000C12343F0004343EA505311F0004F23FA6E
:10CB300002F018BF404270474FF00000704750EAC3
:10CB4000013005D111F0004008BF6FF00040704780
:10CB50004FF00000704700BF4A0011D212F50012DA
:10CB600011D20DD56FF47873B3EB62520ED44FEA45
:10CB7000C12343F0004343EA505323FA02F07047C5
:10CB80004FF00000704750EA013002D14FF0FF3003
:10CB900070474FF0000070474FEA4102B2F1E043A6
:10CBA00024BFB3F5001CDCF1FE5C0DD901F0004C94
:10CBB0004FEAC0024CEA5070B2F1004F40EB8300E4
:10CBC00008BF20F00100704711F0804F21D113F110
:10CBD0003872BCBF01F00040704741F480114FEA49
:10CBE0005252C2F11802C2F1200C10FA0CF320FAD2
:10CBF00002F018BF40F001004FEAC1234FEAD323EF
:10CC000003FA0CFC40EA0C0023FA02F34FEA430358
:10CC1000CCE77FEA625307D150EA01331EBF4FF0E1
:10CC2000FE4040F44000704701F0004040F0FE40FC
:10CC300040F40000704700BF80F0004002E000BFF9
:10CC400081F0004142001FBF5FEA410392EA030FF7
:10CC50007FEA226C7FEA236C6AD04FEA1262D2EB41
:10CC60001363C1BFD218414048404140B8BF5B4246
:10CC7000192B88BF704710F0004F40F4000020F0DF
:10CC80007F4018BF404211F0004F41F4000121F0F5
:10CC90007F4118BF494292EA030F3FD0A2F101023F
:10CCA00041FA03FC10EB0C00C3F1200301FA03F17D
:10CCB00000F0004302D5494260EB4000B0F5000FA0
:10CCC00013D3B0F1807F06D340084FEA310102F15F
:10CCD0000102FE2A51D2B1F1004F40EBC25008BF11
:10CCE00020F0010040EA03007047490040EB0000DB
:10CCF000013A28BFB0F5000FEDD2B0FA80FCACF1DC
:10CD0000080CB2EB0C0200FA0CF0AABF00EBC25008
:10CD100052421843BCBFD0401843704792F0000FF6
:10CD200081F4000106BF80F400000132013BB5E749
:10CD30004FEA41037FEA226C18BF7FEA236C21D0BF
:10CD400092EA030F04D092F0000F08BF0846704724
:10CD500090EA010F1CBF0020704712F07F4F04D1F2
:10CD6000400028BF40F00040704712F100723CBF05
:10CD700000F50000704700F0004343F0FE4040F42F
:10CD8000000070477FEA226216BF08467FEA2363ED
:10CD90000146420206BF5FEA412390EA010F40F4D8
:10CDA000800070474FF0000304E000BF10F0004324
:10CDB00048BF40425FEA000C08BF704743F096430B
:10CDC00001464FF000001CE050EA010208BF704726
:10CDD0004FF000030AE000BF50EA010208BF7047AD
:10CDE00011F0004302D5404261EB41015FEA010CC2
:10CDF00002BF84460146002043F0B64308BFA3F1BA
:10CE00008053A3F50003BCFA8CF2083AA3EBC2539B
:10CE100010DB01FA02FC634400FA02FCC2F12002BA
:10CE2000BCF1004F20FA02F243EB020008BF20F0F1
:10CE30000100704702F1200201FA02FCC2F1200257
:10CE400050EA4C0021FA02F243EB020008BF20EA4C
:10CE5000DC7070477BB972B90029BEBF00204FF06B
:10CE6000004106E008BF00281CBF6FF000414FF0F2
:10CE7000FF3000F007BAADF1080C6DE904CE0029CF
:10CE800009DB002B1ADB00F095F8DDF804E0DDE9A2
:10CE9000022304B07047404261EB4101002B1BDBD1
:10CEA00000F088F8DDF804E0DDE9022304B0404238
:10CEB00061EB4101524263EB43037047524263EB23
:10CEC000430300F077F8DDF804E0DDE9022304B065
:10CED000404261EB41017047524263EB430300F073
:10CEE00069F8DDF804E0DDE9022304B0524263EBA7
:10CEF0004303704753B94AB9002908BF00281CBF33
:10CF00004FF0FF314FF0FF3000F0BCB9ADF1080C2D
:10CF10006DE904CE00F04EF8DDF804E0DDE902230F
:10CF200004B07047430803F05533C01A830803F078
:10CF3000333300F03330184400EB101000F00F30A2
:10CF400000EB002000EB0040000E704707EE900A57
:10CF5000F5EEC07AF1EE10FA01D400F00BB8F1EE64
:10CF6000677A08B517EE900A00F004F8404261EBCA
:10CF7000410108BDD0B5FFF7BFFA0C4B00220646B1
:10CF80000F46FFF711FBFFF7E7FD0446FFF792FAA4
:10CF9000074B0022FFF708FB02460B463046394696
:10CFA000FFF74AF9FFF7D8FD2146D0BD0000F03D5C
:10CFB0000000F0412DE9F047089D04468E46002B05
:10CFC0004DD18A42944669D9B2FA82F252B101FA3D
:10CFD00002F3C2F1200120FA01F10CFA02FC41EA4D
:10CFE000030E94404FEA1C48210CBEFBF8F61FFAD2
:10CFF0008CF708FB16E341EA034306FB07F199426D
:10D000000AD91CEB030306F1FF3080F01F8199421F
:10D0100040F21C81023E63445B1AA4B2B3FBF8F0F9
:10D0200008FB103344EA034400FB07F7A7420AD980
:10D030001CEB040400F1FF3380F00A81A74240F2A8
:10D0400007816444023840EA0640E41B00261DB113
:10D05000D4400023C5E900433146BDE8F0878B4248
:10D0600009D9002D00F0EF800026C5E90001304607
:10D070003146BDE8F087B3FA83F6002E4AD18B42E1
:10D0800002D3824200F2F980841A61EB030301208B
:10D090009E46002DE0D0C5E9004EDDE702B9FFDE77
:10D0A000B2FA82F2002A40F09280A1EB0C014FEA22
:10D0B0001C471FFA8CFE0126200CB1FBF7F307FB7F
:10D0C000131140EA01410EFB03F0884208D91CEB22
:10D0D000010103F1FF3802D2884200F2CB804346BF
:10D0E000091AA4B2B1FBF7F007FB101144EA01449E
:10D0F0000EFB00FEA64508D91CEB040400F1FF312D
:10D1000002D2A64500F2BB800846A4EB0E0440EA1A
:10D1100003409CE7C6F12007B34022FA07FC4CEA23
:10D12000030C20FA07F401FA06F31C43F9404FEA16
:10D130001C4900FA06F3B1FBF9F8200C1FFA8CFE2B
:10D1400009FB181140EA014108FB0EF0884202FA7F
:10D1500006F20BD91CEB010108F1FF3A80F0888040
:10D16000884240F28580A8F102086144091AA4B2FD
:10D17000B1FBF9F009FB101144EA014100FB0EFE7E
:10D180008E4508D91CEB010100F1FF346CD28E45AD
:10D190006AD90238614440EA0840A0FB0294A1EB3E
:10D1A0000E01A142C846A64656D353D05DB1B3EB9B
:10D1B000080261EB0E0101FA07F722FA06F3F140CB
:10D1C0001F43C5E9007100263146BDE8F087C2F172
:10D1D0002003D8400CFA02FC21FA03F391400143EA
:10D1E0004FEA1C471FFA8CFEB3FBF7F007FB103623
:10D1F0000B0C43EA064300FB0EF69E4204FA02F4CF
:10D2000008D91CEB030300F1FF382FD29E422DD921
:10D21000023863449B1B89B2B3FBF7F607FB163356
:10D2200041EA034106FB0EF38B4208D91CEB0101D6
:10D2300006F1FF3816D28B4214D9023E6144C91A56
:10D2400046EA004638E72E46284605E70646E3E666
:10D250001846F8E64B45A9D2B9EB020864EB0C0E70
:10D260000138A3E74646EAE7204694E74046D1E77F
:10D27000D0467BE7023B614432E7304609E764442D
:10D28000023842E7704700BF02E000F000F8FEE716
:10D2900072B6374880F30888364880F309883648E4
:10D2A0003649086040F20000CCF200004EF63471BE
:10D2B000CEF200010860BFF34F8FBFF36F8F40F2D3
:10D2C0000000C0F2F0004EF68851CEF20001086076
:10D2D000BFF34F8FBFF36F8F4FF00000E1EE100AE6
:10D2E0004EF63C71CEF200010860062080F31488EF
:10D2F000BFF36F8FB3F06CFEB4F0B6FD4FF0553056
:10D300001F491B4A91423CBF41F8040BFAE71D49F3
:10D31000184A91423CBF41F8040BFAE71A491B4AEC
:10D320001B4B9A423EBF51F8040B42F8040BF8E73E
:10D3300000201849184A91423CBF41F8040BFAE713
:10D34000B3F04AFEB4F0E4FD144C154DAC4203DAE0
:10D3500054F8041B8847F9E701F082FB114C124D89
:10D36000AC4203DA54F8041B8847F9E7B3F032BE45
:10D37000000600200022002000C0000808ED00E0A8
:10D38000000000200006002038E30E0800220020E4
:10D390005C2B0020602B002080550120E0C100089C
:10D3A00030C2000830C2000830C200082DE9F04F3A
:10D3B0002DED108AC1F80CD0C3689D46BDEC108AD3
:10D3C000BDE8F08F002383F311882846A047002092
:10D3D000B2F0F2FDFEE7B2F05FFC00DFFEE7000016
:10D3E00001F0FF01102A2BDB10F0070F08D010F816
:10D3F000013B013A8B422DD010F0070F42B3F6D11A
:10D40000F0B441EA012141EA014122F007047FF032
:10D4100000070023F0E80256083C85EA010586EA89
:10D42000010685FA47F5A3FA87F586FA47F6A5FAC5
:10D4300087F68EB9EED1F0BC01F0FF0102F00702D1
:10D4400032B110F8013B013A83EA010313B1F8D17C
:10D450000020704701387047002D06BF354603385D
:10D46000073815F0010F07D1013015F4807F02BF96
:10D47000013015F4C03F0130F0BC0138704700BFE7
:10D4800010F8012B11F8013B012A28BF9A42F7D06E
:10D49000D01A7047034613F8012B002AFBD1181A43
:10D4A0000138704738B50022002304460D46FFF7C7
:10D4B000EDFA28B920462946BDE8384000F00AB800
:10D4C000204605F1004100F005F8404261EB4101C2
:10D4D00038BD00BFD0B50C4B002206460F46FFF703
:10D4E00063F8FFF739FB0446FEF7E4FF074B002221
:10D4F000FFF75AF802460B4630463946FEF79CFEC7
:10D50000FFF72AFB2146D0BD0000F03D0000F041AE
:10D51000036800221B68184710B503685B6804465F
:10D52000984708B194F84D0010BD00002DE9F04176
:10D53000674B03F5A04490B094F99C2806460F462B
:10D54000002A00F0C28094F8E45835B9614A7FF0AF
:10D55000B9FA284610B0BDE8F081B3F9A4201AB991
:10D56000B3F8A220A3F8A420B3F8A430632B05D805
:10D57000594A394630467FF0A5FA002500212E226F
:10D5800004A80391B7F0E8FCD4F8FC07036803AAE9
:10D590001B6832219847804630B9504A03AB394660
:10D5A00030467FF08FFA4546B4F8D837A3F57A7342
:10D5B0009BB241F65832934206D9494B3A46202154
:10D5C00030467FF077F8002594F90C3A002B6BDD9C
:10D5D00094F9C439002B5BDD424B3A46202130469A
:10D5E0007FF068F800254049D4F80808322303AAE0
:10D5F0008AF014FA804640B903AB00933A463B4B9D
:10D60000202130467FF056F845463949D4F80408C1
:10D61000322303AA87F034FA804640B903AB009363
:10D620003A46324B202130467FF044F845462021CF
:10D6300030467FF037F8C8B104F65803D3ED007ACE
:10D640009FED2C7AF0EEE77AF4EEC77AF1EE10FA5D
:10D650000CD594F90C3A002B02DD94F8703A2BB9F2
:10D66000254A394630467FF02DFA002594F90C3AC8
:10D67000002B7FF76EAF94F9C938002B3FF469AFE8
:10D680001E4B3A46202130467FF014F8002560E713
:10D6900094F8708AB8F1000F06D1194B3A46202150
:10D6A00030467FF007F8454694F9C439002B9ADDDF
:10D6B00094F8F589B8F1000F95D1124B3A46202124
:10D6C00030467EF0F7FF45468DE7012541E700BF74
:10D6D000702B0020A8930C08CA930C08F1930C0837
:10D6E000FC930C080E940C087F940C0883940C088F
:10D6F00095940C080000003499940C08B3940C081D
:10D7000034940C085A940C0838B504467EF0AEFFE9
:10D71000114B93F8A819114B1D68EB6A1A68002980
:10D7200008BF01461268184690475AF031FCEB6A70
:10D7300093F89C1059F066FD94F837305BB190F087
:10D7400085FDEB6AD3F8A030C01AB0F5FA6F24BF9C
:10D75000002384F8373038BD707B00206C2B00200C
:10D7600008B5FFF7D1FF054B05481B68DB6A93F846
:10D770009C10BDE8084010F0D3BF00BF6C2B002008
:10D780004083002070B50E46054664F06BFD64F0E2
:10D790002DFD10B90124204670BD0A4B93F9B2311A
:10D7A000012BF7D164F05EFD437A002BF2D164F0D7
:10D7B00059FD847A002CEDD1034A314628467FF08A
:10D7C00081F9E8E7704B0020CC940C087EF004BF90
:10D7D0002DE9F0472DED028BC47F90B006460F4631
:10D7E0008CB990F90430002B00F00581834B1D6843
:10D7F000A86A03685B6B9847044650B9804A39466B
:10D8000030467FF05FF9204610B0BDEC028BBDE8DA
:10D81000F087B3684BB933685B6B3946304610B05C
:10D82000BDEC028BBDE8F0471847E86AFFF774FECD
:10D8300004460028E7D1394630467FF0B7FFDFF8CD
:10D84000F4810546394630467FF064F998ED717AE7
:10D85000D8ED707AB4EEE77A2840F1EE10FAC5B24E
:10D8600009D598F9BC31032B05D0664A39463046B4
:10D870007FF028F92546D8ED597AB0EE088AF4EE03
:10D88000C87AF1EE10FA0BD517EE900AFEF734FEC7
:10D890005D4ACDE90001394630467FF013F9002595
:10D8A000D8ED5A7AF4EEC87AF1EE10FA0BD517EEED
:10D8B000900AFEF721FE554ACDE90001394630466F
:10D8C0007FF000F90025D8ED5B7AB8EE087AF4EE27
:10D8D000C77AF1EE10FA0BDD17EE900AFEF70CFE98
:10D8E0004B4ACDE90001394630467FF0EBF8002580
:10D8F000B8F95031042B07DC052200923946454A1D
:10D9000030467FF0DFF80025D8F8D00B64F006FD34
:10D9100080B198F9B2316BB1D8F8D03BB8F9B421E5
:10D92000B3F90E309A4205DA3B4A394630467FF069
:10D93000C9F8002539463046FFF724FFDFF8F8A084
:10D94000814639463046FFF7F1FD9AF8D53E002B67
:10D950004AD109EA050500EA050430484FF4806120
:10D9600001F062F878B1D8F8D03BB3F90C30A3F2EB
:10D97000E24292B2B2F5FA7F05D9294A39463046D9
:10D980007FF0A0F80024274890F828355BB100F517
:10D99000A46038F089F9054628B9234A394630464B
:10D9A0007FF090F82C4600212E2204A80DF10C08DF
:10D9B0000391B7F0D1FADAF8C00E4246322109F0ED
:10D9C0004FFB054600287FF41EAFDAF8C00E03684F
:10D9D0009B689847154ACDF8008003463946304683
:10D9E0007FF070F82C460EE7114A394630467FF03A
:10D9F00069F80024B1E7012405E700BF6C2B002083
:10DA0000DC940C08F3940C0816950C0836950C0859
:10DA100058950C087A950C0899950C08702B0020E5
:10DA2000D4950C08707B0020FC950C0874630D08DD
:10DA3000BF950C08704B0020706B002070B5054638
:10DA40000E46FFF79FFE3146044628467FF066FDEE
:10DA50002040C0B270BD0000F0B591B005460E4642
:10DA60007FF0F8F80446D8B1102128467EF01AFE5F
:10DA7000B0B100212E2204A803AF0391B7F06CFAD5
:10DA80001BF074FD32233A4601211BF02FF80446A7
:10DA900030B9054B00973246102128467EF00AFE29
:10DAA000204611B0F0BD00BF10960C0870B50546B9
:10DAB0000E46B1B990F910408CB1164813F05AFDDA
:10DAC000DFED157AB0EEC00AB4EEE70AF1EE10FA17
:10DAD00007D4124A012128467EF0F4FF344620463E
:10DAE00070BDAB689BB10E4B1B68D86AFFF714FD85
:10DAF000044630B163F00AF90A4A04215CF08AFA5C
:10DB0000EDE731462846BDE870407FF06FBB012449
:10DB1000E5E700BF702B0020000000341C960C08C5
:10DB20006C2B00202E960C0838B504467FF0F8FECA
:10DB30000546A8B10B4806F043F938B10A490B482D
:10DB40001BF02CF910B1074800F040FF2046FFF70A
:10DB500007FE0123064984F8373020467FF0F6FDA2
:10DB6000284638BD702B002078820020D83D002048
:10DB700050960C08F8B505460E461746C2B1232943
:10DB800001D0012914D8244808F030FD044668B1BA
:10DB900000242046F8BD95F91030022B08D063F020
:10DBA000B5F81E4A06215CF035FAF2E7002EF2D0F5
:10DBB0003A46314628467FF05FFF04460028E7D00A
:10DBC000174ED6F8C02E06F542639A4203D006F5EA
:10DBD000A95038F09FFCD6F8C00E124F03689B6B1B
:10DBE0009847D7F8203887F8F804012B07D164F05C
:10DBF00039FB542165F0FAFA08B9C7F8200828461D
:10DC0000FFF7AEFD4FF0FF330749C6F8F83E284650
:10DC10007FF09CFDBDE700BF702B002060960C08D4
:10DC2000706B0020707B002078960C082DE9F04F77
:10DC30002DED028BDFF8449191B0074688467EF0C7
:10DC4000DDFD99F987510446CDB94548BD2138F02D
:10DC5000F7FB38B1434B42464FF4804138467EF0E3
:10DC600029FD2C463E48BC2138F0EAFB38B13E4B3A
:10DC700042464FF4804138467EF01CFD00243B4E66
:10DC800096F8E438002B64D01C22002102A8B6F8D4
:10DC900054A5DFED378AB7F05FF904A821F0E4F965
:10DCA00006F5A46B0125A6F5A046554551D20BA853
:10DCB00021F0DAF909AA2946584636F07DF80028FD
:10DCC00047D0BDF82610304607F09CFD80B3BDF864
:10DCD0000A30102B2CD104A90BA821F0F5FC09F671
:10DCE000E843B0EE408A93ED000A2248B4EEE80A19
:10DCF000F1EE10FAB8BF99ED550A20EE000A0EF0C9
:10DD00001BFEF6EE087A60EE277AB4EEE78AF1EEB3
:10DD100010FA0DD517EE900AFEF7EEFB164BCDE983
:10DD2000000142464FF4804138467EF0C3FC002497
:10DD30000DF1240CBCE80F000DF1080EAEE80F0049
:10DD40009CE80700AEE8030001358EF80020ADB274
:10DD5000ABE7204611B0BDEC028BBDE8F08F00BFF1
:10DD6000908000208C960C08B8960C08707B0020E0
:10DD70000000003440830020EB960C08704B00201C
:10DD800000207047014800F0A1BD00BF702B0020AB
:10DD900003685B681847000067F0A6BC64F0B0B980
:10DDA0002FF0D2BF59F0ACBB08F074BD0DF0E4B950
:10DDB00014F03EBE03F0E8BA57F08ABA1FF06ABB0F
:10DDC00067F038B814F09ABE13F052BC1EF0E8BEEB
:10DDD00069F00ABA63F0AEBE62F068B807F0FABE46
:10DDE00005F014BA0CF0B6BC0DF024B914F05CBC0C
:10DDF00014F032BF13F06EBA14F094BD01F096BB6C
:10DE000000F2545022F0C8B908F07EBA90F8C4323B
:10DE1000B02202FB030390F8082393F8A13012B15B
:10DE2000012B28BF012318467047000090F81431D9
:10DE30000BB190F841311846704700000348086064
:10DE40002921117008221A60704700BF1C9A0C0823
:10DE5000F8B5044604F5935600F5AF40083008368F
:10DE6000FFF752FC002130461BF0F2FA80212046D9
:10DE700015F060F918B131F05BFB2FF02BFC04F5C5
:10DE80000055D5ED597A9FED317A67EE877A05F620
:10DE9000E437FDEEE77A04F5B44017EE903AC5F8A2
:10DEA000E03BD5F86C313B60083015F045FBF8B924
:10DEB000D5F8E03B07EE903A04F5805303F2B44204
:10DEC00092ED007AF8EEE77A03F5966367EE877ACB
:10DED000FDEEE77A17EE902AC5F8E02BD3ED007A35
:10DEE00097ED007AF0EEE77A67EE877AC7ED007A71
:10DEF00004F5AD5106F5457035F0DCF904F5A8459B
:10DF000094ED467AD5ED1E7AE7EE007AC5ED1E7ADD
:10DF1000B0EE670A32F030F804F5AF4085ED1E0A26
:10DF200050300DF011FE04F5AF4000215C3083F05D
:10DF3000E3FC4FF40011204615F0FCF820B1304608
:10DF4000BDE8F84019F0AEBBF8BD00BF0000C84204
:10DF5000FFF77EBF70B500F580430546D3F8C00ECD
:10DF600003689B6B984705F5AF445034064620463E
:10DF700010F098FB05F5A043002893F8B73418BFBC
:10DF800000262BB926B105F53150383083F018FC46
:10DF9000204610F01DF818B92046FFF747FF20B1C2
:10DFA0002046BDE8704010F0CBBD70BDFFF7D2BF7A
:10DFB00038B54FF48011054615F0BCF8044620B979
:10DFC0000121284615F0B6F804460221284615F02E
:10DFD000B1F850B114B9284603F0FCF805F5935098
:10DFE0000830BDE8384019F05BBA002CF6D138BDD6
:10DFF000FFF7DEBF38B54FF48011044615F09AF8EC
:10E0000001210546204615F095F818B115B92046AE
:10E0100003F0E0F81021204615F08CF860B120469E
:10E0200003F0CAF94FF48001204615F083F818B9BF
:10E0300031F07EFA2FF040FC2021204615F07AF8CE
:10E0400028B1204603F02EFA204603F047FB4FF498
:10E050000051204615F06EF810B1204603F026FB63
:10E060008021204615F066F828B131F061FABDE84C
:10E0700038402FF053BB38BDFFF7BCBF10B5044686
:10E0800022F07AF990F921308BB190F8403373B1D6
:10E0900094F978355BB1064B1B68DB6A93F89C30CA
:10E0A0002BB904F25450BDE8104021F08DBE10BDD4
:10E0B0006C2B0020FFF7E2BF2DE9F041424B1B68BB
:10E0C000DB6A93F89C300446002B7AD000F580562A
:10E0D00096F87135002B74D008F088FA002870D0BB
:10E0E00004F5F455103596F8DE1F284618F07CFD2F
:10E0F000002866D004F590773846FFF787FE02289F
:10E100005FD994F8E4334FF0B00808FB034393ED74
:10E11000777AF1EE007AB4EEE77AF1EE10FA50D4A5
:10E1200096F8DE1F284619F00FF804F50053B3F9EE
:10E13000502107EE902AB8EEE77AB4EEC07AF1EEFD
:10E1400010FA0CDD94F8E42308FB0242F8EE677A3B
:10E1500092ED777AF4EEC77AF1EE10FA31DCD6F868
:10E160006024D3F8E01B002AB8BF52428A4228DC60
:10E1700006F26442D2ED007AD3ED5A6A9FED136A3B
:10E18000F8EEE77A66EE866AF4EEE67AF1EE10FAD9
:10E1900017DC03F6E43292ED007A27EE067AF4EE0D
:10E1A000C77AF1EE10FA0CD494F8E413B02202FB13
:10E1B00001712846B3F95221BDE8F041D43118F07D
:10E1C00091BBBDE8F08100BF6C2B00200000C8426D
:10E1D000FFF772BF2DE9F04190F8E4332D4D00EBCD
:10E1E00003132F68D3F8948100F5907604463046E7
:10E1F000FFF70CFE474514D0022814D904F58047D8
:10E20000C5F8008097F8F03E012B15D817D104F51A
:10E21000A045D5F81037E3B9D5F81437CBB90523A5
:10E220000BE0022810D804F5804393F8F02E5AB181
:10E23000052283F8F02E07E0013B87F8F03E04F555
:10E24000B55004301CF046FB2046BDE8F0410CF010
:10E250006DBC114B1B68D86A03685B6898478046A1
:10E260000028ECD194F8E413B02303FB0161AC3136
:10E27000204605F017FED5F8F4360FCB05F5DF661E
:10E2800005F5E36586E80F0085E80F0087F8F08E56
:10E29000D5E700BF602B00206C2B0020FFF79ABF52
:10E2A000F8B500F5A047044697F8E43800F5805625
:10E2B000BBB100F5B440083015F044FC18B101239F
:10E2C00086F87135F8BD04F5AF45503528460FF096
:10E2D0007FFE08B10023F3E72846FFF7A7FD0028DB
:10E2E000F8D197F8B734002BF4D1D7F8FC34042BCD
:10E2F000E5D104F5AC4038308CF074FC86F871053B
:10E30000E0E7000010B500F5804400F59843D4F82C
:10E31000C01E2033994200F5A04308D000F59B426F
:10E32000283291421CBF4FF0FF32C3F8702403F52E
:10E330008C620749116003F26443064A1A60FFF7D2
:10E34000AFFFD4F8C00E0368BDE810401B69184742
:10E350000000C8420000C8C2FFF7D4BFF7B500F5FF
:10E36000A0470446D7F8FC348B420D4624D00B1F3F
:10E3700000F5AC46594206F1380659413046019144
:10E380008CF020FB019930468CF01CFB072D0BD143
:10E3900004F54E50D7F880246423052192FBF3F353
:10E3A0000830064A5BF036FE2046C7F8FC5403B03E
:10E3B000BDE8F04003F0E0B803B0F0BD7C970C0876
:10E3C00070B500F580460446D6F8C00E03689B6B16
:10E3D0009847B8B104F5A04595F8F83493B9D6F844
:10E3E000C02E04F5984320339A424CD104F5AF4631
:10E3F000503630460FF002F860B995F8B0347BB96A
:10E40000012108E004F5AF45503528460FF0E0FD46
:10E4100000283ED002212046BDE87040FFF79EBF95
:10E42000B5F85E35152B27D195F83C1611F0010192
:10E4300020D1D5F8FC34072B1CD095F9B2360BB996
:10E440000421E8E7204613F095F8DFED137AB4EEE7
:10E45000E70AF1EE10FAF3DB04F5AC4038308CF04B
:10E4600001FB0028ECD004F54E500C4A0621083080
:10E470005BF0D0FD0721CEE73046FFF7D7FC002840
:10E48000C8D10321C7E704F59B4328339A42F8D14A
:10E4900070BD2846F1E700BF0000B442A0970C0809
:10E4A00038B52F4DD5F8C02E05F542639A422DEDB3
:10E4B000028B0446B0EE408A03D00020BDEC028BF4
:10E4C00038BD28480EF09AFF40B1BDEC028B04F530
:10E4D000AF405030BDE8384010F0B2B805F5805478
:10E4E000D4F8FC34042B32D195F8F13E33B11E49F7
:10E4F000A1F5F47038F086FA0028DFD194F8E438FA
:10E500004BB118480EF07AFF0028D6D115480EF00E
:10E5100035FF0028D1D19FED157AF0EEC87AF4EEE0
:10E52000C77AF1EE10FA09D49FED110A28EE008A9D
:10E53000BDEEC88A18EE103AC4F880340D488CF04D
:10E5400091FA0028B9D0002384F8B334B6E7B4F8C0
:10E550005E15A5F5804007F055F90028C4D1ACE759
:10E56000706B00204083002078820020000000347F
:10E570000000C842A881002010B52DED028B00F5E7
:10E58000A0430446D3F8FC24042A0BD105F0D6F8A6
:10E590002046B0EE408A05F043F938EE400ABDEC63
:10E5A000028B10BD03F5E76393ED000AF7E7000067
:10E5B0002DE9F0412DED028B00F586658AB0044609
:10E5C00028461DF03FFB04F59350002307A90830AF
:10E5D0000793089309931AF0C7FD002800F08E8076
:10E5E0009DED090ADFED5C7A04F5A04505F592631F
:10E5F00093ED007A20EE270ADFED587AA7EE270A7E
:10E6000004F5AC40183004F5804783ED000A68F04B
:10E610003FFF2046FFF7D4FED7F8C00E03689B6B80
:10E620009847064604F5AF40503010F03BF895F897
:10E63000B734002818BF0026002B5AD1002E58D01E
:10E6400095F8F834002B54D1D5F8FC34042B6CD059
:10E650009FED438A204605F005F9C5F8340BD7F83D
:10E66000C02E04F598434C339A4204F500581AD151
:10E6700095F88037BBB9B8F9AC3B002B04DC394ABC
:10E68000D2F88C2BD2060ED5D5F8F416D5F8FC2688
:10E6900049680A33521A64214B438242ACBF9B182B
:10E6A0001B18C5F8343BD5F8341BD5F8FC34D7F823
:10E6B000F42E059120460492039316F03FFAB7F921
:10E6C000027F06462046FFF757FFCDE9006705F5B4
:10E6D000A36504F53150F0EE400ADDE90332D8EDD0
:10E6E0007B1A95ED001A0599B0EE480A383082F091
:10E6F0000BFD0AB0BDEC028BBDE8F08104F5907013
:10E70000FFF784FB02280AD994F8E433B02202FB15
:10E71000034393F8102212B193ED7F0A62E7284673
:10E720001DF02AF9B1EE400A5CE704F5AE4604F5A7
:10E73000AE48083608F1180804F5AD414246783174
:10E74000304620F02DFF002882D04146304620F090
:10E75000BBFFB0EE408A7DE7CDCC4C3ECDCC4C3FEC
:10E7600000000000704B0020FFF722BFF8B500F555
:10E77000804200F59943D2F8C02E40339A420446B5
:10E780000E4623D000F5AF47503738460FF020FC37
:10E790000546A8B138460EF097F870B104F5A044CC
:10E7A000D4F80C0803689B689847DFED097A20EEDF
:10E7B000270A86ED000A2846F8BD9FED060AF8E70D
:10E7C00004F5A9440125A3693360F4E70025F2E7C5
:10E7D0000AD7233C00000000F8B500F5804200F5A0
:10E7E0009943D2F8C02E40339A4204460E4630D0A8
:10E7F00000F5AF47503738460FF0EAFB0546A8B1A1
:10E8000038460EF061F870B104F5A044D4F80C0855
:10E810000368DB68984707EE900AF8EEE77AC6EDE2
:10E82000007A2846F8BDDFED0C7AF8E704F540548D
:10E830000125D4F8A40503681B69984707EE900AE0
:10E840009FED067AF8EEE77A67EE877AC6ED007AF2
:10E85000E7E70025E5E700BF000000000AD7233CFA
:10E86000F8B500F5804200F59943D2F8C02E403348
:10E870009A4204460E4624D000F5AF47503738463A
:10E880000FF0A6FB054688B138460EF01DF850B1D2
:10E8900004F5A044D4F80C38186988F029F886EDFE
:10E8A000000A2846F8BD9FED080AF8E704F5405431
:10E8B0000125D4F8A40503685B69984786ED000A32
:10E8C000EFE70025EDE700BF0000000030B505468A
:10E8D0000FC985B06C4684E80F0040F279322146BA
:10E8E000284605F071F90C4B03F68442D3F8C03E7C
:10E8F00093420ED19DF8001011F0040102D1204680
:10E9000020F04AFC0548214605F018FA012005B020
:10E9100030BD0020FBE700BF706B0020702B002093
:10E9200010B5044606480FF087F940B904F5804455
:10E93000D4F8C00E0368BDE810409B6C184710BDAA
:10E940004083002010B5044606480EF0C5FD40B9CE
:10E9500004F58044D4F8C00E0368BDE81040DB6CB9
:10E96000184710BD4083002070B5044600F5AF4045
:10E9700050300E4615460EF009F950B104F5A0448A
:10E98000D4F8843A9B682B60D4F8843A5B6833608F
:10E9900070BD04F5805303F58E6203F26C43126878
:10E9A0002A601B68336004F50054D4F88C3B9B0547
:10E9B000EED4D4ED7B6AD5ED007A9FED037AE6EED6
:10E9C000C77AC5ED007AE3E735FA8E3C38B50D4DD0
:10E9D000044629460C481AF0F3FA04F5804305F181
:10E9E000300183F8F10E04F5935008301AF080F9E5
:10E9F00004F5AE40D0ED0E7AF1EE677AC0ED0E7AF6
:10EA000038BD00BF78820020D83D002010B50446F4
:10EA100000F590702AF032F82046BDE81040FFF76C
:10EA2000D5BF0000FFF7F2BF00F50050D0F88C3BD7
:10EA3000194214BF012000207047000010B500F5F6
:10EA400080430446D3F8C00E03689B6D9847014687
:10EA500004F59C40BDE810408EF072BAFFF7EEBF9F
:10EA600038B5054B1C6823680A461D68034B0146F0
:10EA70002046A847002038BD6C2B0020702B0020BA
:10EA800070B52DED028B0446036804F500559B6DAF
:10EA90009847D5F88C3B1B0618D5B5F95031B5F918
:10EAA0005211CA1A0B4402EBD27203EBD373521009
:10EAB0005B1000EE902A00EE103A04F59350F8EE49
:10EAC000E00AB8EEC00A083019F098FE5A4BB5F8C3
:10EAD00082211A7004F5AF4565F042FC083565F0F7
:10EAE000D1F800212846FEF773FE544E0123B07181
:10EAF0002846F3717DF0BAFD28B928467EF03AFE2B
:10EB0000B0FA80F04009307128467DF0AFFD04F581
:10EB1000A045D8B994F8E43304EB031341F28832EA
:10EB2000D3F89461D5F88437F31A93420ED904F5DB
:10EB30009070FFF76BF9022808D9C5F88467204662
:10EB400005F03EF905F5C76300221A60B4F9A43058
:10EB50001BB9B4F8A230A4F8A430B4F8A430DFEDA7
:10EB6000388A07EE903AF8EEE77AB7EE008A88EE38
:10EB7000270AD4ED2B7AF0EEE77AF4EEE87AF1EE9C
:10EB800010FA09D5B4F9A23007EE903AF8EEE77A18
:10EB900088EE277A84ED2B7AD4ED2B0A31F0EEF84B
:10EBA00070BB57F039FD40F27D124FF4801157F0E1
:10EBB000EBFC56F043FC56F0ABF895F8E438B0EEB9
:10EBC000408A23B1D5F8040803681B6F984704F501
:10EBD0003C50B0EE480A343075F042FD04F5425026
:10EBE000B0EE480A103075F03BFDB0EE480ABDECBF
:10EBF000028B04F547500430BDE8704075F030BD1D
:10EC0000D4ED2B7A94ED460AF0EEE77AF4EEE87A4A
:10EC1000F1EE10FA09D5B4F9A23007EE903AF8EE09
:10EC2000E77A88EE277A84ED2B7AD4ED2B0A31F03F
:10EC3000A5F80028B5D0BCE7712300205587002037
:10EC400000000034FFF71CBF70B500F5A046044675
:10EC500096F9B036002B28DD07F0C8FC28BB04F578
:10EC6000AF45083528467EF085FDF0B128467DF099
:10EC7000FDFCD0B18FF0EAFAD6F8A034C01A96F9AC
:10EC8000B0364FF47A72534398420ED301221C21BE
:10EC90002846FEF76FFF40B104F54E50034ABDE829
:10ECA0007040062108305BF0B5B970BDC0970C0804
:10ECB00000B52DED028B9FED0B8AD0ED4E7A67EEFD
:10ECC000887A83B0C0ED4E7A3830019075F026FD19
:10ECD000019820EE080A03B0BDEC028B5DF804EB4E
:10ECE00075F034BE52B87E3F00B52DED028B9FED1E
:10ECF0000B8AD0ED4F7A67EE887A83B0C0ED4F7AF9
:10ED00003C30019075F00AFD019820EE080A03B02E
:10ED1000BDEC028B5DF804EB75F018BE52B87E3F77
:10ED200070B52DED048B044682B000F5935001A917
:10ED300008301AF0EBF9002800F0B78004F5A0467F
:10ED400006F5916595ED007ADDED017AB4EEE77A8E
:10ED5000F1EE10FA07D504F5AF4008307DF090FCD5
:10ED600008B1019B2B6004F5005595ED697AB5F962
:10ED70005031DFED5F6A052BB8BF052307EE903AEF
:10ED8000B5F95231F8EEE78A07EE903AF8EEE77AF5
:10ED9000B6EE009A77EEA77A1820C7EE270ADFEDC5
:10EDA000557A68EEA77AF4EE490A87EE271AF0EE54
:10EDB000007AF1EE10FAB4EE671AC8BFF0EE490A15
:10EDC000F1EE10FA48BFB0EE671ADDED017AF4EE0D
:10EDD000E67AF1EE10FACCBF87EE270AB0EE410AD0
:10EDE00031F0DEF804F5AF405030B0EE408A0FF05D
:10EDF000EFF828B996F8E438D3B396F81139BBB3D5
:10EE000004F5AF4008307DF03BFC88B328EE892A3A
:10EE10009DED011AB4EEC21AF1EE10FA28D5D5ED27
:10EE2000690ADFED351A9FED350AC0EE820A30F02F
:10EE3000E9FF04F53B503C30B4EE408AF0EE408AE6
:10EE4000F1EE10FA48BFF0EE488AFFF731FF04F503
:10EE50004150143004F54054FFF746FFD4EDC17A19
:10EE60009FED277A67EE877AB0EE688AC4EDC17AA3
:10EE7000244819F0F9F890B923484021FFF7D4FD50
:10EE800068B1224BD3F8FC34012B08D1F7EE007A9D
:10EE9000B4EEE78AF1EE10FA58BFB0EE678AB0EE32
:10EEA000480A02B0BDEC048B70BD04F5AF400830D9
:10EEB0007DF0E6FBB7EE008A0028D9D0462064F04A
:10EEC000F7FCB4EEC80ADFED127AF1EE10FAD8BF03
:10EED000B0EE480A87EE800AB3F08EFF2F209FED38
:10EEE0000D1ADFED0D0A31F05BF8B0EE408ABFE796
:10EEF00017B7D1383333333F000000006F12833A25
:10EF000052B87E3FD83D0020702B0020707B00203F
:10EF1000000034428FC2D53F9A99193FF8B5044694
:10EF200063F0A0F90368DB689847054610B900252F
:10EF30002846F8BD04F58046204607F0D3F9D6F8F8
:10EF4000C02E04F59A4350339A42074605D104F582
:10EF5000A04393F8A439022BE9D804F5AF40503010
:10EF60000FF05CFA0028E2D1D6F8C00E03689B6B64
:10EF7000984758B996F8D43E002BD9D004F50054E0
:10EF800094F9BC51023D18BF0125D1E7084BD3F8D5
:10EF9000C00E03685B6B98470028EBD004F5005463
:10EFA00094F9F931002BC2D0032BC0D03D46BFE706
:10EFB000706B0020F0B52DED028B044600F5804605
:10EFC00000F5AF4006F5716383B0503093ED008AD1
:10EFD0000FF038F904F53B5504F5A0473C350028FF
:10EFE00040D1D7F8040803689B689847D7F8943A4B
:10EFF0005B0221D5D7F8043893ED437AD3ED097A33
:10F0000067EE877A9FED2F7AF4EEC77AF1EE10FA69
:10F0100012DB04F53C5393ED007A67EE877AF7EE46
:10F02000006A86EEA77AB4EE667AF1EE10FAC8BFEF
:10F03000B0EE667A85ED497ADFED237A90ED250A08
:10F04000F0EE480A20EE270A28467FF02DFA2846DF
:10F050008DED010AFFF72CFE9DED010A03B0BDEC1A
:10F06000028BF0BDD6F8C02E04F5964330339A4299
:10F0700026D104F50053D3F8C83BB3F90860003E2D
:10F0800018BF012604F58054D7F81035D4F8604431
:10F090001C1B97F80C353BB10C484FF40061FFF78F
:10F0A000C3FC80F00100C3B23246B0EE480A2146EC
:10F0B000284603B0BDEC028BBDE8F0407FF0F8B904
:10F0C0000026DFE700000034E02E6542702B0020B0
:10F0D00010B5044606F0BEFC98B104F5A042D2F883
:10F0E000103503F58C415031C2F8101504F58051EC
:10F0F000D1F860140029BEBFA3F58C43503BC2F881
:10F1000010352046FFF756FFBDE81040042064F09C
:10F11000BBBB00002DE9F04700F5AF442DED048B9B
:10F1200000F580495034054609F571632046D3ED5A
:10F13000008A0FF087F805F5415605F5A04814360A
:10F14000002842D1D8F804080368DB689847D8F84B
:10F15000943A5B0221D5D8F8043893ED447AD3ED84
:10F160000B7A67EE877A9FED4F7AF4EEC77AF1EE6D
:10F1700010FA12DB05F5405595ED167A67EE877AA1
:10F18000F7EE006A86EEA77AB4EE667AF1EE10FA30
:10F19000C8BFB0EE667A85ED5F7A90ED250ADFEDA7
:10F1A000427AF0EE680A20EE270A30467EF0D6FD5D
:10F1B0003046B0EE408AFFF797FDBDEEC80ABDECC1
:10F1C000048BB8EEC00ABDE8F087204605F500576D
:10F1D0000DF0A8FB9FED359A97ED7B8AD8F8143592
:10F1E00028EE098A8246BDEEC88A462018EE102A0B
:10F1F0001A4408EE102A64F05BFBB8EEC88AD7ED1B
:10F20000657AD9F8C00EA0EE278A05F5964330330B
:10F210009842FDEEC87A17EE904A41D1D7F8CC3B20
:10F22000B3F90870003F18BF0127BAF1000F1CD1D5
:10F2300003685B699847C0B9D9F8C00E03689B6B37
:10F24000984790B9D8F82C3B022B0ED1284611F0E4
:10F25000DFFF50B108F5D263D3ED007A67EE897A0B
:10F26000FDEEE77A17EE903A1CB205F58055D5F819
:10F270006434E41A98F80C353BB10D484FF4006142
:10F28000FFF7D2FB80F00100C3B2B0EE680ABDEC1C
:10F29000048B3A4621463046BDE8F0477EF044BE36
:10F2A0000027C2E700000034E02E65420000C8429B
:10F2B000702B002010B5044615F088FD68B100B22F
:10F2C00000EB4000C0EB001300EE103AB8EEC00AAD
:10F2D000BDE81040132064F0D7BA2046FFF71AFFAC
:10F2E000F6E7000010B51048FFF718FED0B10F4840
:10F2F0000FF0CEF9B0B10E4C042064F0D9FAD4F876
:10F30000C80B63F01FFA042064F0BEFA132064F007
:10F31000CFFAD4F8CC0B63F015FABDE810401320F7
:10F3200064F0B2BA10BD00BF702B002040830020F3
:10F33000704B0020F8B52DED028B0446FFF7EEFD73
:10F34000002800F0AB8004F5804704F59642D7F81A
:10F35000C03E6832934200F0A18004F59742243207
:10F36000934200F09B8004F598420432934200F0EF
:10F37000958004F597424032934200F08F8004F567
:10F3800097425C32934200F0898004F599425C32E6
:10F39000934200F0838004F59942783293427DD005
:10F3A00004F59A421432934278D004F59A423432EA
:10F3B000934273D004F59A42703293426ED004F5B2
:10F3C000AF4050300FF064F9002867D0D7F8C02E56
:10F3D00004F596434C339A4260D004F50055F6EE9E
:10F3E000008AD5F8C80B63F06DF8B4EEE80AF1EEC8
:10F3F00010FA40DDB0EE087AFFEE007AE0EE077A10
:10F40000B0EE670AD5F8E02B04F5A04607EE902A87
:10F41000D6F81035B8EEE77A07EE903AF8EEE77ACC
:10F420005142E7EE007AFDEEE77A17EE900AC6F851
:10F43000100530F055FEC6F81005D7F8C02E04F5BB
:10F44000984368339A4222D0D5F8CC0B63F03AF84F
:10F45000B4EEE80AF1EE10FAB0EE408A21DCFEEEDE
:10F46000007AB4EEE70AF1EE10FA22D5B0EE087A8F
:10F47000F7EE007A19E0FEEE007AB4EEE70AF1EE5C
:10F4800010FABFD5B0EE087AF7EE007AB6E7254855
:10F490004FF48051FFF7C8FA0028D5D0BDEC028B9D
:10F4A000F8BDB0EE087AFFEE007AE8EE077AB0EE2B
:10F4B000678A204606F0CEFA08B1B1EE488AD6F83F
:10F4C0001435D5ED5A6A9FED186A05F6E43595EDC9
:10F4D000007AB5EEC08A07EE903AF1EE10FACCBF92
:10F4E00028EE268A27EE488AF8EEE77A66EE866AE4
:10F4F000E8EE067A27EE067AFDEEE77AFDEEE66A9A
:10F5000017EE903ABDEEC77A16EE902A17EE101A53
:10F5100017EE900AC6F8143530F0E2FDC6F814056F
:10F52000BCE700BF702B00200000C842F8B50446BD
:10F5300004F5A0458EF08AFE95F8E438074653B1ED
:10F54000D5F80C09036804F5AA4204F5AA411B6A20
:10F5500010321431984704F58046D6F8D03EFB1A95
:10F56000B3F5FA6F03D9D6F8C00E07F093FD2E4B12
:10F57000C6F8D07ED3F8C00E026813689847002101
:10F58000204611F0F7FFDFED297AB0EEC00AB4EEA5
:10F59000E70AF1EE10FA45D505F5E765D5ED007AF5
:10F5A000B1EE047AF0EEE77AF4EEC77AF1EE10FAF3
:10F5B00038D504F586601CF0DFF9F6EE007AB0EE7F
:10F5C000C00AB4EEE70AF1EE10FA2BD504F5B355F4
:10F5D00095ED037AF0EE087AB4EEE77AF1EE10FAE0
:10F5E00005F10C051ED504F53B503C307EF0D0FFF4
:10F5F00004F5415014307EF047FD04F546502C30A0
:10F600007FF074FC95ED007AF7EE007AB4EEE77ABD
:10F61000F1EE10FA06D504F54C502030BDE8F84064
:10F620007FF0BAB9F8BD00BF706B00200000003455
:10F6300000F5005090F94731012BC3BF00F6784028
:10F6400090ED290ADFED047A9FED040AC8BF20EE91
:10F65000270A462064F018B90000C84200000000E4
:10F660002DE9F8432DED028B00F5804909F5716312
:10F67000D3ED008A054611F0CFFB0746D9F8C00E3E
:10F6800003681B6A984705F546562C3698B14D4CD1
:10F69000D4F8DC34002B0EDD8EF0D8FDD4F8DC3449
:10F6A000C01A40F6B733984205D8B4F9D044304672
:10F6B0007FF028FC78E005F5A04805F5005498F89F
:10F6C000213B43B1B4F9D831002B04DD05F540539B
:10F6D00093F9C23103BBD9F8C03E05F596453035E4
:10F6E000AB426BD00021B0EE680A30467FF0A2F941
:10F6F0000546042064F0DCF82BB207EE903A94ED56
:10F70000637AF8EEE77AE0EE077AFDEEE77A17EE35
:10F71000904A3C4424B2CAE70121284611F06EFD0C
:10F720009FED297AB4F9D831C0EE077A08F21C5857
:10F7300008EE103A58F80C3C9FED240AB8EEC88A3F
:10F7400028EE278A07EE903AF8EEE77A67EE807A9D
:10F750009FED1F0A27EE800AB3F072F9B4F9503119
:10F76000DFED1C7A98ED007A20EE270A07EE903A3A
:10F77000F8EEE77A0021B4EEE77AF1EE10FA58BF1E
:10F78000F0EE477A80EE277A3046DFED137AB0EE5E
:10F79000480AA7EE270AF0EE680A7FF0A7FABDEE46
:10F7A000C00A10EE103A1CB2BDEC028B20460B4989
:10F7B000BDE8F84341F2941230F0A2BC391E18BFE4
:10F7C000012190E7707B002000A08C450AD7233CE4
:10F7D00035FA8E3C0AE81C41E02E65426CEEFFFFD4
:10F7E00038B500F540530546D3F8A4050368DB6837
:10F7F0009847014605F54C5020307FF0AFF804B231
:10F800002846FFF78BFB70B107EE904A05F50055CF
:10F81000B8EEE70AD5F8D40B62F094FFBDEEC00A4B
:10F8200010EE103A1CB220460349BDE8384041F2C0
:10F83000941230F065BC00BF6CEEFFFF38B590F855
:10F84000E433B02202FB030393ED777AF7EE007AFC
:10F85000B4EEE77AF1EE10FA054600F5A0441DD5A6
:10F86000002111F087FEDFED427AB0EEC00AB4EE5F
:10F87000E70AF1EE10FA11D5D4F8FC34012B0DD0C3
:10F88000072B0BD0002384F8743404F58F64002315
:10F8900023602846BDE8384011F0BEBA8EF0D6FC91
:10F8A000D4F87C34C4F87C04C31AB3F57A7F84BFDF
:10F8B000002384F87434284611F0AEFAD4F8FC34EE
:10F8C000012B07EE100A2DD0072B2BD0B8EEC77AEC
:10F8D000DFED286AC7EE267A05F50052B2F99C21C1
:10F8E00000EE102AB8EEC00A27EE800ADFED207A7B
:10F8F000B0EEC07AB4EEE77AF1EE10FA14D4002339
:10F9000084F8743494F8743405F54C502030DBB925
:10F910007EF00CFFBDE83840174900B241F2941266
:10F9200030F0EEBB9FED150A94F87424002AE9D15B
:10F930000122934284F87424E4D0072B1EBF04F5FF
:10F940008F6300221A60DDE704F58F6494ED007A7E
:10F95000DFED0B7A67EEC77A9FED0A7A67EE877A5A
:10F96000FDEEE77A17EE901A7EF0F8FFD2E700BFBF
:10F970000000003400A08C456CEEFFFF000000008A
:10F98000E02E65420000C84270B52DED028B00F5F7
:10F99000AC46383682B0044630468AF093FF0546BE
:10F9A000D8B904F50052D2F8C83BB3F9083073B99E
:10F9B00004F5AE43D3ED0E7A92ED667AF0EEE77A77
:10F9C000F4EEC77AF1EE10FA4CBF0125002530465F
:10F9D0008AF08CFF002808BF002530468AF072FFAD
:10F9E00050BB04F5A043D3F8703401331ED01DBBC7
:10F9F0009FED1C8A2046FFF733FE07EE900AB8EE13
:10FA0000E70A8DED010AFDB9152063F03DFF9DED7C
:10FA1000010A1A2063F038FF04F5B040583002B0F4
:10FA2000BDEC028BBDE8704003F0C2BB002DDFD0FF
:10FA30002046FFF703FF02E02046FFF7D1FE07EE66
:10FA4000900AB8EEE78AD5E71A2064F0C9F99DED6F
:10FA5000010A08B9B0EE480A152063F015FFB0EEB0
:10FA6000480AD6E70000000010B500F5005303F681
:10FA7000E432D3ED5A6ADFED127A92ED007A9FED0F
:10FA8000116A03F6784366EEA76A27EE277AD3ED6C
:10FA90002A7A67EE867AFDEEE66ABDEEC77AFDEE5B
:10FAA000E77A044616EE902A17EE101A17EE900A1F
:10FAB00030F016FB04F5A044C4F8140510BD00BFD7
:10FAC0000000C842A00CB34510B5044613F036FB45
:10FAD000031E2ADB04F5005191F947219A4224DDE7
:10FAE00004F5A040D0F8FC44022C1ED0D1ED687A79
:10FAF000DFED0E6AD31A66EEE76A07EE102A07EE0C
:10FB0000903AB8EEC77AF8EEE77AD0F8143587EE77
:10FB1000876A07EE903AF8EEE77AE6EE867AFDEE2F
:10FB2000E77A17EE903AC0F8143510BD0000C842CD
:10FB300070B52DED028B00F5A0449FED540AD4F86A
:10FB400010359FED537A07EE903AF8EEE77A0546C6
:10FB500067EE807A9FED4F0AF0EEE76AF4EE476AAF
:10FB6000F1EE10FAC8BFF0EE477A27EE800AB2F045
:10FB7000D7FD30F037F9B7EE008AC8EE007A04F509
:10FB8000A36305F50056C3ED007A94F8E438A3B1F9
:10FB9000D4F80C09036805F52F515B6A20319847AA
:10FBA00058B1D6F8E02BD4F81005514230F098FA4D
:10FBB000C4F81005BDEC028B70BD96F97831002BAE
:10FBC000F8D0284605F046FF0028F3D105F5B440EB
:10FBD000083013F0B1FC0028ECD1B6F95031012BFC
:10FBE000B8BF012307EE903A04F21C52F8EEE77A10
:10FBF000D2ED006A86EEA77AB4EEC87AF1EE10FA7A
:10FC000013D840F6C4122449D4F8100530F068FA2D
:10FC1000C4F81005D6F8E02B40F6C4139A42D4BFBE
:10FC2000C6F8E02BC6F8E03BC4E704F5A363D3EDC8
:10FC3000007AF4EEC77AF1EE10FABBDD88EE070A1F
:10FC400020EE000AB2F026FFDFED147AD4F810059A
:10FC500020EE270ADFED127A20EE270A40F6C413C1
:10FC6000FDEEC07A17EE905A9D42B8BF1D462A4657
:10FC7000694230F035FAC4F81005D6F8E03BAB42E3
:10FC8000D4BFC6F8E03BC6F8E05B93E70AD7233C55
:10FC90000000AA4235FA8E3C3CF6FFFFE02E65429A
:10FCA0000000C84210B500F540530446D3F8A4053F
:10FCB00003681B68984704F50053D3F8E02B5142C2
:10FCC00030F00EFA04F5A043C3F810052046BDE855
:10FCD0001040FFF72DBF0000704700000120704763
:10FCE0000820704701207047014B93F8840170474A
:10FCF000704B0020034B93F98409003818BF012092
:10FD0000704700BF704B0020014B93F9860170478C
:10FD1000704B002013B5064BD3F8C00E4B69046836
:10FD2000009308310EC9646CA04702B010BD00BF3B
:10FD3000706B0020704700007047000038B5254DFB
:10FD4000D5F8C00E03685B68984719283BD8DFE8F0
:10FD500000F00D38360D0D363636363A383838382C
:10FD600038383A36363636383A0D383840241A4B59
:10FD700093F8812312B193F880330BB944F0100447
:10FD8000164BD5F8C02E9A42A3F11C0303D09A4219
:10FD900018BF44F01004124991F9F911A9B19A421F
:10FDA00015D0032902D10F4B9A4201D144F04004EF
:10FDB0000D487CF05BFC50B144F0800407E0102457
:10FDC000D5E71824D3E70124D1E79A42F0D144F0D3
:10FDD000010038BD706B0020705B0020307800207F
:10FDE000704B002090770020F882002008B504486E
:10FDF00006F0FCFB00280CBF0120022008BD00BF5C
:10FE0000702B0020F0B52DED028B8BB0054619F05C
:10FE1000ADFB4FF48071D0F8047290ED828AD0F877
:10FE20000C6204461948FEF7FFFD30B9184BDFEDB0
:10FE3000197A93ED7B7AA7EE678A17480CF0A6FE35
:10FE400030B1164BD3F8843A5F6893ED028ADE68CE
:10FE50002D7C8EF0FBF9D4F81823D4F81C33D4F899
:10FE600014130892099327221C23CDE90032039032
:10FE7000079103AA1E21284604978DED058A069650
:10FE80005BF0E6F80BB0BDEC028BF0BD702B0020F0
:10FE9000704B002035FA8E3C40830020707B0020A0
:10FEA00038B5C5780B46352D044628BF3525352293
:10FEB00000211846B5F050F82A4604F10C01BDE8BF
:10FEC0003840B4F0FFBF000008B5024813F036F91F
:10FED00000B208BD702B002037B50D46134840F224
:10FEE000EF2203F071FE2C7814F004040AD0696844
:10FEF00003220F481FF0BEF80C4803B0BDE83040A5
:10FF000003F07ABA01AA214628461FF055F90028C5
:10FF1000F2D0DDED017A9FED077A67EE877A22460F
:10FF2000FDEEE77A17EE901AE3E700BF702B002092
:10FF3000888200200000C84210B5054C012384F8D7
:10FF400083335CF007FD002384F8833310BD00BFCA
:10FF5000705B00205FF058BE2DE9F0412DED028B63
:10FF60004FF0000882B0CDE900281E4F9FED1E8A99
:10FF70000C461546B0EE480AB1F90220D7F8C81B66
:10FF80004FF47A73064660F019F90123CDE9005366
:10FF9000B4F90020D7F8CC1BB0EE480A30464FF435
:10FFA0007A7360F00BF9B4F90420D7F8D01B9FEDF9
:10FFB0000F0A43463046CDE9005860F0FFF8CDE91E
:10FFC0000058B4F90620D7F8D41BB0EE480A4FF415
:10FFD0007A73304660F0F2F802B0BDEC028BBDE8F7
:10FFE000F08100BF704B00200000FA4400007A440A
:10FFF00008B55CF0A7FA40F4A67040F0010008BD17
:020000040801F1
:1000000010B504461FF038FC204610BD10B50C4C4E
:10001000002384F8B3345DF097F9A4F58052A4F579
:100020007873D2F8C02E9A4208D194F824352BB9AF
:1000300004F5A460BDE8104036F03EBC10BD00BF22
:10004000707B002013B5124C94F8DE1F04F5696034
:1000500016F0CAFD78B194F8DE1F04F5696017F058
:1000600031F840B194F8DE1F04F5696002B0BDE8D4
:10007000104017F069B819F079FA01A919F046F89B
:1000800018B19DED010A02B010BD9FED020AFAE71A
:10009000703B002000000000044B93F8E40820B1FE
:1000A000D3F80C0903681B6B18477047707B00205E
:1000B00008B5084BD3F8702B002A03DCBDE80840D4
:1000C0005CF084BA03F5296059F096FB90ED000AC4
:1000D00008BD00BF704B002008B51248D0F8C02EF4
:1000E00000F6A4439A4216D0B0F9D83EABB900F559
:1000F000805393F83D2482B990F8D52E6AB993F8CD
:10010000E93463B9A0F5804006F070FA00280CBF0E
:100110000320042008BD0220FCE70520FAE70620A2
:10012000F8E700BF706B002010B5224B03F54C625E
:10013000D3F8C03E934290B0044639D0002302F673
:10014000582002931EF080FF014618B91A4802AAEF
:100150001EF0C6FF247C8EF079F8184BDDED027A94
:10016000D3F82027D3F8243705930023F8EEE77A55
:100170009FED137A0793089309930A930B930C93BB
:100180000D930E934FF6F853ADF83C300023CDE9B4
:10019000030267EE877A96228DF83E303323CDE94D
:1001A0000032572103AA2046CDED067A5AF050FFBF
:1001B00010B010BD706B002088820020707B002082
:1001C0000AD7233CF0B58DB004468EF03FF8184AAC
:1001D000D2F80839C31A642B28D8D2F80438029010
:1001E000D3F88C10D3F89020D3F88460D3F88850DB
:1001F000D3F8DC70D3F894E0D3F898C0D3F89C30EF
:10020000099300238DF82C30069225231622CDE980
:1002100000320591207CCDF81CE002AA5321CDF8D4
:1002200020C00A97039604955AF012FF0DB0F0BD56
:10023000707B002010B55CF0CFFB044688B90A48FB
:10024000A0F58052A0F57873D2F8C02E80F8B344A0
:100250009A4206D190F824351BB900F5A46036F017
:100260002BFB204610BD00BF707B00202DE9F0471E
:100270002DED088B8D4CD4F8C02E04F54C639A42BA
:1002800090B0054600F0EB8003F531600CF07EFC89
:10029000DFED878ADFED879A9FED879A04F5805717
:1002A000002867D007F5FA600CF00EFB002861D03B
:1002B000D7F804089FED810A6C3032F07FFF07F217
:1002C000DC70B0EE60AAB0EE418ACDED070A8DED8C
:1002D000081AF0EE40AA8DED060A81F061FBD7F80E
:1002E00008380146D3F85C23D3F85833059204A8A4
:1002F000049332F063FD09A88DED090AB0EE680A97
:10030000CDED0A0A32F06AFD28EE288A02A8BDEE79
:10031000C88A95F81090CDED030A18EE103A8DEDCD
:10032000020A1EB232F0CEFDDFED657A20EE270A1A
:1003300002A8BDEEC00A6AEEA8AA10EE103A0FFAA3
:1003400083F832F009FEB4EEE90AF1EE10FA58BF74
:10035000B0EE690ABCEEC00AD4F8C02E10EE103A16
:100360009DB204F6DC439A422AEE28AA7CD1DFED46
:10037000558A7FE0D7F81035DFF84CA195F810903A
:10038000DAF8A48507EE903AD7F81435B8EEE7BA54
:1003900007EE903AD8F8003040469B68F8EEE7AA9E
:1003A000984707EE900AF8EEE77A404667EEA87A9B
:1003B00007F59367FDEEE77A04F6FC6417EE903AD2
:1003C0001EB2D8F800301B69984707EE900AF8EE85
:1003D000E77A97ED00AA67EEA87AB4EEE9AAFDEEF7
:1003E000E77AF1EE10FA17EE903ADFED327AAAF5DD
:1003F000405058BFB0EE67AA1DB203F0A1F8D8F87C
:100400000030D4ED007A5B6908EE100A404627EE12
:10041000899A9847B8EEC88ABCEECAAA2BEE28BAC9
:100420006AEEA8AA1AEE103A68EE288A8DED09BA8B
:10043000CDED0AAACDED0B8A8DED0C9A8DED0D0A4E
:10044000ADF83860ADF83A50ADF83C30B7221A2319
:10045000CDE900323E2109AA48465AF0F9FD10B014
:10046000BDEC088BBDE8F087D7F80838D3ED0F7ADC
:1004700067EEA88AD7F80C3804F6FC64D4ED007A4D
:10048000186927EE899A86F033FACDED09AA8DED29
:100490000AAACDED0B8A8DED0C9A8DED0D0AADF803
:1004A0003860ADF83A80ADF83C50CFE7706B002073
:1004B0000AD7233C00FF7F470000C8429F0CB3458A
:1004C000E02E654200000000705B002001480CF047
:1004D0000DBA00BF4083002008B5034BD3F8C00E0F
:1004E00003685B68984708BD706B002030B587B023
:1004F000054619F03BF804462D7C8DF09BFED4F8A0
:100500008422D4F888320492059300211023CD224E
:10051000CDE900320290039102AA42F60C3128463E
:100520005AF096FD07B030BD30B52DED028B89B085
:10053000054619F01BF800F55A7393E8070002AC62
:1005400084E80700DDED020A9DED030A2D7CF1EE43
:10055000600AB1EE400AB2F005FB2046B0EE408AD8
:1005600033F0B0FADFED0B7A049B079328EE278A6D
:100570000C230122CDE90032A82105AA28468DEDE1
:10058000058A8DED060A5AF063FD09B0BDEC028BB9
:1005900030BD00BFE02E6542422938B505461BD06C
:1005A0000AD824290CD0402924D01B2922D028463F
:1005B000BDE8384060F034B9432917D05329F5E736
:1005C0000C2159F043FF044610B90024204638BDE1
:1005D0002846FFF7A9FFF9E7102159F037FF044635
:1005E0000028F2D02846FFF781FFEFE7017C0248A0
:1005F0008AF066F90124E9E7A8810020F0B52DED25
:10060000028B05468DB01646B0EE408A0C46002996
:1006100030D0007C5AF0B2FC0746287C5BF0B2FB7D
:1006200000F121039F4207D2287C0DB0BDEC028B64
:10063000BDE8F04059F0F8BE63690893636A226927
:10064000CDF82530236AA069E1680792CDF82930FA
:100650006222212327680590CDE900320691287C8B
:100660000397192303AAC2218DED048A8DF8246013
:100670005AF0EEFC0DB0BDEC028BF0BDF8B54B4C62
:10068000D4F8C02E04F54C639A42054600F08C80E5
:10069000A4F50056B6F82232DF0713D544480DF012
:1006A00097FC002879D004F58054D4F80408036836
:1006B0009B68984700F1940191ED010A01222846B8
:1006C000FFF79CFFB6F822329C0712D538480DF090
:1006D0007FFC002864D0374BD3F804080368DB683C
:1006E000984700F1940191ED010A02222846FFF794
:1006F00085FFB6F82232580712D52D480DF068FC58
:1007000000284FD02B4BD3F8040803681B69984787
:1007100000F1940191ED010A03222846FFF76EFFD4
:10072000B6F82232190708D52349052291EDD50ADA
:10073000284601F55471FFF761FFB6F82232DA0658
:1007400016D51C4FD7F8FC34042B11D118F00EFF2E
:10075000044607F5C7608AF0E3F894EDC70ADFEDB9
:10076000177A014620EE270A06222846FFF746FFA1
:10077000B6F822329B0617D50D480DF029FC98B12A
:100780000C4BD3F80818284691EDAB0ABDE8F840A9
:10079000042201F52A71FFF731BFA4F6DC718BE763
:1007A0000749A0E70749B5E7F8BD00BF706B002017
:1007B00040830020707B0020705B0020E02E6542AB
:1007C000F05C0020645E002070B504460E4628F000
:1007D00093F990F8C412B02303FB0101AC31204619
:1007E00003F060FB0546C0B13EB118F0BFFE90F8C3
:1007F0007C3243F0020380F87C3204F58043D3F866
:10080000C00E04F598434C33984204D004F59A4442
:100810005034A04201D106F065FB284670BD0000AF
:1008200073B516460191044618F0A0FE019918F020
:10083000B5FA0546C0B13EB118F098FE90F87C328A
:1008400043F0020380F87C3204F58043D3F8C00EF5
:1008500004F598434C33984204D004F59A4450343C
:10086000A04201D106F03EFB284602B070BD000058
:1008700030B5054685B00C46D1E9040130F094FC52
:1008800040B168461EF0F0FB6A46214628465FF0FC
:1008900005FC08B9022067E0344840F24F3269464F
:1008A00003F092F9D4ED037AF4EE677AF1EE10FAE0
:1008B00022D69FED2F7AF0EEE77AF4EEC77AF1EECA
:1008C00010FA54BF012200229DF80030294962F33A
:1008D000410368468DF800301EF0FEFC0028D9D197
:1008E000254869466BF024FD40B957F051FB0522BD
:1008F000162157F0A9FACDE70022E5E7D4ED017AF9
:10090000FDEEE77A17EE903ADB0706D41B4B03F6B1
:100910008442D3F8C03E934225D11949134802229C
:1009200012F01CFA9DF8001011F0040102D1684683
:100930001EF032FC0D48694603F000FA94ED020AFD
:10094000B4EE400AF1EE10FA0BD6B5EEC00AF1EEA5
:1009500010FA06DD9DF800100948C1F3400107F0C8
:100960009DFC002000E0042005B030BD702B00206D
:100970000000003478820020B84B0020706B00200B
:10098000F477002010B52DED028BD1ED017A91EDB9
:10099000008AFCEEE77A8AB0CDED037A9DF80C1060
:1009A00005AA04465FF064FBC8B1DFED0E7A059B33
:1009B000009368EE277A0022FDEEE77A114617EEE3
:1009C000903A06A81EF070FB23682046D3F8C43086
:1009D00006A9984700200AB0BDEC028B10BD02208A
:1009E000F9E700BF0000C84237B5124DD5F8C00E78
:1009F00003681B6A0C46984740B9D5F8C02E05F528
:100A000042639A4202D0042003B030BDD4ED007A94
:100A1000D4ED020A94ED010A0748FCEEE77ACDED29
:100A2000017A9DF8041003F0EBFE0028EBD00020C3
:100A3000EAE700BF706B0020702B0020134610B552
:100A400024220C4618460021B4F086FAA27F827751
:100A5000E27FC277072280F82020A28B8283D4ED28
:100A6000067AF1EE677AC0ED067A10BD10B48C8B71
:100A7000162C03D15DF8044BFFF7E0BF5DF8044B83
:100A80005EF034BD08B591F82030072B0ED109482F
:100A900090F8E43843B191ED060A00F5FA60B1EE42
:100AA000400A0DF05BF818B9042008BD0220FCE7ED
:100AB0000020FAE7707B002008B5D1ED007A9FEDA9
:100AC000087A0848F0EEE77AF4EEC77AF1EE10FA09
:100AD00054BF0121002104F0B7FF002008BD00BF72
:100AE00000000034702B002010B5D1ED007AFCEE30
:100AF000E77A17EE903A9CB2012C02D0022C06D075
:100B000084B91148214666F031FC002010BD0F4821
:100B100090F82C365B0707D560F0F8F80C4A0521F1
:100B200059F078FA0420F1E790F918361BB960F013
:100B3000EDF8084AF3E7A0F5A0400AF049FB0028C9
:100B400014BF00200420E1E788810020707B002092
:100B5000589D0C08739D0C081FB5D1ED017AFCEE71
:100B6000E77A0B46CDED027AD1ED007A1A7C017C52
:100B70000192FCEEE77A0B48CDED037AD3ED027AD1
:100B8000FCEEE77A17EE902A92B2009293ED030AF8
:100B90009DF80C209DF8083009F084FC05B05DF844
:100BA00004FB00BF4083002007B5D1ED007A084860
:100BB000FCEEE77ACDED017A9DF804100BF096FA81
:100BC00000280CBF0420002003B05DF804FB00BF28
:100BD0004083002070B58B8BC02B05460C4633D864
:100BE000B12B0DD8142B00F0AE80162B59D0112B41
:100BF00000F0A68021462846BDE8704060F0A8BC01
:100C0000B23B0E2BF6D801A151F823F0910C01084C
:100C1000F50B0108F50B0108F50B0108F50B0108B0
:100C2000F50B0108F50B0108F50B0108870C01080D
:100C3000F50B0108BB0C0108F70C0108F50B0108C6
:100C4000AB0C01087D0C0108D42B13D007D8D02B96
:100C500023D0D12BCED1BDE87040FFF77DBFB3F5D7
:100C6000967F53D040F6B836B342C3D1BDE870404A
:100C7000FFF79ABFBDE87040FFF71EBF2146BDE8F1
:100C80007040FFF7F5BD2146BDE87040FFF77ABE22
:100C90002146BDE87040FFF7A7BEBDE87040FFF7F2
:100CA00023BFBDE87040FFF7EDBE94ED000A284871
:100CB000FDF7F6FBE8B100201CE0264C94F8F13E6D
:100CC000BBB1254904F5A95035F0F4FE88B104F50F
:100CD0008053012283F8592504F542610222A4F5CC
:100CE000804012F03BF80028E5D11C4B002283F82D
:100CF0005925042070BD174C94F8F13E002BF8D014
:100D0000154904F5A95035F059FEDFE7D1ED007A19
:100D10009FED137AF0EEE77AF4EEC77AF1EE10FA6F
:100D200014D5D1ED017AF0EEE77AF4EEC77AF1EE60
:100D300010FA0BD50B490222054812F00FF8BAE75A
:100D400009490222F8E709490222F5E70220D1E722
:100D5000702B0020706B002078820020707B0020B8
:100D60000000003490770020D8770020BC77002066
:100D700070B5434B03F68442D3F8C03E93428EB025
:100D80000C467BD1CD78272D28BF2725272200218F
:100D900004A8B4F0E1F82A4604F10C0104A8B4F068
:100DA00091F8059B9DF836400093069B0193E44320
:100DB000079B0293E4B2089B03938DF836408DF0B5
:100DC00045FA14F0810F04F08705064601D1802D05
:100DD00013D1684631F05CFDDFED2A7A2A4B20EE14
:100DE000270ADFED2A7AC3F8D46420EE270ABDEE85
:100DF000C00A10EE102AC3F8C82414F0820F01D1E3
:100E0000802D13D1684631F05DFDDFED1E7A1E4B5B
:100E100020EE270ADFED1D7AC3F8D86420EE270AFA
:100E2000BDEEC00A10EE102AC3F8CC2414F0840FD3
:100E300001D1802D13D1684631F054FDDFED117AD8
:100E4000114B20EE270ADFED117AC3F8DC6420EEA7
:100E5000270ABDEEC00A10EE102AC3F8D02463069C
:100E60000CD5DDED0C7A9FED097A074B67EE877A9A
:100E700003F59C62C2ED007AC3F8E4640EB070BD65
:100E8000706B0020E02E6542707B00200000C8429D
:100E900030B5214C91B0084602A9FFF701F8D4F80B
:100EA000C02E04F684439A4233D19DF83C30072B80
:100EB0002FD104F58054DDED056AD4F81C379FED81
:100EC000177A07EE903AF8EEE77AE6EEC77AFDEE8B
:100ED000E77A17EE903AC4F81C375FF017FFD4F8A2
:100EE000F426D4F81C3752689FED0D7A9B1A07EE52
:100EF000903AF8EEE77A054667EE877A17EE900AA1
:100F0000FBF7FAFA074ACDE900010621284659F015
:100F100081F811B030BD00BF706B00200000C842E6
:100F20000AD7233C8C9D0C0810B51D4B03F6844258
:100F3000D3F8C03E9342044696B008460FD108A9A4
:100F4000FEF7AEFF9DF8541003AA20465FF090F81C
:100F500038B95FF0DBFE134A042159F05BF816B094
:100F600010BDBDF8503023F004039BB2002BF6D027
:100F7000DDED0B7A9FED0C7A039B009367EE877A89
:100F80000022FDEEE77A114617EE903A04A81EF013
:100F90008BF8236804A9D3F8C43020469847DEE7CD
:100FA000706B0020A09D0C080000C84230B48D7A00
:100FB0004B7A43EA0523CD7A43EA0543562B044690
:100FC0000A4618D008D8522B0FD0542B10D02046E8
:100FD000114630BC5FF054B903F18073863B23F0B7
:100FE0007F43012BF3D830BC704730BCFFF7C0BE45
:100FF00030BCFFF74DBF30BCFFF796BF00207047F5
:10100000C8207047012070470020704700207047BB
:1010100090F890308B4286BF00EB8100D0F89400AE
:101020000020704790F890308B4286BF00EB810023
:10103000D0F894000020704703207047014B93F8CC
:1010400082017047704B002070B504463E4810F096
:101050008BFA18B1236A43F4000323623A4810F074
:1010600083FA88B1462062F023FCDFED387AB4EED3
:10107000E70AF1EE10FA07D8636A43F400036362EB
:10108000A36A43F40003A362236A43F4F843236290
:101090002F4BD3F8C00E03685B68984701381828B7
:1010A00015D8DFE800F0343C0D3E3C3C3C3C1434A9
:1010B0003434343434143C3C3C3C34143E3434003A
:1010C000244A92F8803353B392F8812352B3224BCF
:1010D0001D68DDB1214E284696F8BA1B4EF0F0FD92
:1010E000A0B1236A43F48073236296F920321BB1C6
:1010F000636A43F48073636296F8BA1B28464EF025
:1011000017FE18B1A36A43F48073A36270BDD4E9DB
:10111000092342F4E04243F4E0436262A362012304
:1011200000E00023616A41F480626262A26A42F4D4
:101130008060A062002BCAD041F4406142F440625A
:101140006162A262C3E700BF702B0020000000B400
:10115000706B0020705B0020FC870020704B00202B
:1011600013B54FF44470CDE900211EF07DFB044619
:1011700028B1DDE900215FF0E7FD024B2360204646
:1011800002B010BD9C9F0C080020704700207047E3
:10119000002070470020704700F50750243070474A
:1011A00000487047E8C50C0800F58040D0F8C00E34
:1011B00003685B681847000000F5804300F598401D
:1011C000D3F8C03E20301B1A5842584170470000E7
:1011D000A22070472DE9F04100F5A045DFED686AD7
:1011E000D5F8103507EE903AD5F81435B8EEE77A11
:1011F00007EE903AF8EEE77A00F5AF4890B027EEA8
:10120000267A67EEA67A08F1500804460023404685
:101210008DED017ACDED027A03930BF0B7FC002837
:1012200000F0A680D5F8043884330FCB0CAF87E8E4
:101230000F0008AE04AF87E80F0086E80F0001A991
:10124000384603AB02AA31F067FB9FED4E0AD5F892
:10125000847A01A831F0B2FF314638468DED080A94
:10126000CDED090A8DED0A1A16F07AFA8CF0EEFF30
:10127000D5F80839C01A632804F57C662DD8D5F84E
:10128000040803689B689847042100F194023046E3
:1012900055F0A0FED5F804080368DB6898470521DF
:1012A00000F19402304655F095FED5F80408036825
:1012B0001B699847062100F19402304655F08AFEDA
:1012C000D5F80828304602F52A72072155F082FE2B
:1012D00004F5B440083013F097F940460CF078FE5E
:1012E00090B1D5F8080884F0DFFF68B1D5F8082878
:1012F0006E219032304655F06DFED5F808286F21EA
:10130000BC32304655F066FE04F540522432692165
:10131000304655F05FFE04F546526A21304655F0DE
:1013200059FE04F5405393F9C22132B9D3ED6E7AD8
:10133000F5EEC07AF1EE10FA06DD04F54B523432C8
:101340006B21304655F046FE04F54C5420342046BF
:101350007DF026FB28B104F130026D21304655F0B6
:1013600039FE18F003F917F015FE10B0BDE8F08152
:1013700004F5935001A9083016F0BAF876E700BFDB
:101380000AD7233CE02E654210B54FF48011044685
:1013900011F0D0FE10B12046FFF71CFF4FF4800182
:1013A000204611F0C7FE28B12EF0C2F8BDE810406B
:1013B0002CF082BA10BD000030B500F5935591B005
:1013C00000230835029302A9002304460DF1070209
:1013D00028468DF8073017F09FFE03A9284616F01F
:1013E00093FE08B92D4B03933022002104A8B3F0DB
:1013F000B3FDA3238DF8103095238DF811308CF0B8
:101400002DFF04F5A042CDF81300D2F81035ADF849
:101410001B3004F58053D2F81425CDF81710462060
:10142000D3F86014D3F86434ADF81D10ADF81F2064
:10143000ADF8213062F03CFA10EE103A1520CDF8EC
:10144000233062F035FA10EE103ACDF8273004F56B
:1014500031539FED137AD3ED377A67EE877A2846BA
:1014600017EE903ACDF82B30029BCDF82F309DF837
:1014700007308DF83330039B0D9318F053F804F5C3
:1014800080433022D3F8043F8DED0E0A04A904F501
:101490007C600F9355F0CEFE11B030BD2292CA7F12
:1014A0000000C84270B58EB035220446002168465F
:1014B000B3F052FDA3238DF8003095238DF8013051
:1014C000012304F5A0458DF802308CF0C7FE04F529
:1014D000405605F59363CDF803001B68D6F8A405C4
:1014E000CDF80710CDF80B3003681B699847ADF8AD
:1014F0000F00D6F8A40503689B689847ADF8110063
:101500001C4802F01DF8ADF81300D6F8A4050368D6
:101510005B69984710EE103AD6F8A405CDF815305F
:1015200003689B69984710EE103ACDF8193004F51E
:10153000804303F6FC6135220968CDF81D10D5F80B
:101540002017CDF82110D5F82417CDF82510D5F89F
:101550001C17CDF82910D5F8341BD3F8F43ECDF87C
:101560002D1004F57C606946CDF8313055F062FEEF
:101570000EB070BD702B002030B587B01622044627
:1015800000216846B3F0E8FCA3238DF800309523D2
:101590008DF8013002238DF802308CF05FFECDF81B
:1015A00003002046CDF8071005F020F804F5AA4303
:1015B0008DF80B001B680393134B1B68D86A90F8D7
:1015C0009C308DF810300368DB69984704F5A0451E
:1015D0008DF8110095F8E9348DF812302DF0A8FF40
:1015E0002DF0F6F8D5F8FC348DF813008DF8143092
:1015F000162295F8EA348DF81530694604F57C60BA
:1016000055F018FE07B030BD6C2B002010B58AB025
:101610002722044600216846B3F09EFCA3238DF8E0
:10162000003095238DF8013009238DF802308CF0BD
:1016300015FECDF803000420CDF8071062F038F94C
:1016400010EE103A1320CDF80B3062F031F910EEA5
:10165000103A4620CDF80F3062F02AF910EE103A19
:101660001520CDF8133062F023F910EE103A032064
:10167000CDF8173062F02CF910EE103A1A20CDF8A0
:101680001B3062F015F910EE103ACDF81F3004F55A
:101690009E43103327221B68CDF82330694604F59A
:1016A0007C6055F0C7FD0AB010BD000013B50446BC
:1016B00000F57C60019055F0FBF8019855F092F927
:1016C00004F58053019893F978300BB155F032FA54
:1016D000204602B0BDE81040FFF798BF70470000F9
:1016E00030B500F5A04389B093F8E428044600F52E
:1016F0007C6552B1D3F8FC071E22694686F004FFD0
:101700000F496A46284655F031FF04F58043D3F867
:10171000C00E03685B68984704F50053014693F8D0
:101720000421284655F046FF04F59350083018F080
:1017300097F904F5907009B0BDE8304026F046BA3C
:10174000A8A00C089FED020A00224CF0A5BB00BF28
:101750000AD7233C134B70B5044640F8043B60F0B5
:1017600001FC114E114B63605425601960F0B0FD0F
:1017700066513035B5F5557FF7D104F5557062F0F7
:101780008DFC0B4A04F5EC6002F6343189F024FF3D
:1017900001232046074984F891394CF07BFF20460D
:1017A00070BD00BFB0370020C8F00C08DCF00C089A
:1017B000B44C0020D8E00C082DE9F04100F50651AA
:1017C0009AB00D22044654F05DF90022BD4827214D
:1017D0004CF0DAFA0421002062F0EAFB1321012028
:1017E00062F0E6FB4621022062F0E2FB15210320B5
:1017F00062F0DEFB62F0ACF904F5A04393F99C388B
:1018000023B19FEDB10AB1484DF0ECFA4DF048F923
:10181000AF4AB04E138843F0040313804FF0000822
:101820000AAF002110223846B3F096FB01238DF851
:1018300030303388ADF8283005A973680B933846EB
:101840004CF0AAF9C8B19DF91430002B15DD60F0F9
:1018500009FD9DF81410036801391B68C9B2984747
:1018600058B1051D28464CF035F930B9B368ADF8CC
:10187000183006A928464DF0CFFD08F10608B8F14A
:101880002A0F06F10C06CCD1934800220DF10B0172
:101890004BF008FF06AD064620B34CF01BF908BB21
:1018A0008E4B0FCB85E80F0004A928464CF074F945
:1018B000002840F033814FF00408894B0FCB87E8B4
:1018C0000F0005A938464CF067F928B105A84CF07F
:1018D00001F908B148F0010803A930468DF80C80E1
:1018E0004DF048FD7F4B0FCB85E80F0003A928463C
:1018F0004CF052F9002846D00998002204A94BF078
:10190000D1FE064600283ED04CF0E4F805460028FB
:1019100039D19DF80C30013BDBB2032B96BF724AE4
:101920000346D35C8DF82830304639464DF022FD11
:101930006E48002205A94BF0B5FE06466AF03AFF54
:1019400078B16AF035FF90F8302090F8281090F8C0
:101950004830114490F840200A44D34214BF012576
:10196000002586B130469DF90C804CF0B3F850B993
:101970001DB1B8F1000518BF0125394630468DF874
:1019800028504DF0F7FC04F506500022B7EE000A8F
:10199000022138304CF080FA012304F5F451009311
:1019A000534A002310318E204CF0F2F994F974C997
:1019B000BCF1000F1AD14F4E0FCE3D460FC50FCED2
:1019C0000FC50FCE0FC596E80F0085E80F006246E1
:1019D000042138464CF0D8F99FED470A47484DF0AE
:1019E00001FA4748B7EE000A4DF0FCF9012504F56D
:1019F0000151444A00950023083140F205104CF093
:101A0000C7F904F5075002212C30FFF79BFE04F5BF
:101A1000055003211430FFF795FE04F5055003210E
:101A20001C30FFF78FFE04F5075003212830FFF725
:101A300089FE04F5075002213030FFF783FE04F5DC
:101A4000055002212830FFF77DFE04F505500221E4
:101A50002C30FFF777FE04F5055002212430FFF704
:101A600071FE04F5AC40383089F0BEF8264A1368A0
:101A7000D90705D42549156004F5FF5310330B60D1
:101A800004F5085021490122283001254CF0D2F9F3
:101A90001F4A0095002304F57C61FD204CF078F985
:101AA0001C4B1A68D20705D41B4A1D6004F58C54E0
:101AB0000C341460184801214CF0D8F91AB0BDE874
:101AC000F08100BF14DE0C0800009643C0C60D086C
:101AD000E087002084E00C08D8DD0C086C910C082D
:101AE0007C910C088C910C0810DE0C08E3DD0C08CE
:101AF000D8210D089C910C0800000000F0DD0C08B6
:101B0000FFDD0C08B4540E08642B002000220020D6
:101B10002CAF0D08682B00200C22002004A84BF0ED
:101B2000D9FF00283FF4C7AE4FF00C08C5E600BF50
:101B30007047000000207047002070470020704769
:101B40000020704700207047704700000020704759
:101B50000020704784B001A880E80E0004B0002087
:101B60007047000000207047002070477047000059
:101B70001020704700487047C4EC0C0800487047BC
:101B8000D4EC0C080020704770470000012070471B
:101B90000120704700207047002343608360C360CA
:101BA00003614361002303767047000010B50446CB
:101BB000FFF7F2FF0023637610BD0000027E531C86
:101BC000DBB2042B037600EB820288BF002382ED98
:101BD000010A88BF0376704710B50446FFF7EEFF91
:101BE000D4ED017A9FED107A94ED020A637E77EED0
:101BF000877A042B77EE807A94ED030A94BF013341
:101C0000052377EE807A94ED040A637677EE807A86
:101C1000637E94ED050A77EE807A00EE103AB8EE16
:101C2000C00A87EE800A10BD0000000010B504460F
:101C30001DF022FE204610BD04F0ECB902F0F0BF0A
:101C400003F0C4BD02F0FABF01F084BC01F034BB64
:101C500001F05EBC01F0F4BCFCF7F6BFFCF7B0BBD2
:101C600070B51F4B036000F540530446D3F83805A8
:101C70001C4AC3F8882308B11DF002FE1A4B2360EA
:101C800004F5805393F82C2E42B9D3F8285E2DB179
:101C900028462AF099FE28461DF0EEFD04F58B50EB
:101CA00010307AF029F804F58350183063F0F6FA12
:101CB00004F6C44504F66446B54204D0183D2846EF
:101CC0002AF0D8FAF8E7094BC4F8983804F69410CB
:101CD00057F06EFA04F5106057F06AFA204670BDAE
:101CE00080D40C08D4C70D0898A80D089C6F0D0867
:101CF00038B5484B044640F8043B63F015FE04F148
:101D000010001BF073F804F1680053F06FF804F54D
:101D1000907025F03DFB04F5866019F003FE04F297
:101D200054501DF0AFFD04F698002BF0B1FE04F501
:101D3000446063F0D7FB04F551604DF0E7FE04F515
:101D40007C6055F0BFF904F58350183063F08EFACB
:101D500004F5855014301CF03BFB04F58B5010301B
:101D600079F0B6FF04F58C500C3053F001FC04F50B
:101D70008F5064F083FF04F580530025264A83F8D2
:101D8000045204F5905004F590530433143013605A
:101D900049F042FB04F593502946083015F096FEB1
:101DA00004F5C550183072F08FFE04F5E5501C3074
:101DB00076F0D4FF04F5EE50143079F0E3F804F532
:101DC000F150183079F018FD04F5F450103014F08B
:101DD0009FFD04F5FF50103073F0D4FA04F5015064
:101DE000083069F0BDFF04F5005304F5045083F892
:101DF00004510A4D1C307AF03FFB2B6813B10848A0
:101E00008CF0F2F9204607494CF044FC2C60204647
:101E100038BD00BF98A80D08D09000203088002061
:101E2000DCEC0C08C0A70D082DE9F04F2DED028B5E
:101E300004469FB0FFF75CFFE24B236004F50850B7
:101E40002830FFF787FC04F52F5004F500577BF08E
:101E500033FE04F507530A33C7F8E83B04F5305066
:101E6000062387F8EC3B143062F012FE04F5315380
:101E700038330E9304F5AC433833C7F8903C0F93D6
:101E80004FF40063C7F8943C5A2387F8143D04F5D7
:101E9000055907F6784304F5935809F10409CA4A2D
:101EA000DFEDCA8AC7F88C9C08F10808C7F8888C4F
:101EB000B7EE008AC3F8602104F53950C44AC3F86C
:101EC0006821C3F8CC2183ED578AC3ED598A1430B9
:101ED00057F08EFC04F53950203057F089FCBD4B8B
:101EE000C7F8703E0E9B002687F8886E03F5FC70DD
:101EF000FFF752FEB84BB949C7F8703E87F8896EB4
:101F00000E984CF0C7FBB64BC7F8903E0E9BC7F837
:101F1000983E07F569630022C7F8948E04F53A5598
:101F20005A63DA6304F53B50012387F8D43E103539
:101F300028301DF099F887F8F86EAA4928464CF029
:101F4000A9FB04F53B5049463C307CF06BF904F5A5
:101F50004150494614307BF0C9FD04F546504946CE
:101F600004F540572C307CF027FD2C22314607F534
:101F70005470B2F0F1FF04F54C509B49203004F549
:101F80004E564CF087FB0836984BC7F8883306F15D
:101F900008008BF01FFB04F54E5A04F5505B0AF164
:101FA000340A0BF1180B50460AF1140A5CF090F950
:101FB000D345F8D10723C7F83C350023A7F84035AF
:101FC0004FF4CB701DF056FCC7F8380504F555509A
:101FD00004308BF0FFFA04F5565008308BF0FAFA13
:101FE000834B1A6802B91E60824BC7F8883304F528
:101FF00056504FF48051C7F8A45528301AF0D0FF3E
:1020000004F5585028304DF0BDFA04F558503C30D6
:102010006BF04CFF04F5964004F58045143004F055
:1020200035FF754BC5F8143B04F59640303004F08D
:102030002DFF724BC5F8303B04F596404C3004F050
:1020400025FF6F4BC5F84C3B04F59640683004F013
:102050001DFF6C4BC5F8683B05F53963002204F59C
:102060009740DA609A605A6083ED008A243004F069
:102070000DFF654BC5F8A43B04F59740403004F0D4
:1020800005FF624BC5F8C03B04F597405C3004F097
:10209000FDFE5F4BC5F8DC3B04F59840043004F0CE
:1020A000F5FE5C4BC5F8043C04F59840203004F084
:1020B000EDFE594BC5F8203C04F598404C3004F037
:1020C000E5FE564BC5F84C3C04F59840683004F0EA
:1020D000DDFE534BC5F8683C04F59940043004F527
:1020E000994604F0D3FE24364E4BC5F8843C304666
:1020F00004F0CCFE4C4BC5F8A43C04F599404030AC
:1021000004F0C4FE494BC5F8C03C04F599405C306E
:1021100004F0BCFE464BC5F8DC3C04F59940783031
:1021200004F0B4FE434BC5F8F83C04F59A40143073
:1021300004F0ACFE404BC5F8143D04F59A40343031
:1021400004F0A4FE3D4BC5F8343D04F59A405030F0
:1021500004F09CFE3A4BC5F8503D04F59A407030AF
:1021600004F094FE374BC5F8703D04F59B400C30ED
:1021700004F08CFE344BC5F88C3D04F59B402830B0
:1021800007F0E0FE04F59B40643004F07FFE2F4B27
:10219000C5F8E43D2E4BC5F8003E4FF4C053A5F8FA
:1021A000543E2C4904F59C404CF074FAFE2385F80B
:1021B000CC3E052385F8F03E4FF0FF3B264BC5F89B
:1021C000C06E4BE080D40C08000080BF0000B44219
:1021D0000000B4C214ED0C0824ED0C08588C0E0855
:1021E000B8890E0860890E08B8870E08D4C70D0894
:1021F0004C8B002070A00C0824F80C0820FF0C0861
:1022000040020D0820F60C0834F90C08BCF90C0843
:102210009CF80C08A4F70C0820F70C08B0FE0C087A
:10222000ACFA0C083CFA0C085CED0C082CFB0C0812
:1022300038FE0C082CFC0C081CFD0C089CFC0C083F
:10224000B4FD0C08ACFB0C08B0F50C08BC010D0883
:102250004CED0C0818AD0E08391C0108C5F8C46E09
:10226000C5F8F8BE119305F57165894B85ED008AB7
:1022700004F59E4004F5A04522464FF400710093FA
:102280001430844B10941AF009F904F5A943C5F8E9
:1022900070B4C3ED038A03230026C5F8FC3405F5AA
:1022A000A363C5F8C864C5F8CC64C5F8D064C5F8A4
:1022B000D464C5F8D864C5F8DC6483ED008A764B35
:1022C000C5F84035754BC5F8483504F5AA40744B40
:1022D000C5F85035C5F83C45C5F84445C5F84C45EA
:1022E00064301CF0C1FE04F5AB401CF0BDFE04F5EB
:1022F000AB4004F5AA4A1C301CF0B6FE0AF1200AD5
:10230000684BC5F8B035A5F8B4B50AF198001CF0D3
:10231000ABFE654B6549C5F814B65046C3F800A03E
:102320004CF0B8F94FF6FF73A5F85C3504F5AC40F6
:102330005F4B6049A5F878B5183018604CF0AAF9E1
:102340005D4BD7F8A4251294CDE913345B4BCDE94E
:1023500015345B4BCDE917345A4BCDE919345A4B40
:10236000CDE91B34594B1D931EA911E903000CAB99
:1023700083E80300DDE91A010AAB83E80300DDE925
:10238000180108AB83E80300DDE9160106AB83E81A
:102390000300DDE9140104AB83E80300DDE9120169
:1023A00002AB83E803005146CDE900290E9B0F984C
:1023B000424688F023FA08F51B7304F5AD40C5F8D2
:1023C000F43678301CF050FE04F5AE4008301CF0B6
:1023D0004BFE04F5AE40183004F5AF471CF044FE48
:1023E00008371022314605F5E560B2F0B5FD3846F4
:1023F0007AF0FCF8364B3749C5F8883738464CF048
:1024000049F9354A3549116004F5AF434033142783
:10241000B0B207FB00120136127C002AF8D1304A14
:102420001080304A166816B12F488BF0DDFE04F597
:10243000AF40443013607AF0C3F82C4BC5F8C43772
:1024400004F5AF404146503009F08AF8284BC5F8F2
:10245000C83A642385F8CC3A264BC5F8003B04F50E
:10246000B540254BC5F8043B244948304CF012F9DF
:10247000234BC5F8C83A20460123C5F8286B85F8D8
:10248000306B85F8B0341FB0BDEC028BBDE8F08F27
:10249000509D0C08391C01083D1C0108411C010815
:1024A000451C01080000FFFF28870020D47D0D088F
:1024B000D4900020F4D50D08491C01084D1C0108DA
:1024C000511C0108551C0108591C01085D1C01081C
:1024D00034970C080C970C08F087002088E20C0851
:1024E000EE870020AC870020F0EC0C0874970C08F5
:1024F00034ED0C082C1E0D08841E0D08D0CE0D08DE
:1025000004200D0810B58BF0CBFA064C064B186072
:102510002046FFF789FC2046044A0549BDE81040E3
:10252000AFF0D8BF702B00206C2B0020C4E9002036
:10253000611C01080069C0F3401070470F299DBF5E
:10254000302303FB0100503000207047014B93F90A
:10255000C9017047704B0020014BD3F8D40B704772
:10256000704B002008B503689B68984730B9044B4E
:1025700093F8DA0EB0FA80F0400908BD0020FCE7BD
:10258000706B002008B504480EF062FD10B9034BD3
:1025900093F8D40E08BD00BF702B0020706B002094
:1025A000022A10B50C4605D1BDE810400948352275
:1025B00010F0ACBC084BD3F8C00E03685B689847BA
:1025C000A04205D15FF04EFEBDE810405FF0D4BDE3
:1025D00010BD00BF702B0020706B0020012910B5CA
:1025E0000C4610D0022904D061B95EF08FFB084A76
:1025F00002E05EF08BFB074A062157F00BFD064B0D
:10260000C3F8684810BD5EF081FB044AF4E700BFE0
:1026100074EE0C084CEE0C08707B002063EE0C0886
:10262000012910B50C4614D0022907D0D1B90E4BA0
:10263000C3F8281B5EF06AFB0C4A05E00A4BC3F89E
:10264000281B5EF063FB0A4ABDE81040062157F0E4
:10265000E1BC5EF05BFB074A062157F0DBFC024B56
:10266000C3F8284B10BD00BF707B0020B3EE0C08F0
:1026700088EE0C089CEE0C08012903D0022914BF37
:1026800000210221014BC3F8741B7047704B0020DE
:10269000012902D0022900D011B9024BC3F82C1B2A
:1026A000704700BF707B00206C2910B400F3A68037
:1026B0003F290FDC162900F39980032940F39A8003
:1026C0007E4B01248C402340002B00F093805DF86A
:1026D000044B7047A1F140032C2B00F28B8001A426
:1026E00054F823F09D280108F5270108F527010873
:1026F000F5270108F5270108F5270108F527010846
:10270000F5270108CF260108F5270108F52701085C
:10271000F5270108F5270108CF260108F52701084C
:10272000F5270108F5270108F52701089328010876
:10273000F527010893280108F527010893280108C7
:102740009328010893280108CF260108F5270108DE
:1027500093280108CF260108F5270108F52701086D
:10276000CF260108CF260108F5270108CF2601084A
:10277000F5270108F5270108F5270108F5270108C5
:10278000F5270108F5270108F5270108F5270108B5
:10279000CF260108CF260108112B2BD801A454F80D
:1027A00023F000BFCF260108F5270108F52701080F
:1027B000F5270108CF260108F5270108F5270108AC
:1027C000F5270108F5270108F5270108F527010875
:1027D000F5270108CF260108CF260108F5270108B3
:1027E000F5270108CF260108CF260108A1F127030C
:1027F000112BD1D95DF8044B60F046BBA0291FDC3A
:102800009529F7DDA1F196030A2BF3D801A454F81A
:1028100023F000BFCF260108F5270108F52701089E
:10282000F5270108CF260108CF260108F527010862
:10283000CF260108F5270108F5270108932801088C
:10284000B52921DCA929D5DDA1F1AA030B2BD1D80B
:1028500001A454F823F000BFCF260108F527010892
:10286000F5270108CF260108F5270108F5270108FB
:10287000CF260108F5270108F5270108F5270108EB
:10288000F5270108CF260108A1F1D003022BB1D80A
:102890001DE75DF8044B002360F0C8BA084B012225
:1028A00083F8242BA3F54053D3F8D00B00283FF432
:1028B0000EAF5DF8044B64215FF01ABD10004100BB
:1028C000707B00206C2938B50346154600F3A280C2
:1028D0003F2912DC38290ADC26296FDC102900F098
:1028E0000581162900F08A81042900F016812A4604
:1028F0001846BDE8384060F08FB8A1F140022C2A9C
:10290000F5D801A050F822F0C52A0108EF280108E7
:10291000EF280108EF280108EF280108EF28010837
:10292000EF280108EF280108F52A0108EF2801081F
:10293000EF280108EF280108EF2801081F2B0108E4
:10294000EF280108EF280108EF280108EF28010807
:10295000672B0108EF280108BB2B0108EF280108AD
:10296000712B0108B12B01085D2B0108F32B010825
:10297000EF280108DB2B0108252B0108EF280108AF
:10298000EF280108B32A01080B2C0108EF280108E1
:10299000032B0108EF280108EF280108EF280108A0
:1029A000EF280108EF280108EF280108EF280108A7
:1029B000EF280108932C01082B2B0108A1F1270215
:1029C000112A94D801A050F822F000BFB32A0108C0
:1029D000EF280108EF280108EF280108B72A0108AD
:1029E000EF280108EF280108EF280108EF28010867
:1029F000EF280108EF280108EF280108152B01082E
:102A0000FD2A0108EF280108EF2801080F2B010813
:102A1000092B0108A02921DC95297FF768AFA1F1D6
:102A200096020A2A3FF663AF01A050F822F000BFD9
:102A3000152C0108EF280108EF280108EF280108EC
:102A40001B2C01086D2C0108EF2801087B2C0108C4
:102A5000EF280108EF2801083B2C0108B52923DCE9
:102A6000A9297FF744AFA1F1AA020B2A3FF63FAF95
:102A700001A050F822F000BF312B0108EF28010817
:102A8000EF2801085B2C0108EF280108EF28010856
:102A9000372B0108EF280108EF280108EF2801086B
:102AA000EF280108B32C0108A1F1D002022A3FF659
:102AB0001EAF01248FE0A91E864B4D424D4183F885
:102AC000CD5EF6E7AA1E5542834C554184F8235B40
:102AD0005EF01CF9814A94F8231B814B002908BF42
:102AE0001346804A062157F095FAE2E70A21FFF7DC
:102AF00057FDDEE72A4601211846F8E72A46042159
:102B0000FAE72A460321F7E72A460C21F4E72A468A
:102B10000F21F1E72A460021EEE70B21E7E72A46DD
:102B20000D21E9E72A460521E6E72A461521E3E7D4
:102B30002A461121E0E7AB1E5A425A41664B93F8F0
:102B4000C8189142B5D083F8C8285EF0DFF8664A0D
:102B5000664B022D08BF1346654AC3E7294618464F
:102B6000FFF78AFDA5E729461846FFF737FDA0E7DE
:102B7000594CD5B1022D0DD1012384F8203BA4F589
:102B80008053D3F8C00E03685B6A984710B1594868
:102B900000F070FB5EF0BAF8534A94F8201B534BD8
:102BA000002908BF1346544A9CE784F8205BE6E7F7
:102BB00029461846FFF734FD7BE7012445B1022D75
:102BC00009D1454BC3F82048002283F8102902E0C0
:102BD000414BC3F82058204638BD01242DB1022DA9
:102BE000F9D1464B83F8DC4FF5E7444B83F8DC5FC3
:102BF000F1E729461846FFF74BFD5AE7022A7FF412
:102C000058AF3C4808F0E4FA53E75FF02BFB5FF065
:102C1000B3FA4EE72A4607216EE7184629465FF0C9
:102C20002BFE374879F022FD044600283FF441AFDF
:102C3000294B0122C3F82028C6E7274BD3F8E038F8
:102C4000002B3FF436AF012425B1022DC3D183F808
:102C50002C40C0E783F82C50BDE7022D7FF429AF4C
:102C60009FED280A2348FBF71BFC22E7022D7FF487
:102C700020AF20480EF0FAF81BE701242DB1022DF9
:102C8000A9D1154B83F8224BA5E7134B83F8225BA0
:102C9000A1E7022D12D10F4DD5F8C00E0368DB6BF2
:102CA0009847044678B10121A5F5804002F0CCFE9A
:102CB00091E71548294689F01FFEFAE60D480021E4
:102CC00002F0C2FEF5E65EF021F8104A042157F04A
:102CD000A1F9EEE6706B0020707B0020C8EE0C08B6
:102CE00013D70C08D0EE0C081CC10C088CFF0C0884
:102CF000E0EE0C08702B0020ECEE0C08703B00207E
:102D0000F88200200000000070790020FFEE0C081F
:102D100010B599B104681168416004B90160126886
:102D200001681B68521A9A4202D80021084610BD59
:102D3000017A012381F001010372F7E7037A3BB1C5
:102D400044682CB11368029A12681B1B9342ECD999
:102D50000023C0E90033EFE70023C0E90533C0E9F1
:102D600008338385037780F828307047F0B52DED60
:102D7000028B044687B0A148B0EE408A0F4679F036
:102D80007FFC40B1236933B1206B00F50E7010F069
:102D9000B5FB054638B12046FFF7DEFF002007B03F
:102DA000BDEC028BF0BD236B93F93C22002A1EDDA3
:102DB00093F8A032DBB1924ED6F82C2B002AEAD140
:102DC0002369D4ED007A991E4842F5EEC07A484155
:102DD000F1EE10FA84F82C0027D8C4E90822C4E9DF
:102DE000052284F82D2084F828202277D7E7854E05
:102DF000D6F8C00E03689B6B984728B106F580563D
:102E000096F8F834002BD6D07F4800210EF0B2FBA4
:102E1000DFED7E7AB4EEE70AF1EE10FACBDA7A480B
:102E200003F0E4FB0028C6D1B5E76FB1F4EEC87A31
:102E3000F1EE10FA3CDD236BD3F8C432DB0403D58A
:102E4000734815F011F9074684F82D708BF0FEF9E0
:102E5000D4ED027A9FED6F7A039067EE877AFCEEED
:102E6000E77A17EE903A5B000593B4F90630CDEDA2
:102E7000047A002B1EDC0023C4E9083384F82830D0
:102E800094F90430002B41DC0023C4E90533237797
:102E900094F82C00002882D194F82D0000287FF4AB
:102EA0007EAF94F8280000287FF479AF207F76E782
:102EB0001746C9E70421544800F0AEFCB4F90630C7
:102EC00007EE903AF8EEE77A05ABF4EEC07AF1EE51
:102ED00010FA0093CCBF0121002104AB03AA04F136
:102EE0002000B0EE408AFFF713FF0028C8D05DF045
:102EF0000DFF074618EE100AF9F7FEFA464ACDE92B
:102F000000010421384657F085F8B9E7434F9FED9B
:102F1000447AD7F86024DFED436A07F58051D1ED9C
:102F2000597A82EAE270B0EE476AA0EBE270A7EE4F
:102F3000A66A07EE900AF8EEE77AF4EEC67AF1EEAA
:102F400010FA56D8D7F8640491ED5A6A07EE900A41
:102F5000A6EE267AF8EEE77AF4EEC77AF1EE10FAEA
:102F600047D591ED5B6A9FED307AA6EE267AF4EEB6
:102F7000C77AF1EE10FACCBF4FF0010C4FF0000C05
:102F8000642113FB01F1D6F81035D21A002AB8BF1C
:102F900052428A4230DAD7F86424D6F81435D31A6C
:102FA000002BB8BF5B428B42ACBF0023012304F16E
:102FB0001400BCF1000F01D183F0010505AB0093B3
:102FC00003AA04AB2946FFF7A3FE00283FF460AF35
:102FD0005DF09CFED7F86014D7F86424642392FB5C
:102FE000F3F291FBF3F300920421104A57F012F828
:102FF0004EE74FF0000CC3E70023D8E7F88200202B
:10300000707B0020706B0020702B002000000034CB
:10301000D83D002000007A44F8F00C08703B0020F6
:103020000000FA430000C8420000FAC309F10C088E
:1030300073B58289036BD20704466CD493F93C22A2
:10304000002A03DD93F8A022002A64D1524DD5F85E
:10305000C01E05F5576291425DD0A5F54055B3F904
:103060000860D5F8603407EE903AD5F86434B8EECD
:10307000E77A07EE903AF8EEE77A6846CDED017A06
:103080008DED007A2FF068FF730007EE903AF8EEAE
:10309000E77AB0EEC00AF4EEC07AF1EE10FA42D44C
:1030A000236B93F8F1223AB307EE906AF8EEE77AD1
:1030B000F4EEC07AF1EE10FA1EDB002183F8F11273
:1030C000236B586B81F0ECFF236B9FED347ADA6B46
:1030D000D2ED067A05F26C6267EE877A92ED007A9D
:1030E000F4EEC77AF1EE10FA06D5986B84F038FA50
:1030F000236B986B83F0CEFFA389226B13F002033E
:1031000002D192F8F11299B9002382F8F232236BBE
:1031100093F8F10205E0002083F8F102236B83F8B5
:10312000F20202B070BD236B012283F8F122B7E7EF
:1031300005F28451D1ED007A9FED197AF0EEE76A3D
:10314000F4EEC76AF1EE10FADFDD05F27C51D1ED45
:10315000006A9FED146AB0EEE67AB4EEC67AF1EE3C
:1031600010FAD2DD104991ED007AB0EEC77AB4EED4
:10317000C67AF1EE10FAC8DD67EEA67AF5EEC07AEF
:10318000F1EE10FAC1D5D5F8643408498B42ACBFD2
:1031900000230123B9E700BF706B00200AD7233C4E
:1031A000C2B8323E920A063FF04000206CEEFFFFAC
:1031B00008B5036B93F8F2223AB1DA6A92F8A020CC
:1031C000022A03D0002283F8F22208BD0B4B9FEDA8
:1031D0000C0AD3ED007AF5EEC07ADFED0A7AF1EE53
:1031E00010FAD8BFB0EE670A152060F04DFBBDE8BD
:1031F00008409FED050A132060F046BBF440002014
:1032000000A08CC500A08C450000000000F58040A7
:10321000D0F8C00E03681B6C1847000000F500537F
:1032200093ED7A7A00F5A040B5EEC07AF1EE10FA8F
:103230005DBFD0F8F436DFED086AD3ED017AD0F83F
:103240000C075FBFF8EEE77AE7EE267AFDEEE77A45
:1032500017EE900A704700BF0000C84200F500500A
:1032600090F8200228B141F00101084214BF01206A
:103270000020704700F5A040D0F80C37C0F8283780
:103280000023C0F82C37704700F5A0404A68C0F80A
:1032900028270B78DB0741BFD0F8F4365B689B1812
:1032A000C0F828377047000000F5A040D0F8283754
:1032B0001944C0F82817704710B54B68516800F5DD
:1032C000A0448B42D8BF0A46D4F82807CCBF1A4680
:1032D00019462CF005FFC4F8280710BD10B50446A8
:1032E000414868F099FE10F0080217BF3F4BDFED30
:1032F000407A93ED157AD3ED177A1FBF77EE877A70
:103300009FED3C7A012267EE877A10F0010317BF28
:10331000364B9FED377AD3ED176A93ED147A1CBFC5
:1033200037EE667ADFED336A04F5005118BF27EEF9
:10333000267AD1ED7C6AF5EEC06A18BF0123F1EE62
:1033400010FA4BDD294A9FED2B6AD2ED7C6A66EEBE
:10335000866AF4EE676AF1EE10FA58BFF0EE667A0C
:10336000F3B11A4604F5A043D3F8F416D1ED016A7F
:10337000D3F82817F8EEE66A76EE876A07EE101A99
:10338000B8EEC77AF4EEC76AF1EE10FAD8BFB0EE25
:10339000667ABDEEC77A17EE101AC3F828170AB37B
:1033A00004F5A044D4F8F43693ED017AD4F8283724
:1033B000B8EEC77A77EE277A07EE103AB8EEC77AFA
:1033C000F4EEC77AF1EE10FA58BFB0EE677ABDEEB0
:1033D000C77A17EE103AC4F8283703E0002ABFD1A5
:1033E000002BBFD110BD00BFB84B0020704B002098
:1033F000000000000000C84200F5A0400023C0F813
:103400002C37704713B500230446104601AA0193D8
:103410001BF0E6FE034648B1DDED017A9FED177A19
:1034200067EE877AFDEEE77A17EE903A04F5A04151
:10343000D1F8FC24C1F82C37042A1DD004F500541F
:10344000B4F91A22002A14DD83EAE370A0EBE370DA
:1034500007EE900A9FED0A7AF8EEE77A67EE877A30
:1034600007EE102AB8EEC77AF4EEC77AF1EE10FA3A
:1034700002D50023C1F82C3702B010BD0000C842AD
:103480000AD7233C0B78D1ED017A00F5A04013F068
:10349000010F1CBFD0F8F43693ED017AF8EEE77A0D
:1034A00018BFB8EEC77A00F20C7318BF77EE877AB0
:1034B00093ED007AB8EEC77AB4EEE77AF1EE10FA3F
:1034C000CCBF0120002070477047000000F500537A
:1034D00000F58042B3F9D231D2F8C02E00EE103A96
:1034E00000F5984320339A42B8EEC00A0ED100F599
:1034F000A040D0F8FC34042B02D090F8B1342BB1AA
:1035000000F5C760D0ED007A30EE270A7047000062
:10351000014608B501F5A041FFF7D8FF01F20C7391
:10352000D3ED007A9FED057AF8EEE77AE0EE477A80
:10353000FDEEE77A17EE900A08BD00BF0000C84212
:1035400010B5044604F5A044FFF7E2FFD4F828378D
:10355000181A10BD70B504462DED028B04F5A04578
:10356000FFF792FEDFED340A40F24310B7EE001A87
:103570000E462CF015FDD5F82C27534207EE903A55
:10358000F8EEE77AD5F8283767EE807AB0EE408A11
:10359000FDEEE77A17EE901A1944C5F8281704F5DE
:1035A0000053D3ED876AF5EEC06AF1EE10FA3FDD05
:1035B000002A3DDD2046FFF7C3FF9FED207A07EE8E
:1035C000900A66EE876AF8EEE77AF4EEE67AF1EEB4
:1035D00010FA2DD531462046FFF756FE04F5AE41D0
:1035E000324608312046FFF70DFFD5F82C2753420D
:1035F00007EE903AF8EEE77AD5F8283767EE887A42
:10360000B5EEC08AFDEEE77AF1EE10FA17EE901AE9
:103610001944C5F828170BDD07EE902AF8EEE77A73
:1036200087EE887ABDEEC77A17EE103AC5F82C37C8
:10363000BDEC028B70BD00BF000000000000C8C2DE
:10364000014608B5FFF742FF01F5AE40D0ED0E7A16
:1036500037EEC00ADFED047A20EE270AFDEEC07ACD
:1036600017EE900A08BD00BF0000C8422DE9F041E6
:1036700000F5AE4800F5AE4508F1080818350446D7
:10368000294640461CF020F804F5A04704F5AD4655
:1036900007F5936378362A46314683ED000A4046A3
:1036A0001BF048FF07F29C43DFED220A83ED000A7E
:1036B000B7EE001A76202CF073FC04F5315383ED3D
:1036C0007F0A2046FAF77CFE04F58043D3F8C00E4B
:1036D00003685B6898470B280BD006D80A280FD0E0
:1036E0000023C7F82C37BDE8F0810E38C0B201289E
:1036F000F6D829462046FFF7C5FE0028F0D011E095
:1037000029462046FFF7BEFE30B90B484FF48041F2
:10371000FBF78AF90028E3D12046FFF791FFB0F5C7
:10372000FA6FE6DD2A4631462046BDE8F041FFF754
:1037300069BE00BF00000000702B002010B500F52E
:10374000A04300F58054D3F81C2793F818379FED59
:10375000146A13F0010F07EE902A08BFD4F8D8348A
:10376000F8EEE76A08BF07EE903A66EE866A04BF95
:10377000F8EEE77AE7EEC66AFFF7CAFE04F59B6348
:1037800093ED000A07EE900AB8EEC00AF8EEE77A69
:1037900026EE400AA7EE860A30EE660A10BD00BF8C
:1037A0000AD7233C38B50446FFF758FD78B904F52D
:1037B000AF45503528460AF03FFA28B3284609F0AD
:1037C000DDFD08BB2046BDE83840FFF7B7BF04F574
:1037D000005595F8F03BDB0704D505F60C4595ED53
:1037E000000A38BD04F5AF4050300AF04BFA00280B
:1037F000DDD095F8BA1B04F551604CF057FA022859
:10380000D5D19FED040AECE704F5AE4494ED0E0A21
:10381000E7E700BF000000000022FFF7C3BF000081
:1038200010B504468AF012FD04F50053D3F8042CB9
:10383000801A41F2883290420FD802212046FFF7C9
:103840000DFD50B104F5A044D4F8FC24042A04D1A1
:1038500003F6F83393ED000A10BD9FED010AFBE774
:103860000000000008B52DED028B00F5A0430146D5
:10387000D3F8F426D3F828375268DFED0D8A9B1A67
:1038800008EE103AFFF722FEB8EEC88A0846A0EE0E
:10389000288AFFF7C5FFBDEEC88AB8EEC88AA0EE39
:1038A000288AFDEEC87ABDEC028B17EE900A08BD9F
:1038B0000000C842F0B52DED048B00F5005489B02E
:1038C00000F5516694F8BA1B0391054630464CF05A
:1038D000EDF90399074630464CF0FAF9042F0399A5
:1038E000B0EE408A21D1002305A88DED050A06938C
:1038F00007932FF0B1FD05F5AC5005A908302DF068
:1039000079FCDFED997A8DED050AB4EEE71AF1EE58
:1039100010FACDED060A8DED071A06DB05F580538A
:1039200093F8E47417F001070CD194F8F03B0022EF
:1039300062F3000384F8082C84F8F03B09B0BDEC76
:10394000048BF0BD94F8F03B9A075FBF43F002038D
:1039500084F8F03B04F6F43383ED008A04F60C435C
:1039600083ED001A94F8083C092B79D804F54163DB
:10397000D3ED000A9FED7D9AB0EE480A2CF0FEF9D7
:1039800000BB04F6F43394F8BA1BD3ED008A30463A
:103990004CF0BCF907EE900A9FED757AF8EEE77AE5
:1039A00078EEC88A67EE877AF0EEE88A67EE897A61
:1039B000F4EEE78AF1EE10FAC2BF94F8083C013346
:1039C00084F8083C04F5416394F8BA1BD3ED008AEF
:1039D00030464CF09BF907EE900AF8EEE77A9FED3F
:1039E000657A67EE897A78EEC88A67EE877AF0EEB4
:1039F000E88AF4EEE78AF1EE10FA02DD002384F89B
:103A0000083C04F5416383ED008A94F8F03BDA0743
:103A100094D52846FFF792FE04F60C4696ED008AF0
:103A200030EE488A8AF012FCD4F8042C41F2883136
:103A3000821A8A42034604F6F83204F6FC315AD957
:103A400082ED008A284681ED008A0221FFF706FCFC
:103A500018B105F5AC456A6C2A64C4F8043C6DE7FE
:103A600094F8F03B43F0010384F8F03B05F5A043E4
:103A7000D3F8FC6405F58043301FD3F8C02E05F55C
:103A80009A43464203F1340346419A4212D005F567
:103A90009A4350339A420DD005F5984320339A4209
:103AA00009D1354B05F5AF40B3F85E15503009F03C
:103AB00081FC00B13E4694F8F03B5907A1D4002E9A
:103AC0009FD002212846FFF7C9FB002899D043F078
:103AD000040384F8F03B04F60C4305F54E561868D1
:103AE000F8F70AFD0836CDE90001244A06213046E0
:103AF00056F090FA85E79FED1F0A92ED007ADFED10
:103B0000207A28EE008AA7EE278A82ED008AC4F880
:103B1000040CD1ED007A38EE678AF3EE0E7AB0EE3F
:103B2000C88AB4EEE78AF1EE10FA7FF707AF94F88F
:103B3000F03B5B070CD53068F8F7DEFC05F54E541A
:103B40000834CDE900010F4A0621204656F062FAFA
:103B500005F52F5024220021303009B0BDEC048B34
:103B6000BDE8F040B1F0F8B9000000340AD7233CBA
:103B7000CDCC4C3DCDCC4C3E707B002020F10C08D0
:103B8000CDCC4C3F3DF10C0838B52DED028B0D46E8
:103B90000446FFF7D3FD002320462B70B0EE408A89
:103BA000FFF73EFE0221204638EE400AFFF756FBA3
:103BB00028B104F5005494F8F00B00F00100BDECBE
:103BC000028B287038BD000070B50B7803F0050338
:103BD000042B05460C46164615D105F5A04552F0B6
:103BE0001BFDB2B24FF4801152F0CEFCD5F8F42692
:103BF000636852689B1A13F5FA7FC8BF6360237825
:103C000043F00103237070BDF8B500F5805300F553
:103C1000A047D3F8D864D7F8C054B542044619D0A9
:103C20000E4A1268D26A92F89C209AB100F5AE4111
:103C3000751B25221831FFF7C7FF07EE905AB8EE23
:103C4000E70ADFED077A04F5315020EE270A383015
:103C50007DF0E8FBC7F8C064F8BD00BF6C2B002006
:103C60000AD7233CF8B500F5A044054694F8B3C440
:103C70000F4604F5DF66BCF1000F53D004F5E36393
:103C80000FCB86E80F00012384F8B43497E80F00C7
:103C900004F5E36686E80F00D4F8203705F5AE4654
:103CA000183693B9D4F824377BB9D4F81037D4F840
:103CB0001C27C4F82037D4F81437C4F8243722B9A5
:103CC000D4F80C1730461BF0D5F931462822284687
:103CD000FFF77AFF94F8181711F0040102D130466B
:103CE0001BF05AFA05F5AD4105F5AE403246783184
:103CF00008301BF055FC38B104F5DF6604F5E164CB
:103D000094E80F0086E80F00284606F0D3FC28460A
:103D1000FFF7ACFC284607F0C7F82846BDE8F84096
:103D2000FFF774BA04F5E1630FCB86E80F000123B7
:103D300084F8B33484F8B4C4A8E70000F8B500F5FB
:103D400000530446B3F97A31002B0E4634DB0B786E
:103D500013F0020F14BF4FF0FF33012304F5A04509
:103D600005F5DF6785F8D03605F5E1630FCB87E809
:103D70000F0096E80F0005F5E36787E80F0004F5EC
:103D8000AE41572218312046FFF71EFF2046FFF7AD
:103D900071FA20460026FFF769FC204607F084F8F8
:103DA00085F8B464C5F8D46685F8B964204606F091
:103DB00081FC85F81269F8BD4FF0FF33CEE70000B3
:103DC0002DE9F043364B1B6885B00546D86AF9F7F4
:103DD000A3FB002861D105F5005393F9883B5A1CD9
:103DE00054D0002B05F5866711DD95F84124242178
:103DF00007EE903A01FB027292ED0B7AF8EEE77A49
:103E0000B0EEC77AB4EEE77AF1EE10FA3EDC05F5D3
:103E1000805305F5935693F8E43413F0010406F14A
:103E2000080629D0C3F340089B0732D495F8E41361
:103E300095F828444FF0B00909FB015191F8C131C0
:103E40004CBB022B18D968461BF00EF96946304668
:103E500015F0B6F8044678B195F8E43309FB03533E
:103E60004246D3F8D01168461BF004F915F07EFBEA
:103E7000694614F093FF0446384617F027FE304693
:103E800014F0AAFE2846FAF7A1FD204605B0BDE8C9
:103E9000F0830024F0E74446EEE70020F6E700BF99
:103EA0006C2B002038B50C4B1B680546D86A0C46B5
:103EB000F9F732FB10B10024204638BD15F056FB4F
:103EC000214614F06BFF04460028F4D005F5AA4003
:103ED000203030F0DBF8EFE76C2B0020F0B500F578
:103EE000A045002385F8B33485F8B43405F5E163C3
:103EF000044600EE101A0FCB87B005F5DF6686E8A2
:103F00000F0002AE04F5AE42B8EEC00A30461749C3
:103F100008324BF03FFC96E80F0005F5E36787E8B1
:103F20000F0004F5AE4140F25712183120460191BE
:103F3000FFF74AFE01992046FFF7C6FA019920468D
:103F4000FFF7A2F904F500532046B3F97A31002BAC
:103F5000B4BF4FF0FF33012385F8D036FFF786FB5F
:103F6000204607B0BDE8F04006F09EBF98610020F3
:103F700010B5034904464BF00DFC204610BD00BFB0
:103F800098610020F8B500F5A04404F5E16305460A
:103F90000E460FCB04F5DF6787E80F0006F1080136
:103FA0002846FFF75FFEB388D4F81C2703EB830392
:103FB00003EB83039B001BB2002BD8BF4FF4C873E5
:103FC000A4F8AE34D4F8F4365968521AC4F88024F0
:103FD0009A680A32C4F82027DB680A33C4F8243709
:103FE0000023C4F8943484F8B03484F8C434C4F89A
:103FF000843404F58F6300221A604FF0FF33C4F855
:10400000703495F8412405F58663242101FB0233C1
:1040100004F59564DB6A2360F8BD000070B50E46B8
:1040200008310546FFF71EFEB38805F5A04443B3EB
:10403000642213FB02F3C4F88034B4F9AE34002BCD
:10404000D8BF4FF47A7305F52F50D8BFA4F8AE341B
:10405000242200213030B0F07FFF04F5E76305F53E
:10406000AC4093ED000A3146383086F0BDFCD4F800
:10407000FC34072B0CD128460421BDE87040FAF728
:104080006DB9D4F88034002BD7DC40F6B833D2E7D2
:1040900070BD000030B5083104460FC985B06D46CB
:1040A00085E80F0004F5AE41083128461BF014F9ED
:1040B00020462946FFF7D6FD04F580440123C4F8C5
:1040C000E83E05B030BD00000B7A00F5A04013F0CB
:1040D000020F14BF4FF0FF33012380F8D036704732
:1040E0007FB501F1080305460E460FCB6C4684E808
:1040F0000F0005F5AE41083120461BF0EDF82146D2
:104100002846FFF7AFFD31462846FFF7DDFF04B034
:1041100070BD00007FB501F1080304460E460FCBC9
:104120006D4685E80F0004F5AE41083128461BF0C6
:10413000D3F829462046FFF795FD20463146FFF784
:10414000C3FF337907EE903A337E9B0748BF9FED5C
:104150000C7AF8EE677A04F5A04448BF67EE877AD8
:104160009FED087A67EE877AFCEEE77A17EE903AD1
:10417000C4F8C8360123C4F8E83604B070BD00BFE7
:104180000000803B00A00C477FB501F10803044606
:104190000E460FCB6D4685E80F0004F5AE410831A1
:1041A00028461BF099F829462046FFF75BFD20467C
:1041B0003146FFF789FFB38804F5A0444FF47A72C3
:1041C0005343C4F8E0360123C4F8E83604B070BDA8
:1041D0002DE9F34100F5AE450446183500F5AD4034
:1041E0000E46783029461BF037F804F5A047C0B9D1
:1041F0004FF0FF33C7F8703406F1080840461AF054
:1042000063FF032802463AD1F16828461AF032FFCC
:10421000B388C7F8E836204602B0BDE8F041FFF7A2
:10422000EBB824F069FCF9F7F1FD012812D94FF041
:10423000FF33C7F8703424F05FFC90F8C432DFED30
:10424000150AB02202FB030090ED300A28461BF04D
:10425000E1FAD1E704F58058D8F868042BF074FE31
:1042600008F58D63C7F87004D3ED007A9FED0A0A54
:10427000DFED080AF8EEE77A27EE800AE6E701AA02
:10428000002140461AF02CFF0028C1D001990022DD
:10429000BBE700BF00007A440AD7233C7FB501F199
:1042A000080304460E460FCB6D4685E80F0004F563
:1042B000AE41083128461BF00FF829462046FFF78B
:1042C000D1FC20463146FFF7FFFE04F5A044002351
:1042D000C4F8E83604B070BD37B504460D4689F021
:1042E000B5FF2062D5ED027AF5EEC07AF1EE10FA54
:1042F00015DD9FED127A67EE877AFCEEE77AC4ED62
:10430000077A5CF003FDE2694FF47A73B2FBF3F3D2
:104310000B4A062103B0BDE8304055F07BBE67F084
:10432000C9FC0023009395F90D2095F90E3095F9FD
:104330000C1067F05BFCE061E3E700BF00007A442B
:1043400060F10C082DE9F0432DED028B85B0044699
:1043500015F00CF914F0F2F904F5805304F5A045BA
:1043600093F860370BB9002877D0D5F87034013353
:1043700073D1D5F89434002B4BD089F067FFD5F872
:104380009434C01AB0F5FA6F67D394F8E423DFEDE4
:104390005F7A9FED5F8A4FF0B00808FB024292ED12
:1043A000780A20EE270A2BF0E7FD05F58F69D9ED95
:1043B000007A30EE670A2BF0DFFDDFED567A20EE53
:1043C000080A04F54E5720EE270A2BF07DFDFDEE7E
:1043D000C07A083717EE906AC5F87064D9ED007A94
:1043E00067EE887A17EE900AF8F786F8CDE90201B1
:1043F00094F8E43308FB0343D3F8DC01F8F77CF8C6
:10440000454ACDE9000133460621384655F002FE03
:1044100023E004F59070F9F7F9FC02281DD994F80F
:10442000E433B02202FB034393ED777AF1EE047A92
:10443000B4EEE77AF1EE10FA0FDD384B1B68D86A5C
:104440000368DB699847012803D089F0FFFEC5F8AF
:104450009404D5F89434002B8FD104F54053D5F84B
:104460007014D3F8A4054A1C036846D01B6B984708
:104470002B4810F011FD20B104F5AA40203032F095
:1044800049F82046FFF7DCF8D5F880348342064629
:1044900036DA07EE906A9FED237AF8EEE77A04F5B4
:1044A0004E5467EE877A083417EE900AF8F724F82E
:1044B0001D4ACDE900012046062155F0ABFD01243F
:1044C0004FF0FF33C5F8703485F8B04405F5E1636B
:1044D0000FCB05F5DF6605F5E36786E80F0087E893
:1044E0000F00124867F062FD002385F8B3342046C0
:1044F00005B0BDEC028BBDE8F0835B6B9847B7E776
:10450000074810F0A9FC0028C3D1F1E735FA8E3C2A
:10451000E02E65420000C84270F10C086C2B0020B0
:10452000702B00200AD7233C94F10C08B84B0020D4
:104530002DE9F04100F5AD4700F5AE457837183567
:104540000446294638461AF087FE04F5A04604F5CD
:10455000405830B3D6F870144B1C22D0D8F8A405BC
:1045600003681B6B9847D6F8E836012B47D0D6F87E
:10457000E836022B06D12046FEF7CAFFD6F81C37D4
:10458000984243DD2046FEF7C3FFD6F81C37C01A19
:104590000028B8BF4042B0F5FA7FCCBF0020012010
:1045A00035E004F5AE40294608301BF08DF8DFED0C
:1045B000197AB4EEE70AF1EE10FA16D53846294614
:1045C0001AF052FF9FED147ADFED140AF6EE007A2E
:1045D000E0EE077A28469FED120AFDEEE77AF8EE44
:1045E000E77A27EE800A1BF015F9D8F8A4059FEDAD
:1045F0000D0A03682A469B6A39469847B3E7204666
:10460000FEF786FFD6F81C379842B0DB0120BDE8E4
:10461000F08100BF00004843A00CB3450000964362
:104620000AD7233C0000000073B5394CD1ED026A73
:10463000D4F80C379FED377A07EE903AF8EEE77A28
:104640000546D7EE876A0E46F5EEC06AF1EE10FA1F
:1046500008DD5CF05BFB304A062155F0DBFC0120F5
:1046600002B070BDD1ED037AF5EEC07A04F5926424
:10467000F1EE10FA94ED006A12DDF4EEC67AF1EE76
:1046800010FA0DD55CF042FB05462068F7F734FFC1
:10469000224ACDE900010621284655F0BBFCDEE7A1
:1046A000DFED1F7A337CB4EEE76AF1EE10FA54BF07
:1046B000B0EE677AB0EE467A0BB90020D0E7B5EEDF
:1046C000C06AF1EE10FA0CDC86EE876A03EB830316
:1046D00007EE903AF8EEE77AF4EEC67AF1EE10FAC9
:1046E000EBD595F82440002CE7D189F0AFFDAB6AFB
:1046F000C01A337C4FF47A7253439842DDD90123B8
:1047000085F8243089F0A2FDA8622046A8E700BF02
:10471000707B00200AD7233CB0F10C08C1F10C08D3
:104720000AD723BC38B5054679F0C0F977F0A8FF61
:10473000044640B989F08AFD2B6AC01AEB69984299
:1047400084BFEC610124204638BD000038B5044622
:104750000D4689F07BFD04F5A0439FED077AC3F871
:10476000EC06D5ED027A67EE877AFDEEE77A17EE72
:10477000902AC3F8E82638BD00007A4410B50446F4
:1047800089F064FD04F5A043D3F8EC26801AD3F831
:10479000E82690424FF0000084BFC3F8E8060120ED
:1047A00010BD000000F5A04303F59361D3F8E8269F
:1047B00091ED007A22EAE27207EE902AF8EEE77AAB
:1047C0000020B4EEE77AF1EE10FA44BFC3F8E80631
:1047D0000120704710B500F5005300F5A040B3F973
:1047E0007A31002BB4BF4FF0FF33012380F8D0366D
:1047F00000F5E36400F5E1600FC884E80F0010BD28
:1048000038B504462DED028BF0EE408AB0EE608A9A
:1048100009B301295ED0B5EEC08AF1EE10FA69DD68
:10482000DFED357AB4EEE78AF1EE10FA62D8FCEEED
:10483000C87A04F54E5017EE903A304A06210830F7
:1048400055F0E8FBFDEEC87A04F5005417EE903AF7
:1048500084F847313CE0F8EE000A2BF08FFA40B1C3
:1048600004F580444FF0FF33C4F8F83EBDEC028BF2
:1048700038BD04F50053B3F9502107EE902AF8EE45
:10488000E77AF4EEE87AF1EE10FAC4D8B3F95231CF
:1048900007EE903AF8EEE77AF4EEE87AF1EE10FAE5
:1048A000B9DBDFED157A68EEA77A04F58043FDEEFB
:1048B000E77A04F54E5017EE902AFCEEE87AC3F83A
:1048C000F82E062117EE903A0D4A083055F0A2FB5B
:1048D0000120CBE7FCEEC07A00F54E5017EE903A7F
:1048E000084A0621083004F5005455F093FBC4ED46
:1048F000578AEDE70020B9E70000C84207F20C082C
:10490000E0F10C08F4F10C08D1F80D3000EE903A0B
:10491000D1F80930097A00EE103AFFF771BF0000B4
:1049200070B58B88012B04460D4611D100F59076A9
:104930003046F9F76BFA02280AD994F8E413B02349
:1049400003FB01612046AC31BDE87040FFF7AABA15
:1049500014F00CFE05F10801BDE8704014F01EBA19
:10496000F0B500F5A047002489B0054687F8B944A2
:1049700008460E462FF09CF9A0B3012387F8B03407
:1049800005F54053D3F8A4050368DB6B984787F817
:10499000B744C7F8D44603A81AF066FBB7F85C150D
:1049A0004FF6FF73994208BF2146013105F5AA4031
:1049B00001AA89B2203031F02FF9F0B1BDF80630EC
:1049C000A3F115025342534187F8B13450B105F5B4
:1049D000AF40BDF80610503008F0ECFC10B10023D9
:1049E00087F8B13473885E2B4ED8522B07D8103B12
:1049F0009AB20F2A22D90024D5E00346E4E7533BBC
:104A00000B2BF8D801A252F823F000BFA14B0108EC
:104A1000AD4B0108BD4B0108F7490108F7490108F2
:104A2000F7490108F7490108F7490108F749010862
:104A3000F7490108094C0108BD4B01080F2BDAD8D2
:104A400001A252F823F000BF254B01085F4B01087B
:104A5000694B0108734B0108874B0108314B010872
:104A6000F74A0108F7490108F7490108F749010821
:104A7000F7490108F7490108F7490108F749010812
:104A8000974B01087D4B0108BD2B1AD8BB2B47D88B
:104A9000B22B00F0A7800DD8702B00F09E80722BF7
:104AA000A9D1D6ED027AFDEEE77A17EE903AC7F873
:104AB000E83635E0B32B9ED131462846FFF730FF6C
:104AC0002EE0D42B00F0938040F6B832934200F0F1
:104AD0009680D22B8FD1B388012B21D803F001030C
:104AE00087F8B23405F54E50B3884B4A062108309A
:104AF00055F090FA14E0002305F5AF4487F8E93447
:104B000050347188204607F0F9FE314628B120461E
:104B100009B0BDE8F04008F0F3B82846FFF732FAD4
:104B2000012440E006F108012846FFF79BF8F7E76B
:104B300005F5AF4450341521204608F03BFC48B140
:104B4000002387F8E9343146204609B0BDE8F0403B
:104B500007F0DABF31462846FFF760FAE0E7314652
:104B60002846FFF7BDFADBE731462846FFF7D2FAC1
:104B7000D6E731462846FFF707FBD1E731462846FE
:104B8000FFF78CFBCCE705F5984129224C312846EC
:104B90000EF0E4F8C4E731462846FFF719FBBFE7FB
:104BA000012487F8B744204609B0F0BD002305F57D
:104BB000AF4087F8E93431465030A9E705F5AF47F3
:104BC0005037384608F0DAFB3146044618B128461B
:104BD000FFF760FAE7E73846B7E731462846FFF7C0
:104BE000B5FD9DE731462846FFF78EFE98E7B18870
:104BF000003918BF0121284600F026FF90E7317ADE
:104C0000064807F073FA8BE705F5984031462030E7
:104C1000FFF762FB84E700BF18F20C084083002016
:104C200000F5804200F59843D2F8C02E20339A4216
:104C300001D1FFF795BE01207047000010B500F5C7
:104C4000804200F59843D2F8C02E20339A420446A1
:104C50000ED100F5984108224C310EF07FF804F592
:104C60004E50044ABDE810400621083055F0D2B934
:104C700010BD00BF28F20C082DE9F04F2DED048B7C
:104C800000F5A04808F5056393ED008ADFEDD77ABB
:104C9000B0EEC87AB4EEE77AF1EE10FA48BF00F54C
:104CA0000053DFEDD37A42BFB3F97A3108EE103A00
:104CB000B8EEC88A00F58045B4EEE78AF1EE10FA46
:104CC00094BF4FF0FF37012788F8D076D5F8E83E3B
:104CD0009BB004460E46F0EEC88A052B16D8DFE8D6
:104CE00013F006002C0069008800C500600100F583
:104CF00040543A46D4F8A4050368B0EE680ADB6A6B
:104D000008319847BB4806F00BF908B9002049E183
:104D1000B94CD4F8F436B4F990185B68642201FBFE
:104D20000231A4F5A040FFF7D9F8A4F5A04005F0A2
:104D3000C1FC0123C5F8E83EE8E700F540533A46D8
:104D4000D3F8A4050368B0EE680ADB6A0831984717
:104D5000D8F8CC36002BB8BF5B42012BD6DD98F8D3
:104D6000D1361BB998F8D236002BCFD004F5AE530C
:104D7000D3ED040A93ED050AF1EE600AB1EE400AA4
:104D8000ADF0F0FEDFED9D7A20EE270A05F6EC632C
:104D900083ED000A10EE100AF7F7AEFB04F54E544F
:104DA0000834CDE90001964A0621204655F032F933
:104DB0000223BFE700F5AE4901F1080A09F108092D
:104DC000494650461AF080FC30EE680AF1EE047A4B
:104DD000B0EEC00AB4EEE70AF1EE10FA00F3E78095
:104DE000D8F8CC360133022B40F2EB800323C5F810
:104DF000E83E04F5405306F10808D3F8A40503681B
:104E00003A46DB6AB0EE480A41469847DFED7D6AD4
:104E10009FED7D7A05F6EC63D3ED007A012F18BF84
:104E2000B0EE667A04F5A35377EE877A93ED050A20
:104E30009FED767AA7EEC70A2BF09EF8DFED747A25
:104E4000B0EEC00AB4EEE70AF1EE10FA7FF55EAFFD
:104E500004F54E50062108306E4A55F0DBF8042365
:104E6000C5F8E83E41462046FEF7FCFE06F108057F
:104E700095E80F000AAF0DF1380887E80F0088E8C1
:104E80000F0004F5804303F6EC6A9FED639A9AEDF8
:104E9000000ADFED620A0393384630EE090A1AF081
:104EA000B9FCDFED5E0A9AED000A9FED5D8A40468F
:104EB0001AF0B0FC04F540534246D3F8A405036849
:104EC00039469B6AB0EE480A984795E80F0004F50A
:104ED000AF490DF1480B09F150098BE80F00DAEDED
:104EE000009A484607F030FD79EE899A04F5AE48FD
:104EF000F0EE400A5846B0EE690A08F108081AF0C8
:104F000089FC5A46394640461AF04AFB834695E8E2
:104F10000F009AED000A16AF87E80F00F0EE680A5E
:104F200030EE090A38461AF075FC394640462A46E2
:104F30001AF000FB04F5935007A90830F0EE408A00
:104F40008DED078A8DED088A8DED098A14F00CF934
:104F5000002867D0294640461AF0C2FA05A907A8DA
:104F6000CDED060A8DED050A2EF00AF8DFED237A65
:104F700020EE270A2AF094FFB0EEC00ABBF1000F22
:104F80003FF4C4AEF3EE0E7AB4EEE70AF1EE10FA97
:104F900023D5039A0523C2F8E83E3146484607F078
:104FA000B3FD01201BB0BDEC048BBDE8F08F49467A
:104FB00050461AF089FBB4EEE80AF1EE10FA7FF5DC
:104FC0000FAF04F540543A46D4F8A4050368B0EE98
:104FD000680ADB6A5146984798E6F6EE007AF4EEE6
:104FE000E78AF1EE10FAD4DC90E600BF000000344E
:104FF000000000B4702B0020707B0020E02E654282
:1050000050F20C080000B4420000874335FA8E3C91
:10501000C2B8B23D72F20C080000344300007A447A
:1050200000000000BBF1000F3FF470AEB1E700BF1D
:105030002DE9F041074600F5AF408EB0503088466C
:1050400008F0DCF9044650BB09AE07F5A045304630
:105050001AF00AF8B5F85C354FF6FF72934208BFB4
:105060000023013307F5AA4007AA99B2203030F097
:10507000D3FDC0B1B8F1000F01D0C5F8CC4696E819
:105080000F0001AC84E80F00D5F82437009305F534
:10509000E36595E80E00054803F0CCF90446204688
:1050A0000EB0BDE8F0810124F9E700BFD8770020F9
:1050B00070B5064606F5A045002106F001F8D5F8C2
:1050C000D4467CB9304605F02BFF10B900242046A9
:1050D00070BDD5F8CC36012BF8DD89F0B7F8C5F8EE
:1050E000D406F4E7D5F8E81661B189F0AFF8D5F841
:1050F000D436C01AD5F8E0369842E7D90023C5F86F
:10510000E83601213046FFF793FF04460028DDD042
:1051100006F54E50044A0621083054F07BFF002368
:1051200085F8B934D3E700BF94F20C0870B50A468D
:105130008B88190A137E0546DB0748BF01EB810106
:1051400005F5A04448BF4900002605F0B9FF84F8E2
:10515000B964284605F0E4FE10B90024204670BD6D
:10516000D4F8E81651B1D4F8CC36D4F8C826934216
:10517000F3DD012BF1DDC4F8E86601212846FFF7D5
:1051800057FF04460028E8D005F54E50024A062194
:10519000083054F03FFFE1E7ACF20C0838B50546A3
:1051A00005F5A044898805F08BFFD4F8E83683BB69
:1051B000D4F8CC36002BB8BF5B42012B02DC0024B4
:1051C000204638BD94F8D12694F8D23672B9002B17
:1051D000F5D005F54E50D4F80C276423062192FB38
:1051E000F3F308300C4A54F015FF01E0002BF0D126
:1051F0000121C4F8E8162846FFF71AFF04460028E4
:10520000DDD005F54E50054A0621083054F002FF66
:10521000D6E70021EFE700BFC4F20C08E2F20C0869
:1052200010B504460B4808F0D3FE48B10A4BDFED39
:105230000B7AD3F80C3893ED090A20EE270A10BD3B
:1052400004F50054B4F9A83100EE103AB8EEC00AE3
:10525000F5E700BF40830020707B00200AD7233C85
:1052600038B52DED028B00F5005300F5A045B3F9DC
:10527000AC110029ACBF01234FF0FF330029B8BFA8
:10528000494285F8D036044689B205F019FF05F584
:105290009365204695ED008AFFF7C2FFB5EEC00A80
:1052A000F1EE10FAD8BF9FED0E0ABCEEC00AB8EEC0
:1052B000400AB4EEC08AF1EE10FA0AD804F54E5056
:1052C0000830084A062154F0A5FE0120BDEC028BEF
:1052D00038BD204605F024FE0028EFD1F6E700BFD8
:1052E00000000000FCF20C082DE9F04700F5A04793
:1052F0002DED028B4FF0FF33C7F8703407F5E363F1
:105300008C4605460FCBBCF804609CF8049088B02E
:1053100004AC360A84E80F0020D005F5AD4808F14A
:105320007808214640461AF0CFF921464046B0EEB3
:10533000408A1AF099F8DFED587AB4EEE78AF1EE78
:1053400010FA0BDBF3B200EE903ADFED547AF8EE90
:10535000600A20EE270A20461AF05CFA05F5405A4A
:1053600097F8B424DAF8A4059FED4D0A036805F513
:10537000AE489B6A08F1080832B305F5AD412246F4
:105380007831984705F50053B3F9AA31002B1EDD9B
:1053900007EE903A07F59362F8EEE77A92ED007A1D
:1053A000B4EEE77AF1EE10FA11DD05F5AD412246D3
:1053B000783140461AF0F4F8F8B90026304608B0C3
:1053C000BDEC028BBDE8F08722464146D9E7B9F132
:1053D000000F1DD1002E3DD1DAF8A46533682846B0
:1053E000D3F82090FFF71CFF07F28C43D3ED000A9F
:1053F0003046C847B0EE408A0EE0002EDDD107F5FA
:10540000DF6407F5E16797E80F0084E80F00D5E750
:1054100007EE909AB8EE678A214640461AF054F992
:10542000B4EEC08AF1EE10FA17DBB7F85C350393DF
:10543000214640461AF048F9BCEEC00A05F54E5028
:10544000039B184A8DED000A0621083054F0E2FD56
:105450000126B3E79FED128ADEE705F5AD4122464E
:10546000783140461AF09CF806460028A5D0B7F8D7
:105470005C350393214640461AF026F9BCEEC00A7B
:1054800005F54E50039B084A8DED000A06210830B1
:1054900054F0C0FD92E700BF00000034E02E6542EA
:1054A0000000000014F30C0832F30C082DE9F0475B
:1054B0004B881F2B8AB004460D466BD80F2B41D862
:1054C00004F54E50BF4A0421083054F0A3FD9BE080
:1054D000A3F1BC02182AF3D801A151F822F000BFB1
:1054E0000956010809560108C1540108C1540108B0
:1054F000C1540108C1540108C154010809560108EA
:10550000C154010809560108C1540108C1540108D9
:10551000C154010809560108C1540108C1540108C9
:10552000C154010809560108095601080956010825
:10553000C1540108C154010809560108C1540108A9
:1055400009560108A3F110020F2AB9D801A151F898
:1055500022F000BF455601082B57010835570108B6
:105560004157010857570108515601081B560108B9
:10557000C1540108C1540108C1540108C1540108B3
:10558000C1540108C1540108C15401086157010800
:105590004B5701085E2B21D8522B91D9A3F153020E
:1055A0000B2A8DD801A151F822F000BF6B570108DA
:1055B0007D57010887570108C1540108C1540108EB
:1055C000C1540108C1540108C1540108C154010863
:1055D000C1540108B157010887570108722B00F028
:1055E000E28007D8702B7FF46BAF0AB0BDE8F047BC
:1055F000FFF7C4B8D42B09D8BB2B3FF669AFA3F192
:10560000B202012A3FF65CAF012052E0DF2BFBD053
:1056100040F6B8329342F7D052E700F5AF46503625
:105620001621304607F06AF930B1294630460AB0F3
:10563000BDE8F04707F056BC20460AB0BDE8F04789
:10564000FEF780BE29460AB0BDE8F047FFF74CBE22
:1056500000F5AF4550351521284607F0ABFE28B1BF
:1056600028460AB0BDE8F0470BF0A2B904F5A04502
:1056700004F5AC46D5F8FC3404F5AD4704F5AE4866
:1056800004F5AE49072B06F1380607F1780708F153
:10569000180809F108090FD104F5A94478340194D8
:1056A000D5F88034009342464B463946304685F063
:1056B0005FFA0AB0BDE8F0870DF127018DF82700E9
:1056C0004148FEF761FA05F2BC43D3ED007AD5F804
:1056D000A0A405F59263D3ED000A05F29C4330EED9
:1056E000670A93ED001A8DED070A04F5AF40083004
:1056F000CDED060A8DED051A76F0B8FF0546204679
:1057000000F074FF9DF827309DED051ADDED060AC7
:105710009DED070ACDE90203CDE900A54B464246BF
:105720003946304685F07AF9C3E7A98805F0C8FC08
:105730000020BEE729460AB0BDE8F047FFF7F6BCF7
:105740000AB0BDE8F047FFF7B3BC29460AB0BDE890
:10575000F047FFF723BD0AB0BDE8F047FFF780BD73
:105760000AB0BDE8F047FEF7E3BE04F598402946CD
:1057700020300AB0BDE8F047FEF756BF04F5AF4051
:105780002946503053E704F5AF465036304607F00F
:10579000F5FD08B9304664E729462046FFF76CFA64
:1057A0000028F7D185E70AB0BDE8F047FEF7FABF59
:1057B00004F59840294620300AB0BDE8F047FEF7CE
:1057C000B1BF00BF50F30C08702B002070B500F57E
:1057D000804200F59843D2F8C02E20339A42054605
:1057E0000E4602D00024204670BDFFF75FFE04463F
:1057F0000028F7D005F54E503188083058F04AFDA2
:10580000F1E7000021F04003152B04D0A1F15E0365
:1058100058425841704701207047000000F580420F
:1058200000F59843D2F8C02E20339A4207D100F5F4
:10583000A040B0F85E355B1A5842584170470020CE
:1058400070470000192963D8DFE801F00D11151920
:105850001D2125282C62303437563A3A3D404347C3
:105860004A4E62525A5E00F599404030704700F54A
:1058700096401430704700F596403030704700F580
:1058800096404C30704700F596406830704700F500
:1058900097402430704700F59740E6E700F59740C1
:1058A0005C30704700F598400430704700F5984030
:1058B0002030704700F59840E3E700F59840E4E7B2
:1058C00000F59940F0E700F59940E2E700F59940CE
:1058D000E6E700F599407830704700F59A40C8E750
:1058E00000F59A403430704700F59A4050307047C8
:1058F00000F59A407030704700F59B4028307047A3
:1059000000F59B406430704700F59B400C307047B9
:105910000020704700290DDB074890F8EC2BCBB234
:105920009A4207D3D0F8E83B0122595CA0F5005019
:105930000DF0ECBA704700BF704B00202DE9F34129
:1059400000F5005300F54E5593F8B83B03F00106FF
:1059500003F0020803F004075B07044605F108059D
:1059600035D01F4A0621284654F054FB26B104F5D1
:105970003B503C3078F0A8FEB8F1000F04D004F59D
:105980004150143078F01CFC27B104F546502C30FF
:1059900079F0C4FA04F5A044012384F8213B114AAC
:1059A000114B1249B8F1000F08BF1A46002F08BF6B
:1059B0001946CDE900210E4A0621002E18BF1346D4
:1059C00028460C4A54F026FB02B0BDE8F0810A4A92
:1059D0000621284602B0BDE8F04154F01BBB00BFD1
:1059E0007DF30C0872F30C0804DD0D0879F30C0844
:1059F0006CF30C088EF30C08A0F30C0810B50446E9
:105A000000F53B503C3078F08BFE04F541501430EB
:105A100078F002FC04F546502C3079F0B9FA04F520
:105A2000A04393F8212B5AB1002283F8212B04F5CF
:105A30004E50044ABDE810400621083054F0EABA3E
:105A400010BD00BFC0F30C0809B1FFF777BFFFF727
:105A5000D5BF000000F580430A4AD3F8C01E91422A
:105A60000DD093F8CD3E43B900F5984220329142D3
:105A700003D100F5A04090F8B234184670470023D7
:105A8000FBE700BF3078002010B5044688F0DEFB4D
:105A9000054BD3F8E03EC01A642804D82046BDE880
:105AA00010405CF059BB10BD706B002010B500F5C4
:105AB0002E54D4ED0A7AF5EEC07AF1EE10FA8AB0DF
:105AC0004FF0000304F1280445D907930893099384
:105AD00006AB019300F5935007AB009303AA05AB07
:105AE00004A9083013F0E0F930B3DDED080A9DEDAC
:105AF000070AACF09BFEDDED090AACF097FED4ED91
:105B0000007A9DED047A77EEA76AB4EEE70AF1EE2B
:105B100010FAF4EEC76AACBF01200020F1EE10FAD3
:105B20000CD802309DED037AF4EEC77AF1EE10FA4C
:105B30000CD8003818BF01200AB010BDF4EEC77AA7
:105B4000F1EE10FA9CBF0130C0B2EBE7012894BF20
:105B500000200120F0E70020EEE7000038B5124BEE
:105B60001A7A0446FAB901251D7252F011FA2A4632
:105B700004F5AF451121503552F066F9284607F07B
:105B800081FC80B1284607F039FC062238B104F5C3
:105B90009A413431BDE8384004480DF0DFB804F5CF
:105BA00099417831F6E738BDA8860020702B002097
:105BB00010B5074B1A7A4AB100241C7252F0E8F96A
:105BC00022461121BDE8104052F03EB910BD00BF81
:105BD000A88600202DE9FF41054605F59358684643
:105BE00008F1080819F040FA6946404613F0B0FA87
:105BF0000646E8B1374876F039FD50B105F52E5329
:105C0000D3ED0A7AF5EEC07AF1EE10FA94BF0126D0
:105C1000002605F5AF40503007F034FC2E4C2F4FD6
:105C200000B146B1002328462380FB73FFF7C0FF75
:105C300004B0BDE8F0812846FFF738FFA0B36378D1
:105C40007BBB23780133DBB2082B237002D14046A3
:105C500013F096F92378092B02D1404613F088F906
:105C60002378092B1DD94FF48573238052F090F9C6
:105C70000222102152F0E8F888F0E8FA6368C01AAE
:105C800047F23053984209D905F54E50144A022183
:105C9000083054F0BFF988F0D9FA60602846FFF761
:105CA0005DFF6378FB73C3E72378002BF9D0013BDA
:105CB0006278DBB22370002AF3D0002BF1D166703A
:105CC00052F066F93246102152F0BEF82846FFF72E
:105CD0006FFFE6E7F8820020A886002055870020A5
:105CE000D4F30C0810B500F5A044D4F8FC34042B10
:105CF00001D1012010BD00F5AF40503008F04EF941
:105D00000028F6D194F82805F4E7000073B500F5F3
:105D100080450192A5F8D81E044688F097FAC5F888
:105D2000DC0ED5F8C00E03685B68984785F8D60E80
:105D3000D5F8C00E03685B689847019A182818D8F0
:105D4000DFE800F00D170D0D0D0D0D0D0D1752179D
:105D50005917595917414141171717415900334BEA
:105D600093F8223B03B304F59741243120460CF00D
:105D7000F5FFD5F8C00E95F8D66E03685B689847B6
:105D800004F54E54864204F1080447D0D5F8C00EFD
:105D900003689B689847264A03460421204602B0C0
:105DA000BDE8704054F036B904F5005393F9BC31A6
:105DB000022BD8D0042B0BBF04F5974104F5964174
:105DC00040311431D2E704F5A043D3F8943AD90214
:105DD00003D504F598414C31C8E704F59A419B0678
:105DE0004CBF50313431C1E720460192FFF77AFFB2
:105DF000019A0028BDD104F50056019296F9BC31F4
:105E0000002BB6D0D5F8C00E03685B68984785F8BC
:105E1000D60E96F9BC31019A022BCAE7054A042135
:105E2000204602B0BDE8704054F0F4B8707B00200A
:105E3000E4F30C0806F40C08F0B5044604F58046BB
:105E400085B00F4615465CF00DF9D6F8C00EA6F8E1
:105E5000D87E03685B68984718281ED8DFE800F0F2
:105E60000D0D0D0D0D0D0D0D0D1D64810D0D7070C1
:105E70001D5252521D1D1D520D003D4AD2F8FC14F8
:105E8000012921D104F5005393F8BD31023B012BC8
:105E90001AD904F5405383F88413D6F8C00E354A56
:105EA000354B052D18BF134602680393926890473F
:105EB00004F54E5408340090039B304A04212046D8
:105EC00054F0A8F805B0F0BD92F8223B3BB104F5C0
:105ED00097412A46243120460CF040FFDDE704F5C7
:105EE000005393F9BD31032B03D1204605F050F93F
:105EF000D3E7022BEBD0042B2ED104F598412A4690
:105F00002031E8E704F5A043D3F8943ADA0223D429
:105F10009B0604D504F59A412A465031DBE704F587
:105F20009A412A463431D6E72046FFF7DBFE0028A7
:105F3000B3D104F5AF40503007F0CEFA0028EED1CF
:105F400004F5005393F9BD31032BCED0022BBED004
:105F5000042BD2D0012BA0D104F598412A464C3114
:105F6000B9E704F5005393F9BD31042B95D1C4E78B
:105F7000707B00201CF40C0898D80C0824F40C0842
:105F800070B500F54E5504460835124A04212846DE
:105F900004F5804654F03EF80023A6F8D83E04F5F8
:105FA000005393F80431032B12D196F8D61E3022F9
:105FB00020460CF0ABFFD6F8C00E03689B689847EC
:105FC000054A034606212846BDE8704054F022B831
:105FD00070BD00BF38F40C084FF40C0800F54053B6
:105FE00010B500220529044600F54E5083F884239D
:105FF00000F108000CBF054A054A042104F580445D
:1060000054F008F80023A4F8D83E10BD68F40C083A
:1060100079F40C08013A38B50446052A3ED8DFE881
:1060200002F04B1B8711900300F5A04393F8E4386E
:1060300043B100F59B4104220C314448BDE838408F
:106040000CF08CBE04F5A04393F8E43823B104F5BA
:106050009A4104223431F0E704F58043D3F8C02E8E
:1060600004F59A4334339A4226D004F59B430C330B
:106070009A4221D004F5A043D3F8FC34042B1BD062
:10608000334D95F8F13EBBB1324905F5A95030F0DA
:1060900095F920B1304B012283F8282538BD2D49D0
:1060A00005F5A95030F08AFC30B104F5984104227E
:1060B0002031A5F58040C1E704F58043D3F8C02E18
:1060C00004F59A4334339A42E8D004F59B430C33E9
:1060D0009A42E3D004F5A04304F5AF405030D3F822
:1060E000FC5407F05BFF0028D8D1042DD6D004F56E
:1060F000005393F98731022B0DD004F598412046C7
:1061000004224C310CF02AFE04F505500730BDE89E
:10611000384048F095BB0E4890F8F13E002BECD08B
:106120000C4900F5A95030F049F90028B2D1E4E754
:1061300000F5AF40BDE83840012214210830F7F7E0
:1061400019BDBDE8384005F023B800BF702B002012
:10615000706B002078820020707B002070B52DEDE0
:10616000068B044688F066F8414BB4F8BE101A88D6
:10617000404E8A420546404A06D0198000233060CE
:106180001370BDEC068B70BD33683C49C31A8B425B
:1061900065D9012313705CF065F85BF01DFF356075
:1061A0005CF060F85BF018FF5BF03EFF0428E8D974
:1061B0005BF058FF204600210BF00CF82046002130
:1061C000B0EE40AA0BF010F820460121F0EE409A04
:1061D0000BF0D0F900212046B0EE408A0BF00EF80B
:1061E00004F5AF400830F0EE408A76F049FA9FEDB2
:1061F000249A0028B0EE4A0A4FF0040008BFB0EE1F
:10620000498A5DF041FBB0EE690A13205DF03CFB6A
:10621000B0EE680A15205DF037FBB0EE680A1A2070
:106220005DF032FBB0EE480A46205DF02DFB012107
:1062300008465DF035FEB0EE490A02205DF024FB11
:10624000B0EE490A03205DF01FFB20460BF0C0FBB7
:10625000BDEC068B2046BDE870400CF00BBB1278FD
:10626000002A8ED044F6206293428AD993E700BF79
:10627000B4860020B8860020B6860020400D0300BA
:106280000000000000F5804200F59843D2F8C02ECF
:1062900020339A4204D100F5A04090F82805E8B1D7
:1062A0000F4B93F8040103F54053A0F12702012A94
:1062B00093F8303B0FD92C2809D00A2809D0A0F137
:1062C0003102504250410A2B18BF00207047012074
:1062D000F9E7012070470A3B58425841704700BF18
:1062E000704B002008B500F5005393F8482042B1E8
:1062F00093F884302BB1FFF7C5FF80F00100C0B2E6
:1063000008BD0120FCE700002DE9F04700F500552D
:10631000B04E95F884A0044600F5AF408AB008302E
:1063200076F0A4F9D6F8FC34042B814642D1012141
:1063300004F5015808F10808404666F09DF996F802
:10634000303B0A2B074605D1B9F1000F54D1002389
:1063500086F8303B95F84830002B58D195F94E30EF
:106360009D4D012B03D0063BDBB2012B11D895F8D4
:1063700004310A2B0DD104F58047D7F8C00E03680D
:106380001B6A984728B1D7F8C41E2B2220460CF070
:10639000E5FC96F8303B0A2B04BF372386F8303BE8
:1063A00095F804310A2B02D1372385F804310AB05D
:1063B000BDE8F0870028BAD004F58043B6F85E75D2
:1063C000D3F8C00E03685B6898471428AFD004F573
:1063D000AF40503007F030FC0028A8D13946A6F570
:1063E000A040FFF70FFA01460028A1D096F8241527
:1063F0004B1E594259419BE740EA0A03DBB2002B8E
:10640000A8D1764800F0F2F80028A0D0A2E7B9F1B0
:10641000000FCCD004F5AC40383084F075FA002879
:10642000C5D12046FFF72EFF0028C0D1002F00F075
:10643000BF806B493A46404665F0F6FC95F94E90B0
:10644000B9F1010F07D040F38780A9F10603DBB251
:10645000012B00F281805FFA89F9B9F1010F4ED169
:1064600004F5804204F59843D2F8C02E20339A42B6
:1064700009D104F5A04393F8283523B195F8873165
:10648000013B012B93D904F598410A224C31204657
:1064900006AE0CF063FC304618F0E6FD95F961207D
:1064A00092BBB9F1010F2FD004F5A049B5F96230C4
:1064B000D9F8F416DFED4B5AD1ED017A002BF8EE46
:1064C000E77A52DD07EE103AF8EEC76AE6EEA57AF3
:1064D0003046FDEEE77A17EE901A18F0CBFD002358
:1064E0004046CDE9043366F063F904A966F0A4FEE2
:1064F000002857D0049B0893059B099317E004F5E7
:1065000099410A220431C2E72046FCF787FE07EED4
:10651000900AE84604F5AE42083221464046B8EEFD
:10652000E70AFDF725FD98E80F0086E80F0095F9CA
:106530004E30012B10D031462046FCF7C5FF3146C6
:106540002046FDF7FBFB95F94E30072B04D104F5EF
:106550004054012384F8823351F01AFD3A46092150
:106560000AB0BDE8F04751F06FBCD5ED146A95ED67
:10657000175A95ED157A35EE076A36EEC57AB4EE00
:10658000C67AF1EE10FA89BF37EE067A95ED7A7A7F
:1065900027EE257AF6EE006A94BFE7EE257AE7EE5D
:1065A000267A95E7D9F8F4369A680892DB68A4E76A
:1065B000BAF1000F3FF4FBAE95F88430002B7FF466
:1065C000F6AE04F54E50084A0521083053F022FD7E
:1065D000C2E700BF707B0020704B0020702B0020B2
:1065E00094F40C080000C8429DF40C0810B5044651
:1065F00000F5AF40083076F043F898B104F5AF40AD
:10660000503008F0C1F960B904F5AA4494ED007A5D
:10661000DFED087AB4EEE77AF1EE10FAACBF0120B4
:10662000002010BD04F5AA4494ED007ADFED027A53
:10663000F0E700BFCDCCCC3D6666663F70B500F597
:10664000804600F59B43D6F8C02E28339A42044674
:1066500000F5A04502D195F8F804D8B904F5AF408B
:10666000B5F85E15503006F049F9A0B9D6F8C03E2D
:1066700004F598442034A3420CD195F8F8344BB17A
:10668000D5F8FC34032B05D1B5F85E05A0F116034F
:106690005842584170BD0020FCE700002DE9F74F3B
:1066A00000F5804200F59843D2F8C02E20339A427C
:1066B000044600F5A04504D100F5005B9BF960316C
:1066C0003BB90023C5F8EC3485F8E93403B0BDE8E4
:1066D000F08F87F0BBFDD5F8A464804636B1861BE9
:1066E00040F6C3139E4294BF002601262046FFF7C2
:1066F0007DFF019028B1002785F8E8744FF0000A6B
:1067000046E004F5AF40083075F0B0FF8146002840
:10671000F1D004F5AC4A0AF1380A504684F0F4F896
:106720000746002845D095F8E8A4BAF1000F3BD100
:1067300056B304F5805041F27071D0F86024002AFD
:10674000B8BF52428A4206DCD0F86424002AB8BF9F
:1067500052428A422BDD04F5AA4104F5AE40643171
:10676000083018F0B1FFDFED487AC5F8EC84B4EEDC
:10677000E70AF1EE10FA4FF000024CBF4FF0010AA9
:106780004FF0000AC5F8F024012285F8E8243746C6
:1067900004F59070F7F73AFB022832D9002F44D164
:1067A0000023C5F8EC3491E7019EB246ECE756466B
:1067B000EAE7504684F090F8824648B1002E9DD01A
:1067C0004FF4FA73C5F8F0344FF0000A4F46DFE794
:1067D000D5F8FC24012A07D0032AD9D12046FFF797
:1067E0002DFF00288AD1E9E7DBED807AF5EEC07A4B
:1067F000F1EE10FA82DD95F8F834002B7FF47EAFCD
:10680000DEE704F5F45604F58059103699F8DE1FDA
:10681000304610F05FFB0028C2D099F8DE1F3046EA
:1068200010F050FC0028B9D1BAE7D5F8EC0410B943
:10683000C5F8EC844AE7D5F8F024A8EB00089045A9
:10684000FFF444AF95F8E924002A7FF43FAF01221A
:1068500085F8E9249BF86011CB0705D504F5AF4016
:106860000C210830F7F786F904F54E500830BAF1DC
:10687000000F06D0054A022103B0BDE8F04F53F0E7
:10688000C9BB034A5146F7E700009642B4F40C082E
:10689000CAF40C082DE9F04F2DED028B044685B0AB
:1068A000002304F50059039387F0D0FCD9ED577A03
:1068B000F5EEC07AF1EE10FAC4BF9FEDC47A67EE30
:1068C000877A04F5907BC8BFFCEEE77A804658468D
:1068D000CCBF17EE907A9627F7F798FA022840F285
:1068E0000C8194F8E4339FEDBA7AB02202FB0343A3
:1068F000D3ED777A67EE877AFCEEE77A17EE903A77
:106900009F428CBF00270127B9F95031022BB8BF35
:10691000022307EE903A04F59350B8EEE78A03A9F4
:10692000F6EE087A083028EE278A12F0EFFB0546CB
:1069300040B1DDED037AF4EEC87AF1EE10FAACBFA7
:10694000012500255846F7F761FA01281AD804F501
:10695000AF40083075F08AFEA0B19DB904F5AA4396
:1069600093ED007ADFED9B7AB4EEE77AF1EE10FA60
:1069700008DDDDED037AF4EEC87AF1EE10FAACBF73
:106980000125002504F5AF40503005F009FA04F563
:10699000A0468246002840F0018104F5AF4008304F
:1069A00075F064FE002800F0078194F8E43304EBEE
:1069B0000313D3F890317BB158460193F7F726FAC9
:1069C000012800F29C80019BA8EB030041F2873371
:1069D00098428CBF00230123D6F8A02402B11BB932
:1069E000002D40F08E803D4604F5804204F598432A
:1069F000D2F8C02E20339A421AD199F98831002B4F
:106A000040F08780002386F8EA34D6F8FC34042B63
:106A100000F0B080072B00F0C380032B08D1204684
:106A2000FFF70CFE20B1002586F8E954C6F8A454FF
:106A300096F8EA3403B18DB907EE905A9FED667A65
:106A4000F8EE677A04F5AA4367EE877AD3ED006A19
:106A50009FED627AE6EE877AC3ED007A2046FFF773
:106A6000C5FD0546A8B196F80415C6F8A08409B975
:106A7000C6F8088504F5804204F59843D2F8C02E84
:106A800020339A4205D1D6F8A43403B109B9C6F827
:106A9000A48496F82C3686F8045565F3C30386F86B
:106AA0002C366EF073FD29466EF04CFD4C4B2046A3
:106AB0005D71FFF7F3FD2046FAF75EFD35B199F8F9
:106AC00006311BB987F0C2FBC9F8080189F80651E5
:106AD0002046FFF78BFD002840F08E8004F5AF4084
:106AE000083075F0CDFD80F00100C0B286F80C05CD
:106AF00005B0BDEC028BBDE8F08F002704E75346DC
:106B00006AE728F015FD27F063FE00287FF46BAFDD
:106B10006AE75B4207EE903A04F69803F8EEE77AEC
:106B200093EDDB7AF4EEC77AF1EE10FA13DD012370
:106B300086F8EA34C6F8F48404F5AA43DFED297A2E
:106B400093ED007AB4EEE77AF1EE10FA7FF75DAFDD
:106B5000C3ED007A59E796F8EA34002B3FF455AFBD
:106B6000D6F8F43440F6B832A8EB030393423FF66C
:106B700049AF4AE704F5AC40383083F0ADFE002859
:106B80003FF456AF06F5926393ED007ADFED157A88
:106B9000B4EEE77AF1EE10FA7FF74AAF012547E746
:106BA00006F5926393ED007AFEEE007AB4EEE77A92
:106BB000F1EE10FAF2D43BE7D6F8FC34002D18BF02
:106BC0003D46012B10D1002532E700BF0000B44242
:106BD0000000C8429A99993E9A99193E9A99593F4C
:106BE00055870020CDCC4C3E04F5AC40383083F0C6
:106BF00069FE0028E7D11BE7002077E700207047F7
:106C00000020704701207047034BD3F8FC04431E5B
:106C100058425841704700BF707B002030B587B0A4
:106C200002A818F021FA374883F04CFE20B136490B
:106C30003648FCF729FB1FE0324883F04DFEE8B1EF
:106C4000334C04F12405234604F11002A4F1100191
:106C5000A4F1D000009583F065FECDE90045A4F5D0
:106C60001C7292ED000A2B4904F11003A4F11002EA
:106C7000A4F1D00083F018FE07B030BD214802A96E
:106C800083F068FE08B102A9D2E7234CD4F8703B28
:106C9000002B0CDD94F8103B4BB1A4F500501C49BF
:106CA000FCF7F2FAA4F50050FCF7A6FBE4E717485E
:106CB00004F036F90028BAD1184CD4F82C37002B40
:106CC000B5D004F5E36204F5DF6104F5E16018F086
:106CD00067FC0028ABD104F29C45D5ED007AB7EEF5
:106CE000000A04F5E361A4F5A04030EE670AFCF762
:106CF00031FC04F5DF6204F5E361A4F5A040FCF784
:106D0000DBFAB9E7A881002088820020702B0020E0
:106D10007882002060570020704B0020707B00209C
:106D200008B50A4890F8F931013B012B03D8A0F5CA
:106D30000050F8F7FFFA0648F8F7CAF90448F8F7E0
:106D4000B9FABDE808400248F8F71EBE704B0020B3
:106D5000702B002010B5044607480CF0F3FE50B12C
:106D6000064B93F8110930B1236820469B6B984776
:106D700080F00100C0B210BD78850020707B00203B
:106D8000124B984210B5044601D1002010BD03F10A
:106D90001C029042F9D003F138029042F5D003F181
:106DA00074029042F1D0D4339842EED003681B6A4B
:106DB000984720B1064B93F88233002BE5D1206928
:106DC00007F006F980F00100C0B2DFE7A0760020EE
:106DD000705B0020174B984210B504460ED003F1AB
:106DE0001C0290420AD003F13802904206D003F10F
:106DF0007402904202D0D433984206D10E4B93F9DC
:106E0000B101B0FA80F0400910BD03681B6A9847D1
:106E100018B10A4B93F8823343B9206907F0D8F8C8
:106E200030B12069BDE8104009F078BC0020EBE7E4
:106E30000120E9E7A0760020704B0020705B002065
:106E400073B50F4E0D46114696F99C281AB90124C8
:106E5000204602B070BD036801915B699847044603
:106E60000028F4D1D6F8943A019913F4802FEED08B
:106E70000448054B00682A46C06A25F03FFDE7E755
:106E8000707B00206C2B0020DCF40C08084A0260A8
:106E9000084A4260111F816002F10801C160A2F13D
:106EA000380102F59C724261034A016182617047B8
:106EB00028F50C0878830020D83D002008B5036829
:106EC0001B6E98470648D0F8C02E00F604439A423D
:106ED00005D0BDE80840A0F58040FEF78FBD08BD95
:106EE000706B00202DE9F3415A4C04F58F630022AA
:106EF0001A60A4F57873C11A4B42A4F500584B41AF
:106F000088F8183604F59163002684F85C64A4F8C8
:106F1000B26484F8B66484F8746484F8E96484F82C
:106F2000EA64C4F8DC64C4F8D864C4F8D464C4F86F
:106F3000E4641A608369D3F8FC31A4F8AC3404F536
:106F4000E16305460FCB04F5DF6787E80F0084F89F
:106F5000B56484F8C464C4F8D46687F077F9A4F5FE
:106F60008057C7F8C80E2B6828465B6998474FF0D2
:106F7000FF3384F8B964C7F8F83E88F8846384F86E
:106F8000B804286906F0B2F984F8B7642B6828467B
:106F9000DB6D98470646002858D02B6828469B6B27
:106FA000984784F8F804D8F8A4050368DB6B984781
:106FB000A4F5E75077F0F0FCA4F5A0400AF05CF8E7
:106FC000A8F6B87065F0BEFB94F82835CBB1A4F5EF
:106FD000A040FFF70BFBA0B904F5F16075F050FB82
:106FE00078B9D7F8C00E03685B6B984748B959F079
:106FF0008DFE194A062153F00DF804F5A4602FF018
:1070000089FA1648F7F7DCF92B6993F9CC206AB1B5
:10701000586801A912F07AF82C699DED010A014621
:1070200004F18800FBF7A2FE84F841012B68284692
:107030005B69984750B12B6993F93C22002A02DD25
:1070400093F8A03213B9002387F8CD3E304602B042
:10705000BDE8F081707B0020E8F40C08702B002064
:1070600070B503685B6E0E4615469847044650B9E6
:1070700095F900303BB90548054B00683246C06AB7
:10708000294625F03BFC204670BD00BF6C2B00203C
:107090000CF50C0810B50E4C204677F079FA04F583
:1070A000AC7076F0F1FF04F52C7077F01FFF094B00
:1070B00003F5A042002182F8741402F58F620021CA
:1070C00003F500531160012283F8482E10BD00BF64
:1070D0006C5A0020702B002008B52DED028B152076
:1070E000B0EE408A5CF0D0FBB0EE480ABDEC028BFB
:1070F0001A20BDE808405CF0C7BB000008B508488E
:1071000090F9B1310121A0F5005033B10AF032FA03
:10711000BDE8084046205CF0B7BB0AF053FAF7E739
:10712000704B0020012070470120704701207047FC
:1071300001207047012070471920704700487047B0
:1071400090F50C0800487047A0F50C0884B010B505
:1071500003AC84E80E000369B3F9C01064235943FB
:107160002046012217F086FF04482146FCF7E6FD81
:10717000BDE81040012004B0704700BF702B002014
:1071800013B50F4901AAA1F1100018F029F840B178
:10719000DFED0C7A9DED017AB4EEE77AF1EE10FAAC
:1071A0000CD8094CD4F8A40503689B6B984728B108
:1071B00006492E22A4F540500BF0D0FD02B010BDC0
:1071C00088820020000000B4705B0020A4780020BA
:1071D00030B51D4C0546D4F8C40E036887B05B6912
:1071E000984738B119491A482F220BF0B7FD0120F2
:1071F00007B030BD174806F0EBFE0028F2D1A4F529
:107200008054D4F8A40503689B6B984728B1D4F840
:10721000A40503681B6C984798B10F4B0FCB02ACC9
:1072200084E80F00284601F065F82868059B009364
:1072300094E80E00446C2846A0472846FFF7A0FFBC
:10724000D5E7064BEAE700BF706B0020A47800206A
:10725000702B00204083002078820020888200204C
:1072600010B50446FFF78CFF2046BDE8104001F042
:107270007DB80000042070470048704795FB0C085B
:107280000048704795FB0C08037F73B1D0ED087A76
:10729000FDEEE77A17EE903A084AC2F81035437FC0
:1072A0003BB1436AC2F8143570478369D3F8F831AB
:1072B000F2E78369D3F8FC31F4E700BF707B00206C
:1072C00008B50023838300F12801806911F034FFA1
:1072D000012008BD70B56E4E2DED048B06F59E4362
:1072E00004460121304693ED049ADFED6A9A09F0D5
:1072F00071FF0121B0EE408A304609F075FFC8EEFB
:10730000297A06F50055A069B5F9D43104F12801B0
:1073100008EE903AF8EEE88AB5F9D63168EEA78A19
:10732000C0EE297A08EE103AB8EEC88A28EE278A0D
:1073300011F002FF95F9DA3163B39FED577AF0EE61
:10734000E87AF4EEC77AF1EE10FA23D5227FA3692A
:10735000002A55D1012222770022226294ED087A78
:10736000DFED4E7AD3F8F8314D4A4E4867EEC77AD2
:107370009FED4D7A67EE877AB0EE490AFDEEE77A27
:1073800017EE901A0B44C2F810350023012277F053
:107390008FF808E0002343482377F0EE490AB0EE67
:1073A000680A77F081F804205CF06EFA95F9DA311A
:1073B00043B19FED397AF0EEC87AF4EEC77AF1EE78
:1073C00010FA28D4002339486377F0EE490AB0EE6A
:1073D000480A76F0C3FC13205CF056FAB5F9D831B0
:1073E000002B03DD324E96F9C23163BB28482021C1
:1073F000F7F71AFB002843D1254809F00DFD42E0BC
:10740000D3EDC56A96ED467AD4ED087AE6EE877A32
:10741000C4ED087AA2E7637F2BB901236377A369E0
:10742000D3F8FC3163621E4B616AC3F81415A3697B
:10743000D3F8FC010023091A1A461C48B0EE490A89
:1074400076F072FDC7E70121A6F5405009F0D6FE9F
:1074500080EE297AB5F9D831002106F5D67007EE0D
:10746000903AF8EEE77AF0EE490A27EE870A77F0CD
:107470003DFCBDEC048B2046BDE87040FFF72CBE00
:107480000348F8F7EDF807EE900AB8EEE70AF0E7E0
:10749000702B002000A08C4500000034E02E6542D7
:1074A000707B00206C5A00200000C842C45B0020A2
:1074B000705B00202DE9F04F2DED0C8BDFF8A4A3BD
:1074C0009FEDDDDA9FEDDD9A97B00AF59E4300F15E
:1074D000280504460121504693ED04BA09F07AFECE
:1074E00001215046F0EE408A09F07EFE012150460F
:1074F000B0EE408A09F082FEDFEDD17A88EEA77AFD
:107500000AF5005601A8B6F9D4310AF5A04B0AEEE7
:10751000903AF8EEEAAAB6F9D631DFEDCA8A6AEEF9
:1075200087AA88EE277A0AEE103AB8EECAAAB6F908
:10753000D8319FEDC58A2AEE07AA80EE277A09EE98
:10754000903AF8EEE99A6AEE8D7A69EE879AF0EE53
:10755000EACAF4EEC8CACDED017AB0EECACA6AEE44
:107560000D7AF1EE10FAF0EEE9BAB4EEC8CACDED3C
:10757000027A58BF4FF0010969EE8D7A48BF4FF08B
:107580000009F1EE10FAF4EEC8BA9AED460ACDED14
:10759000037A54BF4FF001084FF00008F1EE10FAE3
:1075A00054BF012700272BF05DFE01A928462BF0D0
:1075B00003F928462BF0FAF928462BF069F920EE5A
:1075C000090A284620EE280ABDEEC00A10EE103A3D
:1075D000CBF810352BF076F920EE090A20EE280AB8
:1075E000DFED9A8ABDEEC00ACDED0D8A10EE103A9D
:1075F000CBF814350DF1280B4FF07E535946A06996
:107600000A93CDED0C8ACDED0B8A11F095FD00218A
:10761000504609F0AFFFB0EEC00AB4EEC80AF1EE72
:1076200010FA16D55046FEF7E1FF90B9F4EEC8CA3D
:10763000F1EE10FA0DD5B4EEC8CAF1EE10FA08D585
:10764000F4EEC8BAF1EE10FA44BF9BE80F0085E8EB
:107650000F000AA82BF00EFA294612A88DED141A75
:107660008DED120ACDED130ACDED151A2BF014FA9B
:107670000DF1100A51460EA88DED101ACDED048AB9
:10768000CDED058ACDED068A8DED0E0ACDED0F0A02
:10769000CDED111A2AF0CAFFB6F9D431DFED6C7ABC
:1076A00001EE103AB6F9D63109EE103AB6F9D831F2
:1076B00008EE903AB8EEC11AB8EEC99AF8EEE88A28
:1076C00021EE271A29EE279A68EEA78AF4EEC8CA97
:1076D000F1EE10FA21EE0D1A29EE0D9A68EE8D8A60
:1076E00007D594F83830DFED597A002B18BFB0EE8B
:1076F000671AB4EEC8CAF1EE10FA07D594F839301B
:10770000DFED527A002B18BFB0EE679AF4EEC8BADC
:10771000F1EE10FA07D594F83A30DFED4C7A002BF1
:1077200018BFF0EE678A9AE8070007AE86E8070000
:10773000F1EE410AC2209DED070A28F031FCC3207A
:107740008DED070AB0EE491AF1EE490A9DED080ADF
:1077500028F026FCB0EE681AF1EE680A8DED080AF2
:10776000C4209DED090A28F01BFC514630468DEDE2
:10777000090A2BF00DFD12A928468DED120ACDED58
:10778000130A8DED141A2BF017F828462BF00EF97A
:10779000304BDDED076A93ED007A9FED280AC6EEC7
:1077A000877A3046DDED086ACDED077AD3ED567A5B
:1077B00086EEA77ADDED096A8DED087A86EEA77A66
:1077C0008DED097A2BF04EFDB9F1000F01D0CDED12
:1077D00007AAB8F1000F01D08DED08AA0FB1CDEDC9
:1077E000099AF0EE4B0A9DED070A1B4876F05CFE05
:1077F00004205CF049F8F0EE4B0A9DED080A1748AA
:1078000076F0ACFA13205CF03FF80021F0EE4B0A62
:107810009DED090A124877F069FA2046FFF75CFCF3
:1078200084F8389084F8398084F83A7017B0BDEC49
:107830000C8BBDE8F08F00BF35FA8E3CE02E654220
:1078400000A08C450000C842000000340000000089
:10785000CDCC4C3E705A00206C5A0020C45B0020F6
:107860001C5D0020702B002010B50446FFF746FC7D
:107870000B4B93F9DA21022A0DD1B3F9D821002A52
:1078800009DD03F5805393F9C23123B12046BDE8E9
:107890001040FFF70FBE2046BDE81040FFF71ABDAD
:1078A000704B00200A20704700487047A21B0D084B
:1078B00000487047A21B0D08012070470120704747
:1078C0000120704701207047034BD3F8FC04031FCD
:1078D00058425841704700BF707B002038B50546BC
:1078E0002C48D0F8C42E00F684439A4215D12B6957
:1078F00093F844318BB100F5A9502EF0D5F9044628
:1079000058B959F003FA244A032152F083FB2B693A
:10791000012283F84321204638BD204C94F8E438F6
:1079200023B194F99C389A1E5342534184F8B834D9
:1079300004F5E1630FCB04F5DF6504F5E36485E846
:107940000F0084E80F0016482FF024F8154B1C6830
:10795000E56A2B6828465B689847A8B195F84D30D2
:1079600093B1E36A9B8F7BB159F0D0F9E36A0E4A79
:107970009B8F062152F04EFBE36A0948998F2EF047
:10798000F5FDE36A00229A87084883F01DFF012471
:10799000C1E700BF706B002088F60C08707B0020E8
:1079A000908000206C2B0020A2F60C08F8540020D8
:1079B00038B50D4C94F82435012B11D104F5A46091
:1079C0002CF0EAF8B4F85E5504F5FA60294605F0A3
:1079D000F1FC28B9152D03D104F5C76083F052F8E6
:1079E0000023C4F8A43438BD707B002008B511F022
:1079F000BDFD90F87C32DB0704D5BDE808400248A5
:107A00002EF064BE08BD00BF9080002038B5354C14
:107A100094F82435012B0ED0A4F56D710822A4F53D
:107A2000A0400BF09BF959F071F9BDE838402E4A9F
:107A3000062152F0EFBA04F5FA60B4F85E5505F08D
:107A4000DDFC28B104F5FA60BDE8384008F010BE4E
:107A5000162D05D0152D36D1D4F8FC34072B0AD1BC
:107A600022480CF08DFF21480DF0D6F8BDE83840D3
:107A70001E480CF0E7BFA4F5A040F8F713F9A4F5F1
:107A8000A040F7F7F1FFA4F54053D4F8101593F98F
:107A9000182264235A4304F5C76082F04FFFC4F8EC
:107AA000100504F5C76083F08BF830B1BDE83840AD
:107AB0009FED0F0A46205BF0E7BEA4F5A040BDE8AD
:107AC0003840F7F7B5BD1E2D18BF4FF0FF330748FC
:107AD00018BFC4F87034F8F7E5F80448F7F7C4FFA6
:107AE0000248ECE7707B0020BCF60C08702B0020ED
:107AF0000000000070B5134890F99C380E461546FA
:107B000013B90124204670BDD0F8943A5B0310D518
:107B1000B0F85E1500F5FA6004F0F0FE044640B9D6
:107B2000094B0A48006832462946C06A24F0E6FE3E
:107B3000E8E707482EF0B8F804460028E1D1054BE5
:107B4000EFE700BF707B0020E8F60C086C2B0020EC
:107B500090800020FCF60C0810B5144BB3F85E358D
:107B6000532B04461ED10AF009F99FED110A462055
:107B70005BF08AFE9FED0E0A49205BF085FE9FEDCB
:107B80000C0A4A205BF080FE46205BF05DFF492036
:107B90005BF05AFF4A205BF057FF2046BDE81040DB
:107BA000FFF778BABDE81040FFF7BAB8707B002045
:107BB00000000000082070470048704788F70C0854
:107BC0000048704794F70C080120704708B5024838
:107BD000FDF7B4FE012008BD702B0020014800F025
:107BE00061B900BF1477002010B50446FFF798F87C
:107BF0002046BDE81040FFF781BA00000120704721
:107C0000004870470CF80C080048704714F80C083E
:107C1000012070470120704710B5054B03F5E36460
:107C200003F5E1630FCB84E80F00012010BD00BF16
:107C3000707B002008B50B4800F5A04200F500530A
:107C40000321D3F8E03B93FBF1F3C2F81035F7F7CB
:107C50006FFF0448F7F708FFBDE808400148F7F751
:107C6000E7BC00BF702B002007207047004870471A
:107C700055DA0C08004870478CF80C080120704752
:107C800001207047012070477047000008B50023AD
:107C900003774362034883F097FD0348FBF7EAFA52
:107CA000012008BDF8540020702B002010B5194C9D
:107CB000D4F8C83BB3F9083023B9D4F8D43BB3F9AE
:107CC0000830F3B1002303774362D4F8C80B5AF0AD
:107CD000B9FB04F53E63D3ED007A0F48F8EEE77A7E
:107CE00027EE800ABDEEC00A10EE103AC0F810353B
:107CF000A0F5A040F7F71CFFBDE81040074803F0CF
:107D000003B8037F002BE0D0A4F50050F7F7CAFFBB
:107D1000F2E700BF704B0020707B0020702B00202A
:107D200070B54E4DDFED4E7A95F8E4339FED4D7A08
:107D30002DED048BB02606FB035393ED788A9FED5F
:107D40004A9A28EE278A05F5A353BDEEC88A93ED1B
:107D5000050AF8EEC87A044667EE897A97EE870A34
:107D600028F00AF9237FF0EE408A002B62D105F556
:107D70000053D3F8C83BB3F90830002B5AD128463A
:107D800009F04AF8002855D195F8E43395F82814FD
:107D900006FB035393F8C12100294BD1012A49D98D
:107DA00093ED777AF0EE087AB4EEE77AF1EE10FA16
:107DB00040DBDFED2E7AB0EEE80AB4EEE70AF1EE32
:107DC00010FA37D5636A93B386F040FA636AC01A33
:107DD000B0F5FA7F32D8237F002B3CD0244DA5F19B
:107DE000200696E80F0085E80F0094ED088AA5F1BB
:107DF00010013046B8EEC88A17F066FC28EE098AF2
:107E0000DFED1C0A284670EE200AB0EE480A17F093
:107E100001FD194B9FED190AD3F8A405BDEC048BA5
:107E200003682A4631469B6ABDE87040184786F0D1
:107E30000DFA6062636A002BCDD0C5E7104D84ED6A
:107E4000088A012323770023636205F110030FCB17
:107E500085E80F00BFE7BDEC048B70BD702B0020E0
:107E60000000C84235FA8E3C0AD7233CDB0FC93FDD
:107E70008882002000007A44705B0020000000002F
:107E800068820020036A0B60007F704705207047FE
:107E90000048704704F90C080048704714F90C08B2
:107EA0000120704738B54B4D2DED028BD5F8C80B2E
:107EB0009FED498A5AF0C6FAD5F8E03B07EE903AB2
:107EC000F8EEE77A05F5405427EE800AA5F5005054
:107ED000BDEEC00A10EE103AC4F81035F7F728FED0
:107EE000D5F8CC0B5AF0AEFAB5EEC00AF1EE10FAA6
:107EF000DABF05F6E433D3ED007AD5ED5A7A374888
:107F0000CBBF20EE270A20EE270A20EE080A28EE33
:107F1000400ABDEEC00A10EE103AC4F81435F7F767
:107F2000D3FD95ED5A7AD4F8140505F6E43327EE1F
:107F3000087AD3ED007A27EE888AFDEEC77A17EE2D
:107F4000902AFDEEC87A17EE901A28F0C9F8C4F806
:107F500014052248FDF77EFD20B1D4F814355B42AC
:107F6000C4F814351E4B93F8D43E63B195F9BC3177
:107F7000022B08D1002301214620C4F81035C4F893
:107F800014355BF0E5FF5AF06DF95F215BF02EF9D7
:107F9000E8B15BF0FBF8022819D194F8B534B3B915
:107FA00004F5916393ED007AD5ED827AB4EEE77A29
:107FB000F1EE10FA0BD5012384F8B534BDEC028B39
:107FC000084A0948BDE83840042152F023B8BDEC06
:107FD000028B38BD704B00200000C842702B00207F
:107FE000706B00201CF90C08F85E002010B50446E8
:107FF000FEF796FE2046BDE81040FFF77FB8000070
:1080000006207047004870479CF90C0800487047EC
:10801000ACF90C080120704701207047012070471F
:10802000012070477047000008B5044883F0CCFB7E
:108030000348FBF71FF9012008BD00BFF8540020DA
:10804000702B002038B50F4C04F50055D5F8C80B3F
:108050005AF0F8F905F53E62D2ED007AF8EEE77ACB
:1080600004F5A04327EE800A2046BDEEC00A10EEBC
:10807000102AC3F81025F7F75BFD2046BDE838400D
:1080800002F042BE702B00200F207047004870475E
:1080900024FA0C08004870472CFA0C08012070479D
:1080A0000120704701207047012070470120704770
:1080B0000120704730B5184B2DED028B002283F85C
:1080C000822303F51C53083305460FCB85B06C465D
:1080D00084E80F00114804F0CFFB90B1A86900F5C7
:1080E0007F702AF0EFFE0D48B0EE408A04F02CFCC1
:1080F000F0EE400A9FED0A0A204628EE000A17F02B
:1081000089FB00230748EB612146FBF717FE01209E
:1081100005B0BDEC028B30BD705B002040830020B9
:10812000E02E6542702B002038B5424C94F8B934EB
:1081300043B194F8E4382BB104F5FA60BDE8384057
:1081400008F066BAD4F8D434002B18DC3A48F7F7B4
:10815000A9FDD4F8D834002B29DC3748F7F784FC84
:10816000364890F88233002B46D00121A0F54050CC
:1081700009F000FABDE8384046205BF085BB86F088
:1081800065F8D4F8D434C01A40F6B7339842DDD835
:108190002B4DD4F8C804D5F8E02B514227F0A0FFAE
:1081A000C4F81005A5F50050F7F7C2FCD1E786F03A
:1081B0004DF8D4F8D834C01A40F6B7339842CCD82A
:1081C0001F4BDFED206A93ED5A7AD4F8CC0403F606
:1081D000E433D3ED007A27EE267A67EEA67ABDEE79
:1081E000C77AFDEEE77A17EE102A17EE901A27F0FD
:1081F00077FFC4F81405B3E7A0F5805090F9473134
:10820000012B04DCBDE838400B48F7F711BAD4F86D
:10821000E434002BF6D086F019F8D4F8E434C01A10
:1082200040F6B7339842EDD804F59C6494ED000A0B
:10823000A0E700BF707B0020702B0020705B002047
:10824000704B00200000C842D0ED077A0348FCEED6
:10825000E77A17EE903A99B202F032BF702B002005
:1082600084B010B503AC84E80E000B4821466F22A1
:10827000FBF7AAFC9DF80C1011F0040102D1204676
:1082800016F08AFF04482146FBF758FDBDE8104070
:10829000012004B0704700BF702B0020B0EEC00A70
:1082A000FDEEC07A38B54FF6FF7205460C4617EE64
:1082B000900A002127F014FF07EE900A002CF8EE38
:1082C000E77A054BC5ED077A14BF4FF0FF32012264
:1082D00083F8D02638BD00BF707B0020FEF79EBC1F
:1082E0000C2070470048704705FD0C080048704797
:1082F00052620E0808B50C48FCF76CFA0A480B49A4
:10830000FBF7E2F80848F6F709FE40B106484FF4DB
:108310008051F6F789FB10B10348FAF7ABFF02482A
:1083200002F0C8F9012008BD702B002088820020CF
:1083300008B50D48F7F7B6FC0B48F6F7EFFD50B15E
:1083400009484FF48051F6F76FFB20B1BDE80840B3
:10835000054802F0D9BC0448F7F786FBBDE80840A1
:108360000148F7F765B900BF702B002008B50A482F
:108370004FF48051F6F758FB38B108480022D0F886
:10838000281700F5E36016F075FEBDE808400248C6
:10839000002102F095BE00BF702B0020707B0020F2
:1083A000881A10B527F0C4FD104BD3F8CC2600284E
:1083B000B8BF4042002AB8BF524248F6A041B2FBC3
:1083C000F1F24FF47A7102FB011188420CDC93F850
:1083D0001827D20606D503F5E36403F5E1630FCB56
:1083E00084E80F00012000E0002010BD707B002019
:1083F00013B504468069019100F57F702AF062FD93
:10840000DFED0A7A20EE270A27F034FDDFED087A47
:10841000019920EE270A2046FDEEC07A17EE902A39
:1084200002B0BDE81040FFF7BBBF00BFE02E6542C1
:108430000000C84284B070B52DED048B86B00FAD3E
:1084400085E80E004E4CDFED4F8A0646D4F8A405B1
:1084500004F5005404F2E46393ED000A0368B0EEFF
:10846000C00A5B6A9847B4EEE80AF1EE10FAB0EE83
:10847000408A07DA012006B0BDEC048BBDE87040ED
:1084800004B070474049284617F02AF802A8CDEDFD
:10849000030A8DED020A2AF0E5FD04A88DED040A19
:1084A000B0EE480ACDED050A2AF098FC13A928463B
:1084B0008DED000ACDED010A17F012F802A88DED3E
:1084C000020ACDED030A2AF047FDB4EEE80AF1EE08
:1084D00010FACFDBB4EEC08AF1EE10FA9FED2B9AC2
:1084E000DFED2B8ADFED2B9A2BD802A869462AF004
:1084F00065FC04A88DED040ACDED050A2AF0E2FC26
:10850000684620EE098A2AF0DDFC94F9D03607EEA1
:10851000903AF8EEE77A28EE288AA7EEA90A27F023
:108520002BFD20EE090ABDEEC88A20EE280A18EEBF
:10853000101AFDEEC07A304617EE902AFFF730FF92
:1085400099E738EE400A38EE088A80EE080AAAF069
:10855000D5FA02A8B0EE408A2AF0B4FC94F9D036DD
:10856000F0EE007AB0EE697AA8EE677A07EE903AFC
:10857000F8EEE77AA7EE270A27F0FEFCC0E700BF77
:10858000705B00200000003478820020E02E6542FD
:108590000000C842DB0FC93F10B504460848F6F793
:1085A000BDFC20B92046BDE81040FEF737BB0448AB
:1085B0004FF48051F6F738FA0028F3D010BD00BF11
:1085C000702B0020002070470048704714FB0C08F7
:1085D000004870471CFB0C0800207047036993F8A3
:1085E000140118B1D3F8C402C0F380107047000022
:1085F00038B5154C05460021204608F0EBFD042057
:108600005BF042F90021204608F0EEFD13205BF0FC
:108610003BF90021204608F0F1FD2846FEF75CFDFD
:108620002046012108F0A6FF46205BF02DF9AB693A
:1086300004F5A044D3F8F831C4F81035AB69D3F889
:10864000FC31C4F8143538BD702B0020FEF722BD74
:10865000172070470048704794FB0C08004870478B
:108660009CFB0C08012070470120704701207047D7
:1086700010B50369002283F8402103690446D3F84A
:108680003C0103689B689847A36818687CF060FC0D
:10869000206904F06DFE0349A06910F04DFD012032
:1086A00010BD00BF007700201FB50B4C9FED0B0ADB
:1086B000D4F804086C302AF081FDFDEEE00ABDEE2E
:1086C000C00A10EE903AC4F8143510EE103AC4F80F
:1086D000103504B010BD00BF707B00209F0CB34567
:1086E00030B52DED028B83B0044685F0AFFD014619
:1086F000206900F50E700BF06FF938B1204603B019
:10870000BDEC028BBDE83040FEF70ABB206990F853
:108710004031BBB1012104F0B1FDA368DFED400A97
:108720001868036801215B6EB0EE600A9847206903
:1087300003F0FAF93B4803B0BDEC028BBDE83040D2
:10874000FFF792B8384DDFED398A022104F096FD2B
:10875000D5F8CC0B59F076FE2369D3ED390A93F99D
:108760003C2220EE200A002A60EE280A3FDD93F822
:10877000A032002B3BD0D5F8D40BCDED000A59F038
:1087800061FE2369D5F8C80B93ED3A8A20EE080AFA
:1087900020EE288A59F056FE236993ED381A20EE10
:1087A000410A20EE281ADDED000A2069CDED010A0C
:1087B0008DED001A03F0F4F9A36895F9DA21186831
:1087C0009DED001ADDED010A0368F0EE408A2AB340
:1087D0001B6CB0EE480A9847A36818680368F2EE6D
:1087E000040A5B6E0021B0EE680A9847A2E7D5F84C
:1087F000C80BCDED000A59F025FE2369D5F8D40B3E
:1088000093ED388A20EE080A20EE288A59F01AFEE5
:10881000236993ED3A1A20EE010AC2E7DB6BD8E731
:1088200000000000D8760020704B00200000C842F5
:10883000122070470048704714FC0C08004870472D
:108840001CFC0C0801207047012070470120704774
:1088500038B52DED028B43689FED1C8A1D680446D8
:10886000006904F0A7F9236993ED131AD3ED110AF7
:10887000434200EE103A21EE081A60EE880AB8EE84
:10888000C00A28467DF01EFD636820691D6804F05B
:1088900091F9236993ED131AD3ED110A434200EEC7
:1088A000103A21EE081A60EE880AB8EEC00A28468F
:1088B0007DF082FD9FED060A206903F061F92069D1
:1088C00005F016FFBDEC028B012038BD0000C84248
:1088D00000000000014800F051BE00BF4C780020AD
:1088E00013B5044600698830FAF7A2FB85F0AEFCA8
:1088F0000146206900F50E700BF06EF828B1204695
:1089000002B0BDE81040FEF70BBA206990F8403184
:108910003BB3012104F0B2FCA368DFED170A18682D
:108920000368B0EE600A5B6E01219847206903F08E
:10893000FBF863689FED100A18687EF0EDFE0F48A3
:10894000F6F7C6FB0D48F6F7B5FC20469FED0A0A80
:10895000FEF7C2FB2069883002B0BDE81040FAF78C
:1089600027BC074804F0EEFD2069019004F088F967
:10897000019806F0C9FAE2E700000000702B002021
:108980004083002014207047004870479AF50C0877
:108990000048704765620E0801207047002070474C
:1089A00070B504460E4800F03BF82369002583F8B3
:1089B0004051206904F0A2FF6069052103F058FDD1
:1089C000084826690221FAF727FF86EDB70A2369CE
:1089D000C3F848512369C3F84C51012070BD00BF52
:1089E00084780020702B0020014800F0C7BD00BF34
:1089F0004C780020014800F069B800BF847800205E
:108A0000132070470048704704FD0C080048704769
:108A10000CFD0C08012070470120704701207047B1
:108A200038B52DED028BDFED240AC3689FED238A54
:108A30000446B0EE600A186879F00CFEE368186826
:108A400079F0E6FE636820691D6804F0B3F82369D5
:108A500093ED131AD3ED110A434200EE103A21EEC2
:108A6000081A60EE880AB8EEC00A28467DF02AFC93
:108A7000636820691D6804F09DF8236993ED131A5B
:108A8000D3ED110A434200EE103A21EE081A60EECF
:108A9000880AB8EEC00A28467DF08EFC206905F0F1
:108AA00027FE256985F0D2FBC5F86C01BDEC028B71
:108AB00000230120E36138BD000000000000C8422F
:108AC000014800F05BBD00BF4C78002030B52DEDB3
:108AD000048B0446006985B08830FAF7A9FA38B1EA
:108AE000B74805B0BDEC048BBDE83040FFF7F8BED9
:108AF00085F0ACFB05462069294600F50E700AF0AA
:108B00006BFF38B1204605B0BDEC048BBDE83040AA
:108B1000FEF706B9206990F8403163B3012104F0F3
:108B2000ADFBA368DFEDA70A186803680121B0EE6A
:108B3000600A5B6E9847206902F0F6FF63689FED5C
:108B4000A10A18687EF0E8FDDFED9E0AE368B0EE4A
:108B5000600A186879F07EFDE368186879F058FEBD
:108B60009948F6F7B5FA984805B0BDEC048BBDE816
:108B70003040F6F79FBBC36A93F8CB3013B99348E4
:108B8000FFF74EFF206903F035F918B1E368186864
:108B900079F05CFD2369D3F86C31EB1AB3F5FA7FF9
:108BA0000BD9E368DFED870A1868B0EE600A79F048
:108BB00051FDE368186879F02BFE23699FED848AE4
:108BC000C3F86C510221206904F058FB63682069E6
:108BD0001D6803F0EFFF236993ED131AD3ED110A1B
:108BE000434200EE103A21EE081A60EE880A284649
:108BF000B8EEC00A7DF066FBD4E90335186879F059
:108C000093FDA368186803689B6EF0EE408A98474E
:108C100003AAF0EE400A02A9B0EE680A284603F063
:108C200003F8E368DDED030A18689DED020A79F0A8
:108C300011FD636818687DF037FB18B96368186820
:108C40007EF028FAE368634D1868012179F04CFF43
:108C5000E3681B689B68D3EDCF7AFDEEE77A05F5F4
:108C6000FA6017EE903AC5F81035E3681B689B6808
:108C7000D3EDD07AFDEEE77A17EE903AC5F81435C9
:108C800004F060FC2369D3F83C01036805F2145238
:108C90005B6B05F5A261984748B163681B68D3F820
:108CA0008823C3F89423D3F88C23C3F8982320692E
:108CB000DFED499A04F056FBD5F81035206907EE30
:108CC000903A012105F21453F8EEE78A93ED009AE9
:108CD00006F0B4F8A368B8EEC99A186820EE290A1D
:108CE000036868EEA98A29EE299ADB6A20EE081A41
:108CF00069EE080A28EE880A9847384BD3F8C02E48
:108D000003F634518A4248D1636993F86430062BE4
:108D10000AD8206903F0C2FC30B16069072103F072
:108D2000A7FB206904F0EAFD27480221FAF774FD49
:108D3000206903F08BF8636993F86430072BB0EE79
:108D4000408A08D12369D3F8C4329B0403D4A069B4
:108D5000012110F0B7FE6368B5EEC08AF1EE10FA9B
:108D60001868CCBF01210021B1EE480A7DF030FB2C
:108D7000206907F0DDFD206903F03AFF1248F6F79D
:108D8000A7F91148F6F796FA9FED0E0A2046FEF76E
:108D9000A3F905B0BDEC048B30BD03F684439A42C1
:108DA000206907D190F8423123B19FED060A02F005
:108DB000E7FEE0E7019003F063FF0198F7E700BFEB
:108DC0006878002000000000702B002084780020CC
:108DD0000000C842707B00200AD7233C706B002043
:108DE000152070470048704784FD0C080048704704
:108DF00084FD0C0801207047012070470020704757
:108E0000C369012B06D1044B93F8A409431E5842B1
:108E10005841704700207047707B00200E4BB3F91B
:108E20007A21B3F9AC3107EE102A07EE903AB8EE8A
:108E3000C77AF8EEE77AB0EEC77AF0EEE77AB4EEEA
:108E4000677AF1EE10FAC8BFF0EE477AB7EE080A7B
:108E500027EE800A704700BF704B00202DE9F041DB
:108E6000774C2DED048B94F814898AB00546B8F13F
:108E7000000F0CD03122A4F53371A4F5A04009F005
:108E80006DFF01200AB0BDEC048BBDE8F081012329
:108E9000C36104F5E16696E80F0004F5DF6787E833
:108EA0000F002B69D4F8F426B3F8C070DB6A52685F
:108EB00093F8A0306421022B17FB012740F0988023
:108EC00007EE907A3246B8EEE70AA4F5A04106A86C
:108ED000FBF74EF806A9304616F0F6FB2846F0EEF2
:108EE000408AFFF79BFF2B69B3F9C020D3ED310A0D
:108EF00001EE102AB3F9C220B0EE409A00EE102A1B
:108F0000B8EEC11A1A20B8EEC00A27F049F82B694A
:108F1000B3F9C030F4EEC98A07EE903AF1EE10FAD8
:108F200054BFF0EE686AF0EE496AB8EEE77AC8EE30
:108F3000A67A42460821A4F5A040B0EE408A67EE2A
:108F4000877AB4EE670AF1EE10FA48BFB0EE678A8E
:108F5000FAF728FCDFED3B7A38EE408AB4EEE78A78
:108F6000F1EE10FA1DDBC5F81C8096E80F0004F541
:108F7000E36585E80F0004F20C73D3ED008ADFEDA2
:108F8000327AF8EEE88A3046E8EE278A16F09CF846
:108F9000FDEEE87A024617EE901A284616F06AF8B7
:108FA0006FE7F4EEC98AF1EE10FA21D505AA414621
:108FB000304616F095F818B1059B9F42A8BF1F4692
:108FC00057F0A4FE064619EE100AF3F795FACDE91C
:108FD000020118EE900AF3F78FFA1C4ACDE900015E
:108FE0000621304651F016F86869032103F040FA73
:108FF00039461748FAF772FF286903F0C5FC15488F
:1090000005AA002116F06CF898B1134806AA0021B1
:1090100016F066F868B1DDE905316A698B4292F8AD
:109020002010D4BF0023012363F3000182F8201035
:1090300027E76A69D4F80C37D4F81C17EEE700BFAD
:10904000707B0020000000340000C8428CFD0C083A
:10905000702B00207882002088820020014800F0D8
:109060008DBA00BF4C780020F0B52DED028B99B081
:10907000044685F0EBF80146206900F50E700AF011
:10908000ABFC054638B1204619B0BDEC028BBDE8FB
:10909000F040FDF745BEE36983B1012B00F01E816E
:1090A000A048F6F715F89F48F6F704F99D4819B05F
:1090B000BDEC028BBDE8F040F6F766BC9FED9A8AE6
:1090C00060688DED098A8DED0A8A8DED0B8A8DED34
:1090D0000C8A0BAA09A901230068944D7DF008F8B9
:1090E0002069B0EE480A03F00DF963681B68D3ED00
:1090F000CF7AFDEEE77A05F5FA6017EE903AC5F8FB
:10910000103563681B68D3EDD07AFDEEE77A17EE71
:10911000903AC5F8143504F015FA2369D3F83C01E8
:10912000036805F214525B6B05F5A261984748B1DC
:1091300063681B68D3F88823C3F89423D3F88C237F
:10914000C3F89823206904F013F9A36820691E6806
:109150003368DF6AD5F8103507EE903AD5F8143544
:10916000F8EEE78A07EE903AF8EEE70ACDED050A49
:1091700005F0D8F8DDED050AB0EE401A3046B0EE45
:10918000680AB8472069C36B93ED070A02F0F8FC40
:10919000206903F02DFD63688DED0D8A8DED0E8A3B
:1091A0008DED0F8A18680FA97DF0F4FA0D9B1493CA
:1091B0000E9B159302220F9B169314A910A816F06C
:1091C000F9FA5B4907AA10A816F00AF848B1DFEDD2
:1091D000597A9DED077AB4EEE77AF1EE10FAFFF6D0
:1091E0005FAF0123E36105F5E1630FCB05F5DF66B2
:1091F00086E80F00D5F8F43622695B68B2F8C060E3
:109200004849642216FB023607EE906A4A4AB8EED5
:10921000E70A14A8FAF7ACFE474814A916F054FA66
:109220002046B0EE408AFFF7F9FDB4EEC08AF1EEB9
:1092300010FAF0EE408A21D53D4808AA002115F029
:109240004FFF18B1089B9E42A8BF1E4657F05EFD17
:10925000074618EE900AF3F74FF9CDE9020118EE30
:10926000100AF3F749F9354ACDE9000106213846DD
:1092700050F0D0FE6069032103F0FAF83146294826
:10928000FAF72CFE206903F07FFB294907AAA1F118
:10929000100015F0A5FF636988B19DED077ADFED39
:1092A000257A93F82020B4EEE77AF1EE10FAACBFFD
:1092B0000121002161F3000283F82020F0E6D5F8B7
:1092C0000C27D5F81C178A4293F82010D4BF00222F
:1092D000012262F3000183F82010E1E6206906F024
:1092E0007DF8636993F86430042B08D90F48D0F8EF
:1092F000F4362A46596800F5E36015F0BBFE636951
:1093000093F86430032B02D9206907F051FB2369DD
:1093100093F8D431013B012B3FF6C2AE0148F6F77A
:1093200009F8BDE6702B002000000000707B0020D3
:109330008882002000000034788200208CFD0C0818
:1093400030B5C369012B85B004D1414C94F8A439E0
:10935000012B04D005B0BDE83040FDF75FBCA4F59B
:109360004053DFED3C6AB3F97A219FED3B0A07EEEB
:10937000102AB3F9AC2107EE902AB8EEC77AF8EEBE
:10938000E77AB4F99028B0EEC77AF0EEE77AB4EE57
:10939000677A00EE902AF1EE10FAC8BFF0EE477A35
:1093A000B8EEE07AD3ED7A0A03F6A84270EEC70A67
:1093B00092ED007A27EE267AF5EEC00AF7EE006A03
:1093C000F1EE10FAB4EEE67A48BFDFED230AF1EED3
:1093D00010FAD8BFB0EE667AF3EE046A77EEA71AF9
:1093E00067EEA67AC0EE876A04F5936204F5E3643B
:1093F0006D4693ED557A92ED001AB0EE612AA6EE15
:10940000872AF4EE427AF1EE10FA48BFB0EE672AEE
:10941000F4EE421AF1EE10FAC8BFB0EE612A26F05F
:10942000F1FC94E80F0007EE901A9FED0C7AF8EE2D
:10943000E77A85E80F00E0EE077A09482946FDEE55
:10944000E77ACDED017AF9F71FFF05B030BD00BF17
:10945000707B00209A99193F000000000000C8426C
:10946000702B002011207047004870471CFE0C082C
:109470000048704728FE0C08012070470120704703
:1094800001207047012070470369002283F84021C2
:1094900001207047164B03F6382292ED007AB3F99B
:1094A000D827D3F80C09B5EEC07AF1EE10FA07EE22
:1094B000902AC8BFDFED0F6AF8EEE77ACABF27EE41
:1094C000267A20EE270A27EE000A67EEA07ABDEE84
:1094D000C00AFDEEE77A10EE102AC3F8102517EE49
:1094E000902AC3F814250368034A5B6B111F1847C1
:1094F000707B00200000C842848000201D49DFED01
:109500001E6AB1F9D827A1F54050F5EEC00AD0F88F
:10951000E03B9342A8BF134607EE903AF1EE10FAF3
:10952000F8EEE77AD6BF00F6E43090ED5A7A90ED87
:10953000007A27EE800A07EE902ACCBF27EE267A23
:1095400027EE667AF8EEE77ABDEEC00AB4EEE77A67
:10955000F1EE10FA58BFB0EE677A60EE870A10EEAF
:10956000103AFDEEE00AC1F8103510EE903AC1F85D
:1095700014357047707B00200000C84237B52B4C73
:10958000D4F8C83BB3F908201B8B07EE102A07EE6E
:10959000903AD4F8CC3BB8EEC77AB3F908201B8BCD
:1095A000F8EEE77A054687EE270A214807EE102AEB
:1095B00007EE903AB8EEC77AF8EEE77A8DED010A39
:1095C000C7EE270ACDED000A09F0B6FFDDED000A6F
:1095D0009DED010A28B1284603B0BDE83040FFF7F1
:1095E00059BF04F54053D3F8942A520405D42846B1
:1095F00003B0BDE83040FFF781BFB3F9D82707EECD
:10960000902AF8EEE77A27EE800A67EEA00ABDEE10
:10961000C00AFDEEE00A10EE102AC3F8102510EE85
:10962000902AC3F8142503B030BD00BF704B002052
:109630007885002010B5044684F008FE01462069B4
:1096400000F50E700AF0C8F920B12046BDE81040C0
:10965000FDF766BB114803F075FF206990F9D03023
:109660004BB102F027FA0E48F5F732FDBDE8104085
:109670000B48F5F71FBE02F093FA206905F0FEFBD8
:109680000748F5F725FD0648F5F714FE20469FED3F
:10969000050ABDE81040FDF71FBD00BF4083002054
:1096A000702B0020000000000B207047004870471E
:1096B00042010D0800487047A0FE0C0801207047C9
:1096C00001207047012070470020704738B53048AE
:1096D000F6F7E8FA2E48F6F7C7F92D48F5F7A8FF90
:1096E0002B481021F5F7A0F9E0B12A4AD2F80C373F
:1096F000D2F81C279342D4BF00230123254C94F8B1
:10970000802772B973B304F5E1630FCB04F5DF650D
:1097100085E80F00A4F5A040F9F7A8FF012384F81D
:10972000803738BD1C4AB2F9AC1B0029F9DD02F5BF
:1097300040529FED1A7AD2F80C37D2F8FC269B1AC9
:1097400007EE903AF8EEE77A67EE877A07EE101A9E
:10975000B8EEC77AF4EEC77AF1EE10FACCBF012367
:109760000023CBE7A4F54053642193F91822D4F8E1
:10977000100512FB01F2D3F8E01B8A42A8BF0A468B
:109780005142C3F8E02B26F0ABFCC4F81005C8E743
:10979000702B0020707B0020704B00200AD7233CE8
:1097A000F0B5304C2DED028B04F5E165074695E8E8
:1097B0000F0004F5DF6686E80F0083B0A4F5A04033
:1097C000F9F72CFD0146A4F5A040FAF787FBA4F5B4
:1097D0008052002384F88037C2F8E83E94F8E438D9
:1097E000D3B394F814393BB13122A4F53371A4F505
:1097F000A04009F0B3FA2FE094F99E38032B03D16F
:109800002C22A4F52C71F2E7013BDBB2012B23D80B
:109810003B69DB6A93F8A030022B1DD104F5E361AC
:10982000284615F051FFA4F52C70B0EE408AFFF7E2
:10983000F5FAB4EEC08AF1EE10FA0DD501AA0121B5
:10984000284615F04DFC38B1B4F89038642213FB6B
:1098500002F3019A9342D3DC012003B0BDEC028BEA
:10986000F0BD00BF707B002038B52DED028B244D7C
:1098700095F99E38012B03D00020BDEC028B38BD3A
:10988000A5F54053B3F9AC41002CB8BF6442A4B273
:109890002CB9B3F97A41002CB8BF6442A4B2194B79
:1098A000D3F8A40503689B6B984730B11649174855
:1098B000272209F053FA0120DFE7154AA2F120011F
:1098C00001F1100015F06CFE0028EFD1114805F5EC
:1098D000936595ED008A03F037F807EE904AF8EEAD
:1098E000E77AB4EEE70AF1EE10FA44BF07EE904AC9
:1098F000B8EE670AB4EEC08AF1EE10FABCD5D5E72F
:10990000707B0020705B0020C0780020702B00204E
:10991000888200204083002070B5464C94F8E438DB
:1099200088B0054683BB444DB5F9AC3183EAE37199
:10993000A1EBE37189B2002955D1404801F0C0FB89
:1099400094F8B634002B3ED195F98731022B52D1D1
:109950003B4D95F8F13E9BB13A4905F5A9502DF0E4
:109960002DF868B10123282205F54261A5F5804054
:1099700084F8593509F0F2F928BB002384F85935E9
:10998000012384F8B6341EE094F99E38022BA4F526
:1099900080561AD103AD284615F066FB04F5E36343
:1099A0000FCB85E80F0001A9A4F5A040FBF764F9EF
:1099B000D6F8E83E052B06D12722A4F52C71A4F594
:1099C000A04009F0CBF908B070BD84F03FFCD6F898
:1099D000C83EC01AB0F57A7FA5D92846FFF744FFE4
:1099E0000028A0D0EFE7002BB4BF4FF0FF330123D6
:1099F00084F8D036A1E7012B0CD1104801F090FA81
:109A000040B10E48F9F79CFD0028B8BF4042B0F5C0
:109A10007A7F9DDB95F98731042BD4D1084D95F8D9
:109A2000F13E002BACD0074905F5A9502DF042F8C6
:109A300097E700BF707B0020704B0020702B002048
:109A4000706B002078820020022070470048704729
:109A50001DFE0C08004870474C620E08034B0022A4
:109A6000C3F81025C3F81425704700BF707B002091
:109A700038B5094D04462846F5F72AFB2846F5F780
:109A800019FC2046F5F72EFC2846F5F77DFF204609
:109A9000BDE83840FDF732BB702B00200D20704729
:109AA0000048704788FF0C080048704790FF0C087A
:109AB000012070470120704701207047002380F883
:109AC000273080F83830012070470000014800211D
:109AD00001F0F6BA702B0020F0B5BA4CD4F8142778
:109AE000D4F810372DED088B1343D4F80C2713430B
:109AF00089B005460FD1B448F6F7D4F8B248F5F767
:109B0000B3FF9FEDB20A462009B0BDEC088BBDE85B
:109B1000F04059F0B9BE0FF029FD90F87C32DB0718
:109B2000E9D5B5F91C3095F8271009EE103AB5F9CA
:109B3000243008EE903AB8EEC99AF8EEE88A002987
:109B400040F0DD809FEDA2AA29EE0ABA0122FDEEC7
:109B5000CB7AA4F5A04017EE903AC4F88034F9F718
:109B600021FEA86900F57F700790B0EE408A29F0C9
:109B7000A9F9DFED987A20EE270A26F07BF90798FD
:109B8000F0EE409A29F0E8F9A4F5A040F0EE40AAE2
:109B9000FCF72CFD00287CD104F5E16696E80F0067
:109BA00005F1280787E80F0096E80F0004F5DF6746
:109BB00087E80F0004F5E36787E80F00D4F81C3747
:109BC000854807EE903AF8EEE77AF0EE680A77EE0D
:109BD0008B7AB0EE690AFDEEE77A17EE903AC4F898
:109BE0001C3715F017FE002384F8E93495F9263068
:109BF000754803EB830303EB83039B000121A4F867
:109C0000AE34F4F7ABFB94F8F874002F77D1734BB4
:109C10009FED737AB3F9503107EE903AF8EEE77A98
:109C200067EE877AF4EEE7AAF1EE10FA67DD57F0F7
:109C30006DF8064619EE900AF2F75EFCCDE90401D4
:109C400018EE900AF2F758FCCDE9020119EE100A5D
:109C5000F2F752FC634ACDE900010621304650F08C
:109C6000D9F984F0F3FAC4F86C74C4F8580484F099
:109C7000EDFA0123C4F8680429EE8A0A85F8273032
:109C800026F022F9BDEEC00A10EE103AC4F8703486
:109C900035E084F0DBFAD4F80835C01A42F21073CC
:109CA00098427FF679AFF0EE087AF4EEE7AAF1EE8B
:109CB00010FA7FF771AFBCEEC88A04F5E36718EEBF
:109CC000103A9BB208EE103AB8EEC88A04F5E16685
:109CD000B4EEC89AF1EE10FA48D857F017F8424A95
:109CE000062150F097F996E80F0087E80F0001234E
:109CF00085F827300321A4F5A040F4F72FFB324864
:109D00000BF0CAF830B130480321F4F727FB0023E9
:109D100085F82730D4F8FC34012B40F0B880D4F813
:109D20000C37EA6A9FED2AAA9B1A07EE903AD4F8FC
:109D300070340133F8EEE79A5ED0DFED2C7AE9EE6D
:109D40000A7AF4EEE79AF1EE10FA0ADA284905F1F8
:109D5000280015F0B9FCF4EEC08AF1EE10FA00F21A
:109D6000968019480321F4F7F9FA90E056F0CEFFF7
:109D7000204A062150F04EF996E80F0005F1280C14
:109D80008CE80F0096E80F0087E80F00D4F81C3726
:109D900007EE903A39EE488AF8EEE77AF0EE680A74
:109DA000E8EE0A7A3846B0EE690AFDEEE77A17EE79
:109DB000903AC4F81C3715F02DFD012185F82710C5
:109DC00099E700BF707B0020702B0020000000008E
:109DD0000000C842E02E654288820020704B0020BF
:109DE0009A99993ED9FF0C0898FF0C08000048C3C7
:109DF00078820020B4FF0C08B5F91E3007EE903AC7
:109E0000F8EEE77A05F1280667EE8A7AF4EEE79A2B
:109E1000F1EE10FA55DB4449304615F025FBDFED35
:109E2000437AB6EE008AA0EE278A96E80F00BDEED0
:109E3000C88A9FED3F0AB8EEC88A04F5E36728EEAA
:109E4000008A87E80F00F0EE680A3A48B0EE480A48
:109E500015F0E0FCD4F81C3707EE903AF8EEE77AFC
:109E600028EE0A0AE9EE0A7AFDEEE77A17EE903A52
:109E7000C4F81C3726F028F8BDEEC00A10EE103AE0
:109E8000C4F87034D4F8FC34012B3FF456AF2A48A0
:109E90000AF0E2FF18B128480321F4F75FFAD4F87A
:109EA000FC34012B17D124480AF06AFD22480AF03D
:109EB000B3FE214809B0BDEC088BBDE8F0400AF0C4
:109EC000C1BD1949304615F0FFFBF4EEC08AF1EE32
:109ED00010FAA0D9D6E795F838302BB9174862F0B8
:109EE00065F8012385F838301348F5F7DBFE124892
:109EF000F5F7BAFD1048F5F79BFB114890F884334D
:109F00006BB1002380F8843333220221A0F5405046
:109F100009B0BDEC088BBDE8F040FBF78DBF09B080
:109F2000BDEC088BF0BD00BF78820020A00CB345CB
:109F30000AD7233C88820020702B0020B84B0020D9
:109F4000705B002010B50446FCF7A0FF2046054BCF
:109F500040F8283B15F088F82046034944F09AFB66
:109F6000204610BD8C000D0824000D0818207047F5
:109F700000487047F4000D0800487047FC000D08C9
:109F800001207047012070470120704708B505483F
:109F9000F5F788FE0348F5F767FDBDE8084001487E
:109FA000F5F746BB702B002008B5064881F07AFE15
:109FB000BCEEC00A044810EE103A99B2BDE8084061
:109FC00001F07EB8F8540020702B002010B50D4C25
:109FD000D4F8703B002B12DDA4F50050FAF7FAFB21
:109FE000A4F5005000F066FB04F6881081F0A4FF91
:109FF00004F68810044981F03DFB012010BD0020CB
:10A00000FCE700BF704B002088820020F0B5274E8F
:10A01000D6F8C40E03688FB05B689847072837D01E
:10A020000A2809D0062805D10FF0A0FA90F87C3252
:10A03000DB071DD4012019E006F5805707F25C55B7
:10A040000FCD07AC0FC495E8070084E8070009AB03
:10A050000FCB01AC84E80F00D7F82437009305F547
:10A06000D6730ECB06F66840FEF7E4F90FB0F0BDEC
:10A070000FF07CFA00F51B700FC801AC84E80F00EC
:10A0800006F58055D5F82437009305F5E363E8E736
:10A0900007A906F6DC30FDF7F5FE0028CAD00799BF
:10A0A00006F66840FEF7A4F9E0E700BF706B0020F9
:10A0B000F0B585B00E4E0391144656F027FE06F516
:10A0C00080470546D7F8C40E026892689047039B04
:10A0D0000090084A284606214FF09CFFD7F8C41E7E
:10A0E0002246304605B0BDE8F04008F037BE00BF5C
:10A0F000702B002004010D082DE9F0432DED028B9B
:10A1000097B0002507466D4881F0F6FD0595069548
:10A1100007950FF02BFA05A90EF05EFF70B3684BA0
:10A1200093ED007AB5EEC07AA3F66C39F1EE10FA31
:10A1300009F5005427DBDDED067ADDED056A67EEF3
:10A14000A77A27EE077AE6EEA67AF4EEC77AF1EE62
:10A1500010FA18DDD4F8C40E03685B6898470A2823
:10A1600011D056F0D3FD574A06214FF053FF262257
:10A1700004F64C41A4F5804008F0F0FD17B0BDECAA
:10A18000028BBDE8F083504BD4F8C44E01959C423D
:10A1900002950395049503F5787817D104F63C14DD
:10A1A0000FCC08AE0FC694E8070086E8070011A898
:10A1B00014F05AFFB8F8B4150FAA08F5A4602BF0F4
:10A1C0002BFD78BB02950195049503959FED3F0A01
:10A1D00001A828F00FFE03A88DED080A9FED3B0AA9
:10A1E000CDED090A28F006FE34488DED0F0AB0EED9
:10A1F000401AF0EE601ACDED100A9DED080ADDED73
:10A20000090A81F0D3FC0628044618D10023C8F8B7
:10A21000CC3684F01BF82E49C8F81C0B274881F077
:10A2200029FAABE701A911A815F0CAF80028C9D08E
:10A2300003A90AA815F0C4F80028C3D0C6E709F698
:10A24000C82984F003F8DFED237A99ED008AD8F865
:10A250001C6B28EE278ADFED207AB4EEE78AF1EE58
:10A2600010FA0546384658BFB0EE678AFFF7CEFEB3
:10A2700048B9022C16D0BCEEC88AAD1B18EE103AB5
:10A280009D42FFF47BAF013C062C0ED8DFE804F0C2
:10A29000040A0D0D100D1300104924223846FFF753
:10A2A00007FF6BE70E492522F8E70E491622F5E76E
:10A2B0000D492622F2E70D490122EFE7F85400206C
:10A2C000DC56002020010D08907700200000C842D5
:10A2D0008882002000007A4400409C4646010D0818
:10A2E0005B010D0870010D0888010D089F010D0824
:10A2F000032070470048704724020D08004870474B
:10A3000030020D08F8B52A4D06460027A5F5405045
:10A31000A5F88073F5F70CFCB369A5F58052D3F866
:10A32000F811D2F8E03B994205F5005421DBC4F85E
:10A330001035B36992ED5A7AD3ED7F6A9FED1D6AAD
:10A34000F8EEE66A27EE067AF4EEC76AF1EE10FA46
:10A3500018DBBDEEC77A17EE103A1748C4F814356B
:10A36000FBF778FB20B1D4F814355B42C4F8143500
:10A37000F8BD5B429942DADD012385F88033C4F8E9
:10A380001075D6E702F6E432D2ED007A67EE867AEF
:10A39000F4EEE76AF1EE10FA93BFFDEEE77A0123DF
:10A3A00085F8813317EE903A88BF0023D5E700BFC8
:10A3B000705B00200000C842702B002070B50021A7
:10A3C0002DED028B04463448344D06F003FF32482D
:10A3D0000021F0EE408A06F007FF95F88033B0EEDA
:10A3E000408AD3B1B0EE680A042059F04DFA95F8CE
:10A3F000813393B3B0EE480A132059F045FA26484A
